S01800004762544D6F64756C65535733305765622E737265637E
S3150800800000000120CDE60008F5DE0008FDDE0008C8
S3150800801005DF00080DDF000815DF00080000000076
S315080080200000000000000000000000001DDF00083E
S3150800803029DF00080000000035DF000841DF0008DE
S315080080401DE700081DE700081DE700081DE70008F2
S315080080501DE700081DE700081DE700081DE70008E2
S315080080601DE700081DE700081DE700081DE70008D2
S315080080701DE700081DE700081DE700081DE70008C2
S315080080801DE700081DE700081DE700081DE70008B2
S315080080904DDF00081DE700081DE700081DE700087A
S315080080A01DE700081DE700081DE700081DE7000892
S315080080B01DE700081DE700081DE700081DE7000882
S315080080C01DE700081DE700081DE700081DE7000872
S315080080D01DE7000861DF000875DF000889DF000872
S315080080E01DE700081DE700081DE70008000000005E
S315080080F00000000000000000000000000000000072
S3150800810000000000000000001DE700081DE7000849
S315080081101DE700081DE700081DE700081DE7000821
S315080081201DE700081DE700081DE700081DE7000811
S315080081301DE700081DE700081DE700089DDF000889
S315080081401DE70008B1DF00081DE700081DE7000865
S315080081500000000000000000000000000000000011
S315080081600000000000000000000000000000000001
S3150800817000000000000000000000000000000000F1
S3150800818000000000000000000000000000000000E1
S3150800819000000000000000000000000000000000D1
S315080081A000000000000000000000000000000000C1
S315080081B000000000000000000000000000000000B1
S315080081C000000000000000000000000000000000A1
S315080081D00000000000000000000000000000000091
S30D080081E05FF8E0F166666666C9
S315080081E810B5054C237833B9044B13B10448AFF3DB
S315080081F800800123237010BD400200200000000003
S315080082085864010808B5034B1BB103490348AFF383
S31508008218008008BD000000004402002058640108D8
S31508008228034613F8012B002AFBD1181A01387047A0
S3150800823881F0004102E000BF83F0004330B54FEA01
S3150800824841044FEA430594EA050F08BF90EA020F6E
S315080082581FBF54EA000C55EA020C7FEA645C7FEA01
S31508008268655C00F0E2804FEA5454D4EB5555B8BF24
S315080082786D420CDD2C4480EA020281EA030382EA95
S31508008288000083EA010180EA020281EA0303362D27
S3150800829888BF30BD11F0004F4FEA01314FF4801CFA
S315080082A84CEA113102D0404261EB410113F0004F0C
S315080082B84FEA03334CEA133302D0524263EB4303C3
S315080082C894EA050F00F0A780A4F10104D5F1200E61
S315080082D80DDB02FA0EFC22FA05F2801841F10001BC
S315080082E803FA0EF2801843FA05F359410EE0A5F190
S315080082F820050EF1200E012A03FA0EFC28BF4CF0C1
S31508008308020C43FA05F3C01851EBE37101F0004576
S3150800831807D54FF0000EDCF1000C7EEB00006EEB83
S315080083280101B1F5801F1BD3B1F5001F0CD349080D
S315080083385FEA30004FEA3C0C04F101044FEA445264
S3150800834812F5800F80F09A80BCF1004F08BF5FEAEB
S31508008358500C50F1000041EB045141EA050130BDCB
S315080083685FEA4C0C404141EB0101013C28BFB1F5DD
S31508008378801FE9D291F0000F04BF01460020B1FA28
S3150800838881F308BF2033A3F10B03B3F120020CDAFB
S315080083980C3208DD02F1140CC2F10C0201FA0CF0D9
S315080083A821FA02F10CE002F11402D8BFC2F1200C3E
S315080083B801FA02F120FA0CFCDCBF41EA0C019040F4
S315080083C8E41AA2BF01EB0451294330BD6FEA04043D
S315080083D81F3C1CDA0C340EDC04F11404C4F1200228
S315080083E820FA04F001FA02F340EA030021FA04F33A
S315080083F845EA030130BDC4F10C04C4F1200220FA91
S3150800840802F001FA04F340EA0300294630BD21FACE
S3150800841804F0294630BD94F0000F83F4801306BF94
S3150800842881F480110134013D4EE77FEA645C18BF88
S315080084387FEA655C29D094EA050F08BF90EA020F1F
S3150800844805D054EA000C04BF1946104630BD91EA17
S31508008458030F1EBF0021002030BD5FEA545C05D11A
S315080084684000494128BF41F0004130BD14F5800459
S315080084783CBF01F5801130BD01F0004545F0FE41CD
S3150800848841F470014FF0000030BD7FEA645C1ABF02
S31508008498194610467FEA655C1CBF0B46024650EA39
S315080084A8013406BF52EA033591EA030F41F4002165
S315080084B830BD00BF90F0000F04BF0021704730B5EB
S315080084C84FF4806404F132044FF000054FF00001C0
S315080084D850E700BF90F0000F04BF0021704730B581
S315080084E84FF4806404F1320410F0004548BF404256
S315080084F84FF000013EE700BF42004FEAE2014FEAAB
S3150800850831014FEA02701FBF12F07F4393F07F4F85
S3150800851881F06051704732F07F4208BF704793F088
S315080085287F4F04BF41F40021704730B54FF460749B
S3150800853801F0004521F000411CE700BF50EA01029E
S3150800854808BF704730B54FF000050AE050EA010247
S3150800855808BF704730B511F0004502D5404261EBB7
S3150800856841014FF4806404F132045FEA915C3FF4F8
S31508008578D8AE4FF003025FEADC0C18BF03325FEA95
S31508008588DC0C18BF033202EBDC02C2F1200300FA46
S3150800859803FC20FA02F001FA03FE40EA0E0021FA6B
S315080085A802F11444BDE600BF70B54FF0FF0C4CF459
S315080085B8E06C1CEA11541DBF1CEA135594EA0C0F0B
S315080085C895EA0C0F00F0DEF82C4481EA030621EA46
S315080085D84C5123EA4C5350EA013518BF52EA033581
S315080085E841F4801143F4801338D0A0FB02CE4FF033
S315080085F80005E1FB02E506F00042E0FB03E54FF063
S315080086080006E1FB03569CF0000F18BF4EF0010E5A
S31508008618A4F1FF04B6F5007F64F5407404D25FEA56
S315080086284E0E6D4146EB060642EAC62141EA555109
S315080086384FEAC52040EA5E504FEACE2EB4F1FD0C4B
S3150800864888BFBCF5E06F1ED8BEF1004F08BF5FEAC9
S31508008658500E50F1000041EB045170BD06F000467B
S3150800866846EA010140EA020081EA0301B4EB5C0428
S31508008678C2BFD4EB0C0541EA045170BD41F4801120
S315080086884FF0000E013C00F3AB8014F1360FDEBF45
S31508008698002001F0004170BDC4F10004203C35DA21
S315080086A80C341BDC04F11404C4F1200500FA05F3A4
S315080086B820FA04F001FA05F240EA020001F0004245
S315080086C821F0004110EBD37021FA04F642EB0601BB
S315080086D85EEA430E08BF20EAD37070BDC4F10C04E5
S315080086E8C4F1200500FA04F320FA05F001FA04F2A9
S315080086F840EA020001F0004110EBD37041F1000195
S315080087085EEA430E08BF20EAD37070BDC4F120059F
S3150800871800FA05F24EEA020E20FA04F301FA05F207
S3150800872843EA020321FA04F001F0004121FA04F2AF
S3150800873820EA020000EBD3705EEA430E08BF20EA7F
S31508008748D37070BD94F0000F0FD101F000464000B9
S3150800875841EB010111F4801F08BF013CF7D041EA3B
S31508008768060195F0000F18BF704703F0004652003F
S3150800877843EB030313F4801F08BF013DF7D043EA10
S315080087880603704794EA0C0F0CEA135518BF95EAC6
S315080087980C0F0CD050EA410618BF52EA4306D1D14D
S315080087A881EA030101F000414FF0000070BD50EA6C
S315080087B8410606BF1046194652EA430619D094EAF6
S315080087C80C0F02D150EA013613D195EA0C0F05D1E0
S315080087D852EA03361CBF104619460AD181EA030134
S315080087E801F0004141F0FE4141F470014FF00000EC
S315080087F870BD41F0FE4141F4780170BD70B54FF087
S31508008808FF0C4CF4E06C1CEA11541DBF1CEA135506
S3150800881894EA0C0F95EA0C0F00F0A7F8A4EB0504E8
S3150800882881EA030E52EA03354FEA013100F08880DF
S315080088384FEA03334FF0805545EA131343EA1263A8
S315080088484FEA022245EA111545EA10654FEA00265D
S315080088580EF000419D4208BF964244F1FD0404F516
S31508008868407402D25B084FEA3202B61A65EB030572
S315080088785B084FEA32024FF480104FF4002CB6EB2F
S31508008888020E75EB030E22BFB61A754640EA0C00AF
S315080088985B084FEA3202B6EB020E75EB030E22BFEF
S315080088A8B61A754640EA5C005B084FEA3202B6EB30
S315080088B8020E75EB030E22BFB61A754640EA9C00EF
S315080088C85B084FEA3202B6EB020E75EB030E22BFBF
S315080088D8B61A754640EADC0055EA060E18D04FEA7D
S315080088E8051545EA16754FEA06164FEAC30343EA1D
S315080088F852734FEAC2025FEA1C1CC0D111F4801FEA
S315080089080BD141EA00014FF000004FF0004CB6E7E2
S3150800891811F4801F04BF01430020B4F1FD0C88BF81
S31508008928BCF5E06F3FF6AFAEB5EB030C04BFB6EB8C
S31508008938020C5FEA500C50F1000041EB045170BD7F
S315080089480EF0004E4EEA113114EB5C04C2BFD4EBAC
S315080089580C0541EA045170BD41F480114FF0000E30
S31508008968013C90E645EA060E8DE60CEA135594EAAC
S315080089780C0F08BF95EA0C0F3FF43BAF94EA0C0FAF
S315080089880AD150EA01347FF434AF95EA0C0F7FF424
S3150800899825AF104619462CE795EA0C0F06D152EA78
S315080089A803353FF4FDAE1046194622E750EA41065C
S315080089B818BF52EA43067FF4C5AE50EA41047FF46D
S315080089C80DAF52EA43057FF4EBAE12E74FF0FF3CD2
S315080089D806E000BF4FF0010C02E000BF4FF0010CA3
S315080089E84DF804CD4FEA410C7FEA6C5C4FEA430C1C
S315080089F818BF7FEA6C5C1BD001B050EA410C0CBF6B
S31508008A0852EA430C91EA030F02BF90EA020F0020CC
S31508008A18704710F1000F91EA030F58BF994208BF33
S31508008A2890422CBFD8176FEAE37040F001007047F0
S31508008A384FEA410C7FEA6C5C02D150EA013C07D147
S31508008A484FEA430C7FEA6C5CD6D152EA033CD3D092
S31508008A585DF8040B704700BF8446104662468C468C
S31508008A681946634600E000BF01B5FFF7B7FF0028BF
S31508008A7848BF10F1000F01BD4DF808EDFFF7F4FFE8
S31508008A880CBF012000205DF808FB00BF4DF808ED73
S31508008A98FFF7EAFF34BF012000205DF808FB00BF96
S31508008AA84DF808EDFFF7E0FF94BF012000205DF8B8
S31508008AB808FB00BF4DF808EDFFF7CEFF94BF01206D
S31508008AC800205DF808FB00BF4DF808EDFFF7C4FF66
S31508008AD834BF012000205DF808FB00BF4FEA410CAF
S31508008AE87FEA6C5C02D150EA013C0AD14FEA430C92
S31508008AF87FEA6C5C02D152EA033C02D14FF00000CF
S31508008B0870474FF0010070474FEA410212F500120C
S31508008B1815D211D56FF47873B3EB625212D94FEAAE
S31508008B28C12343F0004343EA505311F0004F23FA98
S31508008B3802F018BF404270474FF00000704750EAED
S31508008B48013005D111F0004008BF6FF000407047AA
S31508008B584FF00000704700BF4FEA4102B2F1E04308
S31508008B6824BFB3F5001CDCF1FE5C0DD901F0004CFE
S31508008B784FEAC0024CEA5070B2F1004F40EB83004E
S31508008B8808BF20F00100704711F0804F21D113F17A
S31508008B983872BCBF01F00040704741F480114FEAB3
S31508008BA85252C2F11802C2F1200C10FA0CF320FA3C
S31508008BB802F018BF40F001004FEAC1234FEAD32359
S31508008BC803FA0CFC40EA0C0023FA02F34FEA4303C3
S31508008BD8CCE77FEA625307D150EA01331EBF4FF04C
S31508008BE8FE4040F44000704701F0004040F0FE4067
S31508008BF840F40000704700BF80F0004002E000BF64
S31508008C0881F0004142001FBF5FEA410392EA030F61
S31508008C187FEA226C7FEA236C6AD04FEA1262D2EBAB
S31508008C281363C1BFD218414048404140B8BF5B42B0
S31508008C38192B88BF704710F0004F40F4000020F049
S31508008C487F4018BF404211F0004F41F4000121F05F
S31508008C587F4118BF494292EA030F3FD0A2F10102A9
S31508008C6841FA03FC10EB0C00C3F1200301FA03F1E7
S31508008C7800F0004302D5494260EB4000B0F5000F0A
S31508008C8813D3B0F1807F06D340084FEA310102F1C9
S31508008C980102FE2A51D2B1F1004F40EBC25008BF7B
S31508008CA820F0010040EA03007047490040EB000045
S31508008CB8013A28BFB0F5000FEDD2B0FA80FCACF146
S31508008CC8080CB2EB0C0200FA0CF0AABF00EBC25073
S31508008CD852421843BCBFD0401843704792F0000F61
S31508008CE881F4000106BF80F400000132013BB5E7B4
S31508008CF84FEA41037FEA226C18BF7FEA236C21D02A
S31508008D0892EA030F04D092F0000F08BF084670478E
S31508008D1890EA010F1CBF0020704712F07F4F04D15C
S31508008D28400028BF40F00040704712F100723CBF6F
S31508008D3800F50000704700F0004343F0FE4040F499
S31508008D48000070477FEA226216BF08467FEA236357
S31508008D580146420206BF5FEA412390EA010F40F442
S31508008D68800070474FF0000304E000BF10F000438E
S31508008D7848BF40425FEA000C08BF704743F0964375
S31508008D8801464FF000001CE050EA010208BF704790
S31508008D984FF000030AE000BF50EA010208BF704717
S31508008DA811F0004302D5404261EB41015FEA010C2C
S31508008DB802BF84460146002043F0B64308BFA3F124
S31508008DC88053A3F50003BCFA8CF2083AA3EBC25306
S31508008DD810DB01FA02FC634400FA02FCC2F1200225
S31508008DE8BCF1004F20FA02F243EB020008BF20F05C
S31508008DF80100704702F1200201FA02FCC2F12002C2
S31508008E0850EA4C0021FA02F243EB020008BF20EAB6
S31508008E18DC7070474FF0FF0C1CEAD0521EBF1CEAE4
S31508008E28D15392EA0C0F93EA0C0F6FD01A4480EAD2
S31508008E38010C400218BF5FEA41211ED04FF00063BB
S31508008E4843EA501043EA5111A0FB01310CF00040E7
S31508008E58B1F5000F3EBF490041EAD3715B0040EA0D
S31508008E68010062F17F02FD2A1DD8B3F1004F40EBDD
S31508008E78C25008BF20F00100704790F0000F0CF0B0
S31508008E88004C08BF49024CEA502040EA51207F3A74
S31508008E98C2BFD2F1FF0340EAC250704740F400004F
S31508008EA84FF00003013A5DDC12F1190FDCBF00F040
S31508008EB800407047C2F10002410021FA02F1C2F1EE
S31508008EC8200200FA02FC5FEA310040F1000053EA8A
S31508008ED84C0308BF20EADC70704792F0000F00F0D8
S31508008EE8004C02BF400010F4000F013AF9D040EADE
S31508008EF80C0093F0000F01F0004C02BF490011F472
S31508008F08000F013BF9D041EA0C018FE70CEAD1536F
S31508008F1892EA0C0F18BF93EA0C0F0AD030F0004CEF
S31508008F2818BF31F0004CD8D180EA010000F00040A3
S31508008F38704790F0000F17BF90F0004F084691F061
S31508008F48000F91F0004F14D092EA0C0F01D142029B
S31508008F580FD193EA0C0F03D14B0218BF084608D164
S31508008F6880EA010000F0004040F0FE4040F40000AE
S31508008F78704740F0FE4040F4400070474FF0FF0C41
S31508008F881CEAD0521EBF1CEAD15392EA0C0F93EA88
S31508008F980C0F69D0A2EB030280EA010C49024FEADA
S31508008FA8402037D04FF0805343EA111143EA101393
S31508008FB80CF000408B4238BF5B0042F17D024FF44B
S31508008FC8000C8B4224BF5B1A40EA0C00B3EB510F26
S31508008FD824BFA3EB510340EA5C00B3EB910F24BF0F
S31508008FE8A3EB910340EA9C00B3EBD10F24BFA3EB94
S31508008FF8D10340EADC001B0118BF5FEA1C1CE0D15C
S31508009008FD2A3FF650AF8B4240EBC25008BF20F00E
S31508009018010070470CF0004C4CEA50207F32C2BF62
S31508009028D2F1FF0340EAC250704740F400004FF0FF
S315080090380003013A37E792F0000F00F0004C02BF30
S31508009048400010F4000F013AF9D040EA0C0093F0FA
S31508009058000F01F0004C02BF490011F4000F013B54
S31508009068F9D041EA0C0195E70CEAD15392EA0C0FBC
S3150800907808D142027FF47DAF93EA0C0F7FF470AFF4
S31508009088084676E793EA0C0F04D14B023FF44CAF37
S3150800909808466EE730F0004C18BF31F0004CCAD1CC
S315080090A830F000427FF45CAF31F000437FF43CAF08
S315080090B85FE700BF4FF0FF3C06E000BF4FF0010C2A
S315080090C802E000BF4FF0010C4DF804CD4FEA40020C
S315080090D84FEA41037FEA226C18BF7FEA236C11D056
S315080090E801B052EA530C18BF90EA010F58BFB2EB09
S315080090F8030088BFC81738BF6FEAE17018BF40F089
S31508009108010070477FEA226C02D15FEA402C05D13C
S315080091187FEA236CE4D15FEA412CE1D05DF8040BC1
S31508009128704700BF844608466146FFE70FB5FFF754
S31508009138C9FF002848BF10F1000F0FBD4DF808ED0C
S31508009148FFF7F4FF0CBF012000205DF808FB00BFFD
S315080091584DF808EDFFF7EAFF34BF012000205DF857
S3150800916808FB00BF4DF808EDFFF7E0FF94BF0120A4
S3150800917800205DF808FB00BF4DF808EDFFF7D2FFA1
S3150800918894BF012000205DF808FB00BF4DF808EDE4
S31508009198FFF7C8FF34BF012000205DF808FB00BFB1
S315080091A84FEA4002B2F1FE4F0FD34FF09E03B3EBDE
S315080091B812620DD94FEA002343F0004310F0004F1E
S315080091C823FA02F018BF404270474FF00000704774
S315080091D812F1610F01D1420205D110F0004008BF13
S315080091E86FF0004070474FF0000070477BB972B9BE
S315080091F80029BEBF00204FF0004106E008BF00283E
S315080092081CBF6FF000414FF0FF3000F0D7B9ADF141
S31508009218080C6DE904CE002909DB002B1ADB00F0DF
S315080092284DF8DDF804E0DDE9022304B07047404252
S3150800923861EB4101002B1BDB00F040F8DDF804E088
S31508009248DDE9022304B0404261EB4101524263EB77
S3150800925843037047524263EB430300F02FF8DDF8E7
S3150800926804E0DDE9022304B0404261EB410170479E
S31508009278524263EB430300F021F8DDF804E0DDE928
S31508009288022304B0524263EB4303704753B94AB901
S31508009298002908BF00281CBF4FF0FF314FF0FF30E8
S315080092A800F08CB9ADF1080C6DE904CE00F006F8AB
S315080092B8DDF804E0DDE9022304B070472DE9F0473C
S315080092C8089D8E4604468846002B4AD18A42174688
S315080092D862D9B2FA82F64EB1C6F1200301FA06F847
S315080092E820FA03F3B74043EA0808B4404FEA174E92
S315080092F8B8FBFEF11FFA87FC0EFB118801FB0CF27E
S31508009308230C43EA08439A4209D9FB1801F1FF30AE
S3150800931880F0EB809A4240F2E88002393B449A1A78
S31508009328B2FBFEF00EFB102200FB0CFCA3B243EACC
S3150800933802439C4509D9FB1800F1FF3280F0D78013
S315080093489C4540F2D4803B44023840EA014000215B
S31508009358A3EB0C031DB10022F340C5E90032BDE8B2
S31508009368F0878B4205D90DB1C5E9000100210846E9
S31508009378F5E7B3FA83F1002946D1734502D3824249
S3150800938800F20881841A6EEB030201209046002D2C
S31508009398E5D0C5E90048E2E7002A00F09180B2FA6C
S315080093A882F6002E40F0A5808A1A0121030C4FEA9E
S315080093B8174E80B2BCB2B2FBFEFC0EFB1C2243EA77
S315080093C8024304FB0CF29A4207D9FB180CF1FF3842
S315080093D802D29A4200F2E380C4469B1AB3FBFEF215
S315080093E80EFB123302FB04F440EA03439C4207D9F6
S315080093F8FB1802F1FF3002D29C4200F2CD800246E9
S315080094081B1B42EA0C40A5E7C1F120068B4022FA4D
S3150800941806F71F432EFA06FA4FEA1749BAFBF9F870
S315080094280EFA01FE20FA06F309FB18AA1FFA87FCAA
S3150800943843EA0E0300FA01FE08FB0CF01C0C44EA8A
S315080094480A44A04202FA01F20AD93C1908F1FF3A7D
S3150800945880F09E80A04240F29B80A8F102083C4416
S31508009468241A98B2B4FBF9F309FB134403FB0CFC62
S3150800947840EA0444A44509D93C1903F1FF3080F0B1
S315080094888580A44540F28280023B3C4443EA084072
S31508009498A4EB0C04A0FB028C64454346E14664D35E
S315080094A861D05DB1BEEB030264EB090404FA06F663
S315080094B822FA01F31E43CC40C5E9006400214EE7B1
S315080094C8B1FBF2FC010C41EA0E4180B240EA0142C6
S315080094D83B46B1FBF7F138463C46B846BE46202619
S315080094E8A2EB080241EA0C4165E7014617E7104670
S315080094F82BE7C6F120012EFA01FCB7400EFA06FE44
S3150800950820FA01F141EA0E014FEA174EBCFBFEF8B4
S31508009518BCB20EFB18CC08FB04F90A0C42EA0C424A
S31508009528B04091454FEA104380B23ED9BA1808F1BF
S31508009538FF3C01D291451FD8A2EB0902B2FBFEF9FE
S3150800954809FB04F80EFB192A8AB242EA0A4242457E
S3150800955829D2BA1809F1FF31C2D24245C0D2A9F1B7
S3150800956802013A44BCE7C6459BD2B8EB02036CEB4A
S31508009578070C0138E14694E7A7EB09094A44B2FB08
S31508009588FEF9A8F1020C09FB04F8DBE703467DE7B8
S31508009598D04665E70846FAE63B44023A30E7ACF1B6
S315080095A8020C3B4419E749469AE7A2EB0902B2FBC3
S315080095B8FEF9C44609FB04F8C4E700BF704700BFB4
S315080095C880B584B000AF3B1D00221A605A609A60C5
S315080095D8184B194A1A60174B00229A60154B002235
S315080095E81A73144B00221A75124B4FF46022DA616B
S315080095F8104B00225A600F4B01221A610D4805F0DC
S3150800960811F90346002B01D002F06AFE08237B6095
S315080096180123BB600023FB603B1D1946054805F07E
S31508009628C5FB0346002B01D002F05AFE00BF1037CF
S31508009638BD4680BD5C0200200024014080B58AB082
S3150800964800AF786007F1180300221A605A609A601A
S31508009658DA607B681B681F4A934237D11E4B9B69A1
S315080096681D4A43F4007393611B4B9B6903F400730B
S315080096787B617B69184B9B69174A43F0040393611E
S31508009688154B9B6903F004033B613B69124B9B69C5
S31508009698114A43F0080393610F4B9B6903F00803CB
S315080096A8FB60FB680823BB610323FB6107F118030A
S315080096B819460A4806F0F4FE0323BB610323FB6137
S315080096C807F118031946064806F0EAFE00BF2837C8
S315080096D8BD4680BD00240140001002400008014034
S315080096E8000C014080B582B000AF03460A46FB71FC
S315080096F81346BB71FB79062B47D801A252F823F00B
S3150800970825970008359700084597000855970008D3
S31508009718659700087597000885970008BB791A4663
S315080097284FF480711D4807F056F82FE0BB791A46A2
S315080097384FF40071194807F04EF827E0BB791A4626
S315080097484FF48061154807F046F81FE0BB791A46BA
S315080097584FF40061114807F03EF817E0BB791A463E
S315080097684FF480510D4807F036F80FE0BB791A46D2
S315080097784FF400410A4807F02EF807E0BB791A4665
S315080097880821084807F027F800E000BFFB790649D2
S31508009798BA79CA5400BF0837BD4680BD00180140CB
S315080097A800080140001401408C02002080B483B0F0
S315080097B800AF0346FB71FB79034AD35C18460C379E
S315080097C8BD4680BC704700BF8C02002080B582B0B9
S315080097D800AF0346FB71FB79062B3BD801A252F86A
S315080097E823F000BF09980008159800082198000872
S315080097F82D980008399800084598000851980008D7
S315080098080221174806F0D0FF034624E0042114482D
S3150800981806F0CAFF03461EE08021124806F0C4FF78
S31508009828034618E08021104806F0BEFF034612E0FA
S3150800983810210E4806F0B8FF03460CE008210B482D
S3150800984806F0B2FF034606E00221064806F0ACFF1A
S31508009858034600E0002318460837BD4680BD00BF0A
S31508009868000801400018014000140140000C01409E
S3150800987880B500AF104805F02DFC00210020FFF741
S3150800988831FF00210120FFF72DFF00210220FFF7F5
S3150800989829FF00210320FFF725FF00210420FFF7F1
S315080098A821FF01210520FFF71DFF00210620FFF7EC
S315080098B819FF00BF80BD00BF5C02002090B587B0C5
S315080098C800AF78600C4B7B610C4B3B617969786813
S315080098D8FFF796F903461C4639697869FFF79AFA35
S315080098E8034619462046FFF749FB0346FB60FB6813
S315080098F818461C37BD4690BD00007A443211803B95
S31508009908B0B586B000AFF860B9607A603B60F868B1
S31508009918FEF7E0FD1CA3D3E90023FEF76FFF024616
S315080099280B4614461D46B868FEF7E6FD02460B4682
S3150800993820462946FEF738FE02460B4610461946C3
S31508009948FFF70AF903467B6179687869FFF714FC1B
S315080099580346002B01D00E4B10E079697868FFF7AB
S315080099684FF9034619467869FFF708FB034619466F
S315080099783868FFF74FFA03463B613B6918461837BC
S31508009988BD46B0BDAFF300800000000000FEAF4042
S31508009998000080BF80B588B000AF0346FB71FB792D
S315080099A8002B03D0082000F03BF802E0092000F05D
S315080099B837F8174805F00EF84FF0FF31144805F048
S315080099C8E3F8134805F0E6F9F861114805F0B0F828
S315080099D8FB69B3F57A6F01D9142315E00D4BBB6102
S315080099E80D4B7B610D4B3B61F8693B697A69B9692F
S315080099F8FFF786FF03461846FFF760FFF860F86822
S31508009A08FFF7CEFB03461BB218462037BD4680BD76
S31508009A185C020020333353400000A04000007A441B
S31508009A2880B586B000AF78607B68FB6001233B6130
S31508009A3803237B6107F10C031946064805F0B6F9B6
S31508009A480346002B01D002F04BFC00BF1837BD4671
S31508009A5880BD00BF5C02002080B500AF174B184ACE
S31508009A681A60164B08225A60144B00229A60134B48
S31508009A780022DA60114B4FF460221A610F4B4FF43B
S31508009A8880125A610D4B00221A760C4B01225A761F
S31508009A980A4B01229A76094B0122DA76074B0022ED
S31508009AA81A77064B01225A77044805F0C1FB034684
S31508009AB8002B01D002F014FC00BF80BD94020020E0
S31508009AC80064004080B500AF174B184A1A60164B59
S31508009AD810225A60144B00229A60134B0022DA604F
S31508009AE8114B4FF460221A610F4B4FF480125A61DA
S31508009AF80D4B00221A760C4B01225A760A4B012284
S31508009B089A76094B0122DA76074B00221A77064B12
S31508009B1801225A77044805F08BFB0346002B01D02F
S31508009B2802F0DEFB00BF80BDBC02002000680040D2
S31508009B3880B58EB000AF786007F1200300221A605E
S31508009B485A609A60DA607B681B68614A934253D107
S31508009B58604B1B6801335F4A13605E4B1B68012B19
S31508009B680BD15D4BDB695C4A43F00073D3615A4BF2
S31508009B78DB6903F00073FB61FB69574B9B69564A1F
S31508009B8843F020039361544B9B6903F02003BB61A0
S31508009B98BB6901233B6200237B620023BB6207F192
S31508009BA8200319464D4806F07BFC02233B62022334
S31508009BB87B620323FB6207F120031946474806F030
S31508009BC86FFC474B5B683B633B6B23F4C0433B63C3
S31508009BD83B6B43F0E0633B633B6B43F4C0433B6337
S31508009BE83F4A3B6B536000220021142006F0C3FA53
S31508009BF8142006F0DCFA67E07B681B68394A93424A
S31508009C0862D1354BDB69344A43F08063D361324B02
S31508009C18DB6903F080637B617B692E4B1B68013324
S31508009C282C4A13602B4B1B68012B0BD12A4BDB697B
S31508009C38294A43F00073D361274BDB6903F00073A5
S31508009C483B613B69244B9B69234A43F008039361AC
S31508009C58214B9B6903F00803FB60FB6820233B62E2
S31508009C6800237B620023BB6207F1200319461E48BE
S31508009C7806F016FC40233B6202237B620323FB6241
S31508009C8807F120031946184806F00AFC144B5B68C6
S31508009C987B637B6B43F0E0637B637B6B43F48003F6
S31508009CA87B630F4A7B6B5360002200213F2006F036
S31508009CB862FA3F2006F07BFA00220021412006F0CE
S31508009CC85AFA412006F073FA00BF3837BD4680BDF8
S31508009CD800640040E402002000100240001401401D
S31508009CE80000014000680040000C014080B400AF45
S31508009CF8084B00221A70074B00225A70054B00229F
S31508009D0862F06902DA7300221A7400BFBD4680BC85
S31508009D18704700BFE802002080B500AF1E4B5A788E
S31508009D281E4B1B789A4206D01B4B5A781B4B1A7047
S31508009D38194B00221A701A4B5B78002B03D0164B66
S31508009D4804225A7716E0174B1B7B002B03D0124BBD
S31508009D5807225A770EE0134B5B7B002B03D00E4B7A
S31508009D680A225A7706E00C4B9B7F002B02D10A4B36
S31508009D7800225A77084B5B7F0021184602F05EF9E5
S31508009D880346002B06D0044B5B7F1A46002106487B
S31508009D980AF068F900BF80BDE80200200703002022
S31508009DA808000020FC0900207064010880B500AF8F
S31508009DB80B4B10221A7000F01FFF0A4B42F2107262
S31508009DC81A80084B40F2DC525A80064B40F6B832E5
S31508009DD89A80044B40F69672DA8000BF80BD00BFB1
S31508009DE8080300202003002080B500AF0C4BD3F8E9
S31508009DF80730184603F000FF094B1A78094B5A71C1
S31508009E08074B5A78074B9A71054B9A78054BDA71BE
S31508009E18034BD3F80330034AC2F8013000BF80BDAC
S31508009E286000002028030020B0B584B002AFAB4B11
S31508009E3893F80A31022B40F0D180A84BD3F80031A9
S31508009E48B3F51C5F47D0B3F51C5F00F2C380B3F5C2
S31508009E58E05F00F0B680B3F5E05F00F2BB80B3F5CB
S31508009E68B85F00F0B280B3F5B85F00F2B380B3F517
S31508009E78B05F00F0AC80B3F5B05F00F2AB80B3F525
S31508009E88A85F00F0A680B3F5A85F00F2A380B3F533
S31508009E98985F00F08680B3F5985F00F29B80B3F56B
S31508009EA8885F6FD0B3F5885F00F29480B3F5805F5A
S31508009EB846D0B3F5805F00F28D80B3F5106F2CD0CD
S31508009EC8B3F5106F00F28680B3F5007F0BD0B3F5B3
S31508009ED8C06F18D07EE0824B01221A707F4B1A8811
S31508009EE8804B1A8076E0804B01221A707F4A7B4B9A
S31508009EF814461D460FCD0FC40FCD0FC40FCD0FC482
S31508009F082B68237066E07A4B01221A70794A734BDC
S31508009F1814460FCB07C423705CE0774B01221A70EE
S31508009F286E4B1B78AA2B03D1744B01221A7002E0D8
S31508009F38724B00221A70694B1A78714B1A7049E0ED
S31508009F4804F042FC03466F4A13606F4B634A92E873
S31508009F5803001860043319706B4B1B88FB806A4B27
S31508009F685B88C3F57A63BB80FB88684AA2FB032330
S31508009F78DB089AB2664BA3F80F20654BBA88A3F894
S31508009F881B2027E004F020FC03465E4A1360614B59
S31508009F98524A07CA03C31A705E4B9A795C4B9A7081
S31508009FA818E004F011FC0346564A13605A4B4B4A0C
S31508009FB892E8030018600433198002330A0C1A70F1
S31508009FC808E0564B01221A7004E000BF02E000BF01
S31508009FD800E000BF414B002283F80A2104F0F4FB95
S31508009FE802464F4B1B68D21A4E4B1B689A42C0F062
S31508009FF874844D4B1B78103B122B00F24F8401A238
S3150800A00852F823F059A00008A5A80008A5A8000832
S3150800A0187FA0000891A0000841A100088BA10008AC
S3150800A028FDA1000839A200088BA2000809A40008A7
S3150800A0380DA500089FA50008F5A5000867A600084D
S3150800A0481DA800085FA800087FA8000891A80008AE
S3150800A05800210020FFF746FB00210120FFF742FBFD
S3150800A068324B1B78032B40F01D8400F0C5FD00F029
S3150800A07851FE00F017BC142000F05CFC4FF4FA708F
S3150800A08800F010FD00F029BC144B93F80A31002B98
S3150800A09801D101F03DFAFA2000F004FD104B1B78B7
S3150800A0A8002B02D0152000F045FC0D4B1B78002B21
S3150800A0B840F0FA8300F0EAFC034642F21072934233
S3150800A0C840F2F2831A4800F07BFD114B09225A77B1
S3150800A0D81849042001F0C2F9E6E300BF6008002029
S3150800A0E81B03002030030020180300203403002037
S3150800A0F819030020680300201A0300201D03002006
S3150800A108AC030020B403002078030020CDCCCCCCC7
S3150800A118E802002088030020940300201C0300207E
S3150800A128100300201403002008030020C1030020A0
S3150800A138FCC0F0FCB8640108964B93F80A31002B6A
S3150800A14801D101F0E5F9FA2000F0ACFC924B5B7AF4
S3150800A158002B02D0162000F0EDFB00F097FC034612
S3150800A16842F21072934240F2A1834FF2F04000F097
S3150800A178D3FC8A4B0A225A778949042001F06EF9DA
S3150800A188ABE3844B93F80A31002B01D101F0C0F9EF
S3150800A198FA2000F087FC834B1B88834AA2FB03231B
S3150800A1A8DB089AB27D4BA3F80F207C4B002242F0BD
S3150800A1B80A02DA7600221A77784B0122DA75764B84
S3150800A1C8DB79052B02D1172000F0B4FB00F05EFC02
S3150800A1D8034642F21072934240F26A834FF2F04005
S3150800A1E800F09AFC6D4B0A225A777049042001F050
S3150800A1F835F972E3674B93F80A31002B01D101F060
S3150800A20887F9FA2000F04EFC644B5B7F002B03D0DD
S3150800A2184FF2F04000F080FC00F038FC034641F2AB
S3150800A2288832934240F24683182000F083FB41E3C4
S3150800A2385A4B0022DA7300221A74584B0022DA762F
S3150800A24800221A77554B0022DA7500F01FFC0346E0
S3150800A25841F2883293420BD94FF2F04000F05CFC89
S3150800A2684E4B0A225A775249042001F0F7F834E38C
S3150800A278494B9B7A002B40F01F83192000F05AFBA4
S3150800A2881AE3444B93F80A31002B02D1002001F057
S3150800A29853F9FA2000F006FC464B1B78002B60D0D1
S3150800A2A81A2000F047FB4449072001F0D7F8434B2A
S3150800A2B81B781A46414B5B781946404B9B780093A6
S3150800A2C80B463F49072001F0C9F83C4BDB781A468C
S3150800A2D83C49072001F0C2F8384B9B881A463A4988
S3150800A2E8072001F0BBF8354BDB881A4637490720A3
S3150800A2F801F0B4F8364A3749072001F0AFF82F4B72
S3150800A308DB681A463449072001F0A8F82B4B9B7CD2
S3150800A3181A462A4B5B7C1946284B1B7C03F2C173E9
S3150800A32800930B462D49072001F098F8234BDA7C51
S3150800A3389B8A1B0213431A462949072001F08EF8FF
S3150800A3481E4B9B7D1A462749072001F087F8264A9F
S3150800A3582649072001F082F8254A2649072001F0F0
S3150800A3687DF800F093FB034641F28832934240F2A7
S3150800A378A582104B1B78002B40F0A082074B0922B8
S3150800A3885A771D4800F01CFC1C49042001F066F8A1
S3150800A39894E200BF60080020FC090020E8020020BB
S3150800A3A8C864010830030020CDCCCCCCE864010889
S3150800A3B808650108180300202865010834030020E9
S3150800A3C834650108486501085C6501087465010873
S3150800A3D83C0300208C650108A4650108B8650108D6
S3150800A3E8E4650108F86501084C03002008660108B9
S3150800A3F85D03002018660108FCC0F0FD2C660108FC
S3150800A408B04B93F80A31002B02D1AA2001F094F830
S3150800A418FA2000F047FBAC4B1B78002B5AD01B20C0
S3150800A42800F088FAA949072001F018F8A84B1B88F4
S3150800A438A84AA2FB03235B099BB21A46A64907202A
S3150800A44801F00CF8A24B5B88A44AA2FB0323DB089D
S3150800A4589BB21A46A249072001F000F89C4B9B8834
S3150800A4689E4AA2FB0323DB089BB21A469D4907208E
S3150800A47800F0F4FF964BDB88984AA2FB0323DB0817
S3150800A4889BB21A469449072000F0E8FF904B1B7ABE
S3150800A498323B1A469449072000F0E0FF8C4BB3F884
S3150800A4A809309BB28D4AA2FB0323DB089BB21A46E6
S3150800A4B88E49072000F0D2FF854BB3F80B309BB2C4
S3150800A4C8864AA2FB0323DB089BB21A46884907205B
S3150800A4D800F0C4FF00F0DAFA034641F288329342E4
S3150800A4E840F2EE81784B1B78002B40F0E981814BCE
S3150800A4F809225A77804800F063FB8049042000F057
S3150800A508ADFFDDE16F4B93F80A31002B01D100F05E
S3150800A518DBFF022004F062F96A4B93F80A31002B34
S3150800A52801D100F0E7FFFA2000F0BCFA00F0AEFA15
S3150800A538034641F2883293420DD9714B1B78002B9A
S3150800A54809D16C4B09225A776E4800F039FB6E49D7
S3150800A558042000F083FF6D4B1B78002B03D01C20CA
S3150800A56800F0E8F9AEE100F091FA03464EF66022EB
S3150800A578934240F2A781624B1B78012B40F0A281D7
S3150800A5885C4B09225A775F4800F01AFB6049042099
S3150800A59800F064FF96E14B4B93F80A31002B02D181
S3150800A5A8002000F0DFFFFA2000F07CFA594B5B7AAE
S3150800A5B8002B02D01D2000F0BDF900F067FA03460B
S3150800A5C841F27072934240F27F81524B5B7A002BBC
S3150800A5D840F07A814FF2F04000F09EFA454B0A2285
S3150800A5E85A774D49042000F039FF6DE1354B93F849
S3150800A5F80A31002B02D1AA2000F0B4FFFA2000F095
S3150800A60851FA464B1B79002B00F060811E2000F09A
S3150800A61891F904F0D9F80346414A1360082000F076
S3150800A628A1FC3E4B5B88C3F57A637B803B4B1B8852
S3150800A6383B803B88294AA2FB0323DB089AB22D4BA9
S3150800A648A3F80F202B4B7A88A3F81B20294B012245
S3150800A658DA7503F0C7FA0346324A136036E104F09E
S3150800A668B3F802462E4B1B68D31AB3F5FA6F0BD903
S3150800A6784FF2F04000F050FA1E4B09225A772A4941
S3150800A688052000F0EBFE28E11A4B1B78012B02D1B6
S3150800A698264800F05DFA174B1B78032B02D123488E
S3150800A6A800F056FA224B5B78002B45D04FF2F04063
S3150800A6B800F032FA0F4B04225A771E49052000F09B
S3150800A6C8CDFE0AE160080020190300203C6601084F
S3150800A6D8680300201F85EB514C660108CDCCCCCC0D
S3150800A6E85866010864660108706601087C660108F0
S3150800A6F888660108E8020020FCC0F1FC9466010897
S3150800A7081A030020FCC0F4FCA46601081D030020F7
S3150800A718B4660108FC090020CC6601087803002005
S3150800A728B4030020B0030020E8660108F0F000042E
S3150800A738080000200C67010800F0F0FC0346032B0C
S3150800A7480BD04FF2F04000F0E7F96C4B08225A7725
S3150800A7586B49052000F082FEBFE00020FFF71AF9D2
S3150800A76803465A2B05DC0120FFF714F903465A2B32
S3150800A77814DD644800F0D0F9604B05225A770020AA
S3150800A788FFF708F903461C460120FFF703F90346B5
S3150800A79822465D49052000F061FE9EE0574B5B7F27
S3150800A7A8002B03D04FF2F04000F0B6F9574B4FF69E
S3150800A7B8FD72DA8003F016FA0246554B1B68D31A5F
S3150800A7C8544AA2FB03235B099AB2504B9A804B4B17
S3150800A7D8B3F815309BB2C3F57A639AB24B4B5A80D5
S3150800A7E8464BB3F813309BB21A46920013445B00E3
S3150800A7F89AB2464B1A80484B93F80A31002B05D172
S3150800A80800F0C4FE312000F04DF966E00A2000F099
S3150800A81849F962E00A2000F045F9384B0022DA7552
S3150800A8283E4B1B68184600F0BFFE00F02FF903469A
S3150800A83842F21072934206D93949042000F00EFEF6
S3150800A848384800F0BDF9384B1B78002B40D020203B
S3150800A85800F070F83CE0FA2000F024F900F0C4FE95
S3150800A86800F014F9034640F6C412934232D922205E
S3150800A87800F060F82EE02D4B1B68184600F0D4FE51
S3150800A888222000F057F828E0294B1B780A2B23D0FA
S3150800A898102000F04FF800F0AFF91DE0102000F086
S3150800A8A849F81AE000BF18E000BF16E000BF14E038
S3150800A8B800BF12E000BF10E000BF0EE000BF0CE0CA
S3150800A8C800BF0AE000BF08E000BF06E000BF04E0DA
S3150800A8D800BF02E000BF00E000BF00F01FFC03460F
S3150800A8E8032B03D1054B01229A7702E0034B00227A
S3150800A8F89A7700BF0837BD46B0BD00BFE8020020FA
S3150800A90828670108F0F00100486701089C03002041
S3150800A918B00300208988888860080020B8030020CA
S3150800A92870670108FDC0F0FC1C030020BC0300206A
S3150800A938C103002080B582B000AF0346FB71424AC6
S3150800A948FB79137003F040FF0346404A13603E4BF9
S3150800A9581B78102B03D13E49072000F07FFD3A4BA0
S3150800A9681B78132B03D13B49072000F077FD364B9C
S3150800A9781B78142B03D13849072000F06FFD324B9A
S3150800A9881B78152B03D13549072000F067FD2E4B98
S3150800A9981B78172B03D13249072000F05FFD2A4B95
S3150800A9A81B78192B03D12F49072000F057FD264B92
S3150800A9B81B781A2B03D12C49072000F04FFD224B90
S3150800A9C81B781B2B03D12949072000F047FD1E4B8E
S3150800A9D81B781C2B03D12649072000F03FFD1A4B8C
S3150800A9E81B781D2B03D12349072000F037FD164B8A
S3150800A9F81B781E2B03D12049072000F02FFD124B88
S3150800AA081B781F2B03D11D49072000F027FD0E4B85
S3150800AA181B78202B03D11A49072000F01FFD0A4B83
S3150800AA281B78212B03D11749072000F017FD064B81
S3150800AA381B78222B03D11449072000F00FFD00BF0D
S3150800AA480837BD4680BD00BF080300200C03002058
S3150800AA58806701088C670108A0670108B4670108C0
S3150800AA68CC670108DC670108F8670108146801085B
S3150800AA782868010840680108546801086C680108D4
S3150800AA88806801089C680108AC68010880B500AFB1
S3150800AA9803F09AFE0246024B1B68D31A184680BD75
S3150800AAA80C03002080B582B000AF786003F08CFEF6
S3150800AAB80346044A1360044A7B68136000BF0837D4
S3150800AAC8BD4680BD100300201403002080B582B05F
S3150800AAD800AF78600C4B5B7F002B03D00B4B002232
S3150800AAE81A7002E0094B01221A70094A7B6813603A
S3150800AAF8084B1B781F2B02D01F20FFF71BFF00BF30
S3150800AB080837BD4680BD00BFE8020020C003002004
S3150800AB18B80300200803002080B582B000AF78602B
S3150800AB28084B00221A70084A7B681360074B1B7883
S3150800AB381F2B02D01F20FFF7FDFE00BF0837BD46B2
S3150800AB4880BD00BFC0030020B8030020080300200A
S3150800AB5880B582B000AF7860084B02221A70084A9E
S3150800AB687B681360074B1B781F2B02D01F20FFF743
S3150800AB78E1FE00BF0837BD4680BD00BFC003002000
S3150800AB88B80300200803002080B500AF0A4B01224D
S3150800AB981A700A4B0022DA752220FFF7CBFE00202E
S3150800ABA801F006F900210020FEF79CFD002101208E
S3150800ABB8FEF798FD00BF80BDC0030020E80200200C
S3150800ABC880B582B000AF7860084B01221A707A689F
S3150800ABD80749042000F042FC064A7B6813602120D6
S3150800ABE8FFF7A8FE00BF0837BD4680BDC003002092
S3150800ABF8C0680108BC03002080B500AF03F0E4FD77
S3150800AC080346314A1360314B00221A70304B002232
S3150800AC181A70304B00221A702F4B00221A702F4BCD
S3150800AC2800221A702E4B00221A702E4B00229A7098
S3150800AC382C4B0022DA752B4B0022DA7600221A777B
S3150800AC48284B0022DA7300221A743122002126487A
S3150800AC5809F01AFA0D220021244809F015FA0522E6
S3150800AC680021234809F010FA05220021214809F095
S3150800AC780BFA02220021204809F006FA09220021C7
S3150800AC881E4809F001FA072200211D4809F0FCF9B7
S3150800AC98082200211B4809F0F7F9082200211A485A
S3150800ACA809F0F2F9134B4FF47A625A80114B4FF4B4
S3150800ACB8FA721A80154B00221A60154B00221A7070
S3150800ACC801F080F900BF80BDB403002018030020F6
S3150800ACD8190300201A0300201B0300201C03002068
S3150800ACE81D030020E8020020340300206803002022
S3150800ACF87803002080030020300300208803002002
S3150800AD08940300209C030020A4030020B00300201D
S3150800AD18AC03002080B500AF01210020FEF7E2FC55
S3150800AD2801210120FEF7DEFC1320FFF703FE00BF12
S3150800AD3880BD000080B500AF854B1B780C2B00F250
S3150800AD48F38001A252F823F085AD0008C3AD0008C8
S3150800AD589DAD00084FAE000809AE000831AF0008DF
S3150800AD6831AF000831AF0008A3AE000831AF0008BC
S3150800AD7805AF0008F7AE0008E9AE0008002001F0A4
S3150800AD8817F8744B1B78002B00F0D280012000F0CE
S3150800AD98E9F8CDE0002001F00BF86F4B5B7F002B3C
S3150800ADA802D1012000F0DEF86B4B1B78032B40F02C
S3150800ADB8C180002000F0C8FFBCE0002000F0F8FFC2
S3150800ADC8654B5B7F002B02D0022000F0CBF8624B64
S3150800ADD81B78032B02D1002000F0B6FF00F09EF97D
S3150800ADE80346032B40F0A8805B4B1B78032B00F027
S3150800ADF8A380042000F0B6F8002000F0D9FF9BE0F5
S3150800AE08002000F0D5FF544B1B78032B02D10020F5
S3150800AE1800F09AFF00F082F90346032B0FD14E4B38
S3150800AE281B78022B02D1032000F09CF84A4B1B78AA
S3150800AE38032B40F08380012000F094F87EE001207F
S3150800AE4800F090F87AE0012000F0B2FF434B1B7837
S3150800AE58222B1AD1424B1B78002B03D10B2000F06A
S3150800AE6881F812E03E4B1B78012B03D10C2000F029
S3150800AE7879F80AE03A4B1B78022B03D10A2000F02E
S3150800AE8871F802E00B2000F06DF8344B1B781E2B86
S3150800AE9856D1082000F066F852E0012000F088FF35
S3150800AEA82E4B1B78222B4DD12D4B1B78002B03D10B
S3150800AEB80B2000F057F845E0294B1B78012B03D1E6
S3150800AEC80C2000F04FF83DE0254B1B78022B03D1E8
S3150800AED80A2000F047F835E00B2000F043F831E087
S3150800AEE8002000F065FF0A2000F03CF82DE000205D
S3150800AEF800F05EFF0A2000F035F826E0002000F092
S3150800AF0857FF154B1B78032B02D1002000F01CFFB6
S3150800AF1800F004F90346022B16D1002000F048FF7A
S3150800AF28012000F01FF80FE0002000F01BF80CE0E5
S3150800AF3800BF0AE000BF08E000BF06E000BF04E063
S3150800AF4800BF02E000BF00E000BF00BF80BD00BF31
S3150800AF58C1030020F20C0020E802002008030020A4
S3150800AF68C003002080B582B000AF0346FB713D4A96
S3150800AF78FB7913703B4B1B78002B03D13A49072002
S3150800AF8800F06CFA374B1B78012B03D13749072099
S3150800AF9800F064FA334B1B78022B03D13449072097
S3150800AFA800F05CFA2F4B1B78032B03D13149072095
S3150800AFB800F054FA2B4B1B78042B03D12E49072093
S3150800AFC800F04CFA274B1B78052B03D12B49072091
S3150800AFD800F044FA234B1B78062B03D1284907208F
S3150800AFE800F03CFA1F4B1B78072B03D1254907208D
S3150800AFF800F034FA1B4B1B78082B03D1224907208B
S3150800B00800F02CFA174B1B78092B03D11F49072088
S3150800B01800F024FA134B1B780A2B03D11C49072086
S3150800B02800F01CFA0F4B1B780B2B03D11949072084
S3150800B03800F014FA0B4B1B780C2B03D11649072082
S3150800B04800F00CFA074B1B780D2B03D11349072080
S3150800B05800F004FA124AFB79537000BF0837BD4658
S3150800B06880BD00BFC1030020D8680108EC68010844
S3150800B078046901081C69010834690108506901084E
S3150800B0887069010890690108B0690108C86901086A
S3150800B098E0690108F8690108146A01082C6A0108B8
S3150800B0A8E802002080B582B000AF03F08DFB0246A7
S3150800B0B8164B1B68D31A632B24D903F085FB034662
S3150800B0C8124A136000F034F80346FB71104B1B78DC
S3150800B0D8FA799A4208D003F077FB03460D4A1360BB
S3150800B0E80B4AFB7913700EE003F06EFB0246094B18
S3150800B0F81B68D31AB3F5967F05D3054B1A78064B02
S3150800B1081A7000E000BF0837BD4680BDC40300209A
S3150800B118C8030020CC030020C203002080B400AF77
S3150800B128024B1B781846BD4680BC7047C2030020F0
S3150800B13880B582B000AF00F051F878602249786887
S3150800B148FEF706F80346002B08D020497868FEF76C
S3150800B1581DF80346002B01D0012331E01C49786805
S3150800B168FDF7F6FF0346002B08D01A497868FEF75C
S3150800B1780DF80346002B01D0022321E0154978680B
S3150800B188FDF7E6FF0346002B08D013497868FDF754
S3150800B198FDFF0346002B01D0032311E00E4978680A
S3150800B1A8FDF7D6FF0346002B09D04FF07E51786885
S3150800B1B8FDF7ECFF0346002B01D0042300E000232B
S3150800B1C818460837BD4680BD00005041000030418A
S3150800B1D86666E6409A9999400000404080B582B074
S3150800B1E800AF0320FEF71CFC0E4803F0F3FB6421AE
S3150800B1F80C4803F0C9FC0B4803F0CCFD78600948F5
S3150800B20803F096FC7868FDF7ADFD0346064918462F
S3150800B218FDF7B4FE03463B603B6818460837BD464B
S3150800B22880BD00BF5C020020CDCCE24280B500AFED
S3150800B238064B074A1A60054804F0D3FF0346002B55
S3150800B24801D001F04DF800BF80BD00BFD003002033
S3150800B2580030024080B485B000AF78607B681B6810
S3150800B268094A93420BD1094B5B69084A43F04003E4
S3150800B2785361064B5B6903F04003FB60FB6800BF3C
S3150800B2881437BD4680BC70470030024000100240A3
S3150800B29880B584B000AFF860B9607A607B689BB205
S3150800B2A81946B86800F006F87B6818461037BD4690
S3150800B2B880BD000080B485B000AF78600B467B80FF
S3150800B2C872B600BF0023FB8145E0284BB3F8043467
S3150800B2D89BB2B3F5806F18D3244BB3F802349BB2EC
S3150800B2E801335A42C3F30903C2F3090258BF53424A
S3150800B2F89AB21E4BA3F802241C4BB3F804349BB22B
S3150800B308013B9AB2194BA3F80424FB897A681344BB
S3150800B318164AB2F8002492B21978144B9954134B6A
S3150800B328B3F800349BB201335A42C3F30903C2F394
S3150800B338090258BF53429AB20C4BA3F800240B4B88
S3150800B348B3F804349BB201339AB2084BA3F8042421
S3150800B358FB890133FB81FA897B889A42B5D362B6A1
S3150800B36800BF00BF1437BD4680BC7047D80300200D
S3150800B37880B483B000AF72B600BF064BB3F8043486
S3150800B388FB8062B600BFFB8818460C37BD4680BCF2
S3150800B398704700BFD803002080B582B000AF72B6E8
S3150800B3A800BF2D4BB3F804349BB2002B02D162B60A
S3150800B3B800BF4EE0284BB3F80434FB80FB88802B8B
S3150800B3C801D98023FB80244BB3F802349BB2C3F51A
S3150800B3D88063BB80FA88BB889A4201D9BB88FB8000
S3150800B3E81D4BB3F804349BB2FA889A420CD11A4B0F
S3150800B3F8B3F802349BB21A46174B1344F9885022FD
S3150800B408184602F01BF90BE0134BB3F802349BB24B
S3150800B4181A46114B1344F9885122184602F00EF9B8
S3150800B4280D4BB3F802349AB2FB8813449BB2C3F3A4
S3150800B43809039AB2084BA3F80224074BB3F8043455
S3150800B4489AB2FB88D31A9AB2034BA3F8042462B6B5
S3150800B45800BF0837BD4680BDD80300200EB480B5A6
S3150800B46885B000AF0346FB71154AFB79137007F1DF
S3150800B4782003BB60BB68FA697E21124808F0C6FD3E
S3150800B488F860FB68002B01DAFB6812E0FB687D2B85
S3150800B49801DD7E23FB60FB680133094A0021D1548C
S3150800B4A8FB689BB202339BB219460548FFF702FFB1
S3150800B4B8FB6818461437BD46BDE8804003B0704798
S3150800B4C8E0070020E107002080B582B000AF02F04F
S3150800B4D889FB02463B461946104602F0C1FB3B4625
S3150800B4E8072206214FF4E06000F060FB00BF08372A
S3150800B4F8BD4680BD80B500AF044B082206214FF42F
S3150800B508006000F053FB00BF80BD00BF2003002089
S3150800B51880B582B000AF01233B7101237B710023FC
S3150800B528BB713B1D032206214FF4185000F03EFB61
S3150800B53800BF0837BD4680BD80B582B000AF034658
S3150800B548FB71074AFB791370054B082206214FF44D
S3150800B558807000F02BFB00BF0837BD4680BD00BFD2
S3150800B5682803002080B584B000AF0346FB71FB7939
S3150800B5783B7307F10C03012204214FF4206000F005
S3150800B58815FB00BF1037BD4680BD000080B500AF6B
S3150800B598044B082206214FF4905000F007FB00BF21
S3150800B5A880BD00BF9C03002080B584B000AF7860DA
S3150800B5B87B681B0EDBB23B727B681B0CDBB27B72AB
S3150800B5C87B681B0ADBB2BB727B68DBB2FB7207F1CE
S3150800B5D80803042204214FF4D05000F0E7FA00BF0C
S3150800B5E81037BD4680BD000080B500AF0B4BD3F8B9
S3150800B5F801300B4A53600A4B00229A700022DA700F
S3150800B608084B9B889AB2064B1A80054B07220621D7
S3150800B6184FF4E85000F0CAFA00BF80BD280300209E
S3150800B628A40300209C03002080B584B000AF78608E
S3150800B6387B681B0EDBB23B727B681B0CDBB27B722A
S3150800B6487B681B0ADBB2BB727B68DBB2FB7207F14D
S3150800B6580803042204214FF4F85000F0A7FA00BFA3
S3150800B6681037BD4680BD000080B58AB000AF07F127
S3150800B678140300221A605A609A60DA607D4B9B6947
S3150800B6887C4A43F0100393617A4B9B6903F01003D5
S3150800B6983B613B69774B9B69764A43F004039361A0
S3150800B6A8744B9B6903F00403FB60FB68714B9B6949
S3150800B6B8704A43F0080393616E4B9B6903F00803CD
S3150800B6C8BB60BB686B4B9B696A4A43F0400393614E
S3150800B6D8684B9B6903F040037B607B68654B9B69F5
S3150800B6E8644A43F020039361624B9B6903F0200385
S3150800B6F83B603B68002230215F4805F06CF8002261
S3150800B7084FF4F8515D4805F066F800224FF40041F9
S3150800B7185B4805F060F8002218215A4805F05BF8DE
S3150800B72800228021584805F056F802237B61002339
S3150800B738BB610023FB6107F114031946504804F05E
S3150800B748AFFE04237B610023BB610223FB6107F17B
S3150800B758140319464A4804F0A3FE30237B610123E3
S3150800B768BB610023FB6102233B6207F114031946F8
S3150800B778414804F095FE44F282037B610023BB61CD
S3150800B7880023FB6107F1140319463C4804F088FEB8
S3150800B7984FF4F8537B610123BB610023FB61022345
S3150800B7A83B6207F114031946344804F079FE4FF44E
S3150800B7B800437B610123BB610023FB6102233B62D3
S3150800B7C807F1140319462E4804F06AFE18237B610C
S3150800B7D80123BB610023FB6102233B6207F11403C3
S3150800B7E81946284804F05CFE80237B610023BB6168
S3150800B7F80023FB6107F114031946224804F050FE9A
S3150800B80818237B610023BB610023FB6107F114033E
S3150800B81819461D4804F044FE80237B610123BB6159
S3150800B8280023FB6102233B6207F1140319461648F5
S3150800B83804F036FE4FF440737B611223BB61032381
S3150800B8483B6207F1140319460F4804F029FE0F4B0B
S3150800B8585B687B627B6A43F0E0637B627B6A43F0E2
S3150800B86802037B62094A7B6A536000BF2837BD46D4
S3150800B87880BD00BF001002400010014000180140BA
S3150800B8880008014000140140000C01400000014076
S3150800B89890B5CDB040AF786007F10C0300221A6066
S3150800B8A85A6007F10C0307F114020021786804F0BE
S3150800B8B82BF80346002B40F05381BB699BB245F22F
S3150800B8C8F462934240F04C81BB691B0A03F47F4338
S3150800B8D8B3F56C4F13D0B3F56C4F00F20C81B3F582
S3150800B8E86B4F57D0B3F56B4F00F20581B3F5C85FB8
S3150800B8F800F0DD80B3F5F05F00F0B680FBE03B7B37
S3150800B908102B3ED17B7B1AB2BB7B1BB21B021BB228
S3150800B91813431BB29AB2944BA3F80421924B012203
S3150800B92883F80721FA7B904B83F806218E4B02226F
S3150800B93883F808218C4B93F808218B4B83F8092147
S3150800B948FB7C1A04BB7C1B0213437A7C13431A46F6
S3150800B958854BC3F80021844BB3F80431FF2B10D864
S3150800B968814C684604F110034FF48072194608F0B2
S3150800B97899FC94E80F0000F041F97B4B012283F803
S3150800B9880A213B7BFF2B40F0E680774B002283F8A1
S3150800B9980A21E0E0744B93F80A31012B40F0DD8068
S3150800B9A83B7B002B00F0DB803B7B222B00F2D78009
S3150800B9B86D4B93F807213B7B9A4240F0D0803B7B3E
S3150800B9C85A1E1346DB009B1A674A981807F10C0398
S3150800B9D801330722194608F065FC634B93F80731CB
S3150800B9E80133DAB2604B83F807215F4B93F80721D6
S3150800B9F85D4B93F806319A4211D95B4C684604F1B7
S3150800BA0810034FF48072194608F04CFC94E80F00AE
S3150800BA1800F03AF9544B022283F80A219FE0524B68
S3150800BA2893F80931002B07D04F4B93F80931013B9E
S3150800BA38DAB24D4B83F809214B4B93F80931002BA1
S3150800BA4840F08D80484C684604F110034FF4807224
S3150800BA58194608F027FC94E80F0000F0CFF8424B87
S3150800BA68022283F809217AE040490420FFF7F6FC08
S3150800BA783B7B19467B7B1846BB7BFA7B0192009376
S3150800BA8803460A463A490420FFF7E8FC3B7C194670
S3150800BA987B7C1846BB7CFA7C0192009303460A46CF
S3150800BAA834490420FFF7DAFCFFF76EF858E0324904
S3150800BAB80720FFF7D3FC3B7B19467B7B1846BB7BE5
S3150800BAC8FA7B0192009303460A462C490720FFF79A
S3150800BAD8C5FC3B7C19467B7C1846BB7CFA7C0192E4
S3150800BAE8009303460A4623490720FFF7B7FC24486C
S3150800BAF8FEF7ECFF34E01C4B93F80A31002B2FD1E4
S3150800BB087B6A9AB2184BA3F80421174B012283F8CB
S3150800BB180721154B012283F80621134B012283F8C6
S3150800BB280821114B002283F80921BB691B0A03F473
S3150800BB387F430D4AC2F800310B4B022283F80A21CB
S3150800BB48094BB3F804311A4607F10C031946064897
S3150800BB5808F0A8FB04E000BF02E000BF00E000BF51
S3150800BB6800BF3437BD4690BD60080020446A010806
S3150800BB78686A0108846A01089C6A0108B86A0108A3
S3150800BB88F0F0004080B500AF074803F071FDFDF7F7
S3150800BB9863FF00F0B3F8044803F026FD02210248C3
S3150800BBA803F0D3FF00BF80BD9402002080B58CB097
S3150800BBB800AFF8607B600B46FB721346BB72FB7AD4
S3150800BBC89A06FB681B02134343F4744343F056036F
S3150800BBD8FB6100237B6204233B62BB7ABB6207F1E5
S3150800BBE8140307F118017A68034803F08AFD00BFB1
S3150800BBF83037BD4680BD00BF9402002084B080B5AA
S3150800BC0882B000AF07F1100C8CE80F0011233B70C7
S3150800BC1897F818317B7097F818311A4697F816313D
S3150800BC28194697F81731CB1A01339A4208DD97F85F
S3150800BC38162197F81731D31ADBB20133DBB27B70BA
S3150800BC4897F81731BB70FF23FB70FF233B71D7F8B2
S3150800BC581031DBB27B71D7F810311B0ADBB2BB7126
S3150800BC68D7F810311B0CDBB2FB713B4608220721BB
S3150800BC784FF46C40FFF79AFF00BF0837BD46BDE88A
S3150800BC88804004B07047000084B080B582B000AF29
S3150800BC9807F1100C8CE80F0013233B70164BB3F80A
S3150800BCA80431DBB27B70144BB3F804311B0A9BB220
S3150800BCB8DBB2BB70104B93F80631FB70FF233B7160
S3150800BCC8D7F81031DBB27B71D7F810311B0ADBB213
S3150800BCD8BB71D7F810311B0CDBB2FB713B46082247
S3150800BCE807214FF46C40FFF761FF00BF0837BD46D0
S3150800BCF8BDE8804004B070476008002080B58AB067
S3150800BD0800AF00237B610023BB610123FB6100238D
S3150800BD183B6000237B600023BB600023FB60002395
S3150800BD283B6101233B623B461946064803F07CFB08
S3150800BD380346002B01D000F0D3FA00BF2837BD46CA
S3150800BD4880BD00BF9402002080B483B000AF0346CC
S3150800BD58FB71FB79002B14BF01230023DBB21A46BB
S3150800BD68044B9A70034B00221A7200BF0C37BD4663
S3150800BD7880BC70470800002080B500AF0A4B1B78C6
S3150800BD88002B05D08021094804F00EFD034609E07A
S3150800BD988021064804F008FD0346002B0CBF012342
S3150800BDA80023DBB2184680BD0400002000180140B5
S3150800BDB880B483B000AF0346FB71044AFB7913705D
S3150800BDC800BF0C37BD4680BC704700BF080000207E
S3150800BDD880B582B000AF02F0F7FC786000F004F98D
S3150800BDE8724B5B78002B40F0DD80FFF7C5FF0346F2
S3150800BDF8002B0CBF01230023FB706C4B1B78002B10
S3150800BE080CBF01230023BB70684B9B78FF2B04D11A
S3150800BE18FA78BB789A4200F0AD80644B9B78FF2B82
S3150800BE2809D1BB7883F00103DBB21A465F4B9A70D7
S3150800BE385E4B00221A725D4BDB78022B4AD0022B26
S3150800BE4800F3B180002B02D0012B2AD0ABE0584B67
S3150800BE581B78002B0FD0554B9B78012B05D1012257
S3150800BE682021544804F0B7FC14E001221021514857
S3150800BE7804F0B1FC0EE04D4B9B78012B05D101224D
S3150800BE8810214C4804F0A7FC04E001222021494867
S3150800BE9804F0A1FC454B0122DA70444A7B685360DA
S3150800BEA867E0424B5B687A68D31A434A128893421A
S3150800BEB85CD3002210213F4804F08DFC0022202183
S3150800BEC83C4804F088FC394B0222DA70374A7B680A
S3150800BED853604BE0354B5B687A68D31A312B47D9E0
S3150800BEE8FFF74AFF0346002B0CBF01230023FB700C
S3150800BEF8FB782E4A9278002A0CBF01220022D2B279
S3150800BF0893420CBF012300237B707B78002B09D052
S3150800BF18264BFF229A70254B0022DA70234B002203
S3150800BF281A7225E0214B1B7A0133DAB21F4B1A72B3
S3150800BF381E4B1A7A214B1B789A4213D31B4B0122A4
S3150800BF485A701A4A7B68D360184B00229A70174BA6
S3150800BF580022DA70154B00221A7219490420FFF7D5
S3150800BF687DFA05E0114B0022DA7001E000BF1AE0FD
S3150800BF7800BF18E00D4BDB78002B0CD000221021EF
S3150800BF880C4804F028FC002220210A4804F023FC67
S3150800BF98064B0022DA70054BFF229A70034B0022E3
S3150800BFA81A7200E000BF0837BD4680BD08000020A9
S3150800BFB8050000200010014006000020C76B010894
S3150800BFC8D46A010880B500AF054B00225A70044BA5
S3150800BFD80022DA6003490720FFF740FA00BF80BD50
S3150800BFE808000020E06A010880B500AF0A4B5B78B4
S3150800BFF8002B0FD0084BDB68002B0BD002F0E4FBB4
S3150800C0080246054BDB68D21A044B1B689A4201D3D1
S3150800C018FFF7D8FF00BF80BD08000020C86B0108DD
S3150800C02880B400AF034B044A9A6000BFBD4680BC83
S3150800C038704700BF00ED00E00080000880B485B0B6
S3150800C04800AF03460A46FB711346BB71BB791F2B23
S3150800C05801D900230EE00023FB73BB79084AD35C99
S3150800C068FA799A4201D00123FB73BB790449FA7914
S3150800C078CA54FB7B18461437BD4680BC704700BFB8
S3150800C0887009002080B584B000AF786002F09CFB88
S3150800C098B8607B68FB60FB68B3F1FF3F12D0104BB2
S3150800C0A81B781A46FB681344FB600BE0FEF7FAFF99
S3150800C0B8FFF78EFEFEF73EFEFDF7B6FE00F0F4FF2C
S3150800C0C801F000F902F080FB0246BB68D31AFA6849
S3150800C0D89A42EBD800BF00BF1037BD4680BD00BFE7
S3150800C0E87400002080B500AF0320FDF76FFB0346F8
S3150800C0F8002B02D1024B01221A7000BF80BD00BF77
S3150800C108E802002080B582B002AFFFF789FF02F087
S3150800C11803FB04F085FB00F073F8FFF7A5FAFDF7B3
S3150800C1284FFAFDF799FCFDF7CDFC01F05BF801F035
S3150800C138F1FF02F031F9FFF779F802F0D9F802F0C1
S3150800C14801F902F053F9FDF793FB00F08DFF4FF460
S3150800C158967002F043FBFDF729FE01F0A7F80023C5
S3150800C168012222490720FFF779F901F07BF8204BCD
S3150800C1781B889BB21A461F490720FFF76FF91C4B05
S3150800C1889B781A461C490720FFF768F9184B9B88BD
S3150800C1989BB21A46164BDB889BB21946144B1B8969
S3150800C1A89BB200930B4615490720FFF757F9FDF789
S3150800C1B81BFEFFF7E7FC00F07DFAFDF797FD00F098
S3150800C1C887FB00F023FC0A20FFF75CFF00F08EF8D7
S3150800C1D8FDF7A2FD00F00EFE0A20FFF753FFFFF752
S3150800C1E881FF3220FFF74EFF00BFE8E7F46A01082F
S3150800C1F8E80C0020086B01081C6B0108306B010865
S3150800C20880B59CB000AF07F13803382200211846DC
S3150800C21807F03AFF07F1240300221A605A609A6069
S3150800C228DA601A613B1D20220021184607F02CFF08
S3150800C2380523BB634FF480333B6404237B640123E3
S3150800C248BB640123FB644FF48033FB630223BB659D
S3150800C2584FF48033FB654FF4E0133B6602237B6695
S3150800C2684FF4C063BB664023FB6607F138031846DC
S3150800C27804F0A6FB0346002B01D000F031F80F2383
S3150800C2887B620223BB620023FB624FF480633B6335
S3150800C29800237B6307F124030221184604F0A6FE4F
S3150800C2A80346002B01D000F01BF803237B604FF4EC
S3150800C2B88073BB604FF40043FB603B1D184605F0CE
S3150800C2C88BF80346002B01D000F00AF8034B01222D
S3150800C2D81A6000BF7037BD4680BD00BF7000424275
S3150800C2E880B400AF72B600BF00BFFDE72DE9B043C2
S3150800C2F884B000AF2E4B00221A712E4B5B78082BA0
S3150800C30804D12B4B012283F8242003E0284B002272
S3150800C31883F8242002F058FAF860254B9B68FA68D7
S3150800C328D31ABB60224AFB689360224BD3F80330C2
S3150800C338BA6802FB03F3204AA2FB03239B097B6026
S3150800C3481B4BD3E90423796800200C46054612EBF3
S3150800C358040843EB0509164BC3E90489144BD3E9CA
S3150800C3680423164BA3FB0223DB0A114A9361104BDD
S3150800C37893F82430002B08D00D4B9A690C4BDB69CF
S3150800C388D31A0C4AC2F807300CE00A4B0022DA71B5
S3150800C39800221A7200225A7200229A72044B9B696A
S3150800C3A8034AD36100BF1037BD46BDE8B08300BF56
S3150800C3B890090020E8020020D34D6210C5B3A29167
S3150800C3C880B582B000AF0346FB71064AFB79D37184
S3150800C3D802F0FAF90346034A136100BF0837BD4657
S3150800C3E880BD00BFFC09002080B500AF02F0ECF95B
S3150800C3F80246024B1B69D31A184680BDFC09002061
S3150800C40880B584B000AF7860884B894A012178687E
S3150800C41803F07AFA0346002B40F00481844B5B68E4
S3150800C428BB603B7A002B40F0FC8002F0CDF903464E
S3150800C438804A1360BB7A03F03F03DBB2022B05D1AF
S3150800C4487D4B7A4A92E8030083E80300BB7A03F037
S3150800C4583F03DBB2042B19D1784B744A92E80300E0
S3150800C46883E80300754B1B791A46754BDA61734BDB
S3150800C4781A7A734B83F82020704BDA79704B83F855
S3150800C48821206E4B9A796E4B83F82220BB7A03F0EB
S3150800C4983F03DBB2062B23D16A4B644A92E80300B2
S3150800C4A883E80300674B5B781A46664B1B781B02C2
S3150800C4B813441A46634B9A60624BDB781A46614BFB
S3150800C4C89B781B0213441A465E4BDA605D4B5B7910
S3150800C4D81A465C4B1B791B0213441A46594B1A61B8
S3150800C4E8BB7A03F03F03DBB2082B05D1564B4F4AFC
S3150800C4F892E8030083E80300BB7A03F03F03DBB244
S3150800C508092B40F08F80514B484A92E8030083E88C
S3150800C51803004E4BDB791A464C4BDA604B4BDA680C
S3150800C5284A4B9B791B021343484AD360474BDA6840
S3150800C538464B5B791B041343444AD360434BDA687A
S3150800C548424B1B791B061343404AD3603F4BDB78A3
S3150800C5581A463E4B9A603D4B9A683C4B9B781B02A1
S3150800C56813433A4A9360394B9A68384B5B781B04ED
S3150800C5781343364A9360354B9A68344B1B781B0627
S3150800C5881343324A9360314B9B68314AA2FB032313
S3150800C5989B09FB812D4BDB682E4AA2FB03235B090B
S3150800C5A8BB81274AFB895380254ABB899380FB8927
S3150800C5B8132B8CBF01230023DBB21A46204B9A7231
S3150800C5C81F4B01221A721D4B1A791D4B9A711C4B67
S3150800C5D8DB79012B26D91A4B5A881F4BA3F8132047
S3150800C5E8174BB3F904309AB21B4BA3F815201A4B0C
S3150800C5F8B3F815309BB21A46174BB3F813309BB2EB
S3150800C60802FB03F3154A82FB03129210DB17D31AAF
S3150800C6181A46114BC3F80320094B9A7A0E4B1A7619
S3150800C62800E000BF1037BD4680BD00BF400A0020A5
S3150800C638240A0020200A0020B8090020C40900207E
S3150800C648FC090020D0090020E4090020EC09002094
S3150800C658D34D62101F85EB51E802002067666666AF
S3150800C66880B58AB000AF0E237B610023BB61012326
S3150800C678FB6100233B6000237B600023BB6000232B
S3150800C688FB6000233B6101233B6201233B610E23C8
S3150800C6987B623B461946064802F0C6FE0346002B4F
S3150800C6A801D0FFF71DFE00BF2837BD4680BD00BF75
S3150800C6B8BC02002080B500AF134802F0D9FFFDF789
S3150800C6C801FAFFF7CDFF104802F08EFF10210E4839
S3150800C6D803F03BFA242200210C4807F0D5FC0B4B43
S3150800C6E80022DA7102F070F80346084A1361074B0C
S3150800C6F847F230525A61054B00221A76002100206B
S3150800C70800F006F800BF80BDBC020020FC09002026
S3150800C71880B584B000AF03460A46FB711346BB7161
S3150800C72807F1080308220021184607F0ADFCFB7933
S3150800C738002B15D10D4B1B7A002B13D0BB79002B78
S3150800C7480CBF01230023DBB23B72F97907F1080312
S3150800C7581A22F02000F066F81420FFF793FC02E08E
S3150800C76800BF00E000BF1037BD4680BDFC090020A9
S3150800C77880B586B000AF0346FB710B46BB801346EF
S3150800C7887B8007F1080308220021184607F07CFC7D
S3150800C798FB79002B40D1BB88952B01D89623BB8003
S3150800C7A81F4B1B7E002B06D1BB88B3F5FA7F02D335
S3150800C7B840F2F313BB807B88642202FB03F37B6198
S3150800C7C8BB884FF47A7202FB03F33B617B691B0E45
S3150800C7D8DBB23B737B691B0CDBB27B737B691B0A79
S3150800C7E8DBB2BB737B69DBB2FB733B691B0EDBB23F
S3150800C7F83B723B691B0CDBB27B723B691B0ADBB2DB
S3150800C808BB723B69DBB2FB72F97907F108031C2294
S3150800C818F02000F007F800E000BF1837BD4680BDD5
S3150800C828FC09002080B58CB000AF3B600346FB715D
S3150800C8380B46BB7113467B71FB7987F82830BB79A1
S3150800C84887F829307B7903F03F03DAB297F82A305C
S3150800C85862F3050387F82A307B8D0A2262F3891367
S3150800C8687B850A2387F82F30BB6A7B610023FB6127
S3150800C8780423BB6108233B621EE0144803F010F842
S3150800C8880346002B0ED007F10C0307F110013A688E
S3150800C8980E4802F036FF034687F82E3097F82E30F2
S3150800C8A8002B0ED00120FFF7EDFB97F92F30DBB2EE
S3150800C8B8013BDBB287F82F3097F92F30002BDCDCE9
S3150800C8C800E000BF3037BD4680BD00BFBC0200206F
S3150800C8D880B582B000AF3B4600221A605A603B46D4
S3150800C8E804220021F020FFF79DFF1420FFF7CAFB5A
S3150800C8F83B4606220021F020FFF794FF1420FFF795
S3150800C908C1FB3B4609220021F020FFF78BFF1420C4
S3150800C918FFF7B8FB394BB3F81B309BB2384AA2FB72
S3150800C9280323DB089BB21A46344BB3F813309BB281
S3150800C93802FB03F31A46334B5B699A4211D9314B0A
S3150800C9485A6913469B0013445B001A462B4BB3F8E7
S3150800C95813309BB2B2FBF3F39AB2284BA3F8112013
S3150800C96806E0264BB3F81B309AB2244BA3F81120DD
S3150800C978224BB3F811309BB2B3F57A7F08D91F4B0F
S3150800C988002262F017025A74002242F003029A74CF
S3150800C9981A4BB3F811309BB21A46184BB3F80F3036
S3150800C9A89BB202FB03F3184A82FB03129210DB17A9
S3150800C9B8D31A1A46114BC3F80B20124B5B7A002B75
S3150800C9C818D00E4BB3F80F309BB20C4AB2F81120A8
S3150800C9D892B219460020FFF7CBFE1420FFF752FB48
S3150800C9E8064BB3F813309BB2B3F5F57F02D9054B5E
S3150800C9F801221A7600BF0837BD4680BDE802002026
S3150800CA08CDCCCCCCFC0900206766666698B500AF25
S3150800CA1801F0DAFE0246B44B1B68D31AB3F5FA7F5F
S3150800CA2820D9B24B00221A72B04B00229A72B04B28
S3150800CA3800221A71AE4B00221A72AD4B0022DA7127
S3150800CA48AB4B00229A71AB4B00229A60A94B002285
S3150800CA58DA60A84B00221A61A74B0022DA60A64BB7
S3150800CA6800229A60A14B1B7A002B03D09F4B1B7898
S3150800CA78002B0CD1A14B0022DA7400221A759F4BA1
S3150800CA8800225A7500229A759C4B00221A769B4BEF
S3150800CA989B7F002B0CD001210420FCF723FE01F014
S3150800CAA893FE0346964A1360904B01221A7010E0CB
S3150800CAB801F08AFE0246924B1B68D31A4EF660228C
S3150800CAC8934206D900210420FCF70CFE874B002266
S3150800CAD81A700520FCF77AFE03461A46834BDA7263
S3150800CAE8824B1B7A002B07D0804B1B7B002B03D16C
S3150800CAF87E4B1B78002B02D17C4B00225A727B4B4B
S3150800CB08DB79092B00F2558101A252F823F000BF00
S3150800CB1841CB000875CB000891CB0008C9CB0008A3
S3150800CB2817CC000859CC0008C3CC00086DCD0008FE
S3150800CB381DCD0008A7CD00086C4B00225A700021AD
S3150800CB480320FCF7CFFD694B1B7A002B00F03581D3
S3150800CB58664B1B78002B00F03081644B1B7B002B3F
S3150800CB6840F02B810120FFF72BFC26E1FFF73CFC60
S3150800CB780346B3F57A6F40F222815C4B01225A725A
S3150800CB880220FFF71DFC1AE1584B00221A760021ED
S3150800CB980320FCF7A7FD554B5B7A002B03D1002031
S3150800CBA8FFF70EFC1CE1554BDB7D002B00F00981D5
S3150800CBB801210020FFF7ACFD0320FFF701FC00E187
S3150800CBC84A4B9B7A002B0CD0484B5B7A002B08D033
S3150800CBD801F0FAFD03464B4A13600420FFF7F0FB01
S3150800CBE8F1E0FFF701FC034642F21072934240F265
S3150800CBF8EA803E4B01225A73404B0A225A77002094
S3150800CC08FFF7DEFB40490420FEF728FCDBE001219C
S3150800CC180320FCF767FD354BDB7A002B03D005208C
S3150800CC28FFF7CEFBD1E0FFF7DFFB0346B3F57A7FC4
S3150800CC3840F2CB802D4B01221A73304B07225A77C4
S3150800CC480620FFF7BDFB31490420FEF707FCBCE0C8
S3150800CC582A4BDB7D002B03D0244B5B7A002B03D1B0
S3150800CC680620FFF7ADFBBBE00520FCF7AFFD034642
S3150800CC781C460320FCF79AFD03469C4217D001F090
S3150800CC88A3FD0246224B1B68D31AB3F57A7F40F2F6
S3150800CC989E801A4B07225A77144B01221A730620CC
S3150800CCA8FFF78EFB19490420FEF7D8FB8FE001F041
S3150800CCB88BFD0346164A136089E0104B00225A7406
S3150800CCC800229A740D4BB3F815309BB21D2B06D962
S3150800CCD8FFF78AFB034641F28832934279D908203E
S3150800CCE8FFF76EFB75E000BF200A0020FC0900204C
S3150800CCF8C4090020D0090020EC090020E802002019
S3150800CD08480A00204C0A0020486B0108586B01089D
S3150800CD18500A002000210320FCF7E4FC314BDB7A9B
S3150800CD28002B07D100210020FFF7F2FC0720FFF7A8
S3150800CD3847FB50E0FFF758FB0346B3F57A7F4AD915
S3150800CD48284B01221A73284B07225A7700210020FC
S3150800CD58FFF7DEFC0720FFF733FB24490420FEF71C
S3150800CD687DFB38E01F4B9B7A002B03D10920FFF780
S3150800CD7827FB32E0FFF738FB034642F2107293426C
S3150800CD882BD9184B01225A73174B0A225A770020B7
S3150800CD98FFF716FB16490420FEF760FB1DE0FFF7B0
S3150800CDA823FB0346B3F57A6F19D90220FFF708FB68
S3150800CDB815E00020FFF704FB12E000BF10E000BFF3
S3150800CDC80EE000BF0CE000BF0AE000BF08E000BFA5
S3150800CDD806E000BF04E000BF02E000BF00E000BFB5
S3150800CDE800BF98BDFC090020E8020020586B01081E
S3150800CDF8786B010880B500AF344B5B7F002B03D0F6
S3150800CE08334800F01FF95FE0304B5B780D2B57D895
S3150800CE1801A252F823F000BF59CE000861CE0008D7
S3150800CE2869CE000871CE000879CE000881CE0008C0
S3150800CE3889CE000891CE000899CE0008A1CE000830
S3150800CE48A9CE0008B1CE0008B9CE0008C1CE0008A0
S3150800CE58204800F0F7F837E01F4800F0F3F833E009
S3150800CE681B4800F0EFF82FE01C4800F0EBF82BE021
S3150800CE781A4800F0E7F827E0194800F0E3F823E035
S3150800CE88174800F0DFF81FE0154800F0DBF81BE04C
S3150800CE98134800F0D7F817E0124800F0D3F813E063
S3150800CEA8104800F0CFF80FE00E4800F0CBF80BE07A
S3150800CEB80C4800F0C7F807E0084800F0C3F803E094
S3150800CEC8044800F0BFF800BF80BD00BFE802002094
S3150800CED854000020180000202400002030000020FC
S3150800CEE83C0000204800002080B487B000AFF860F6
S3150800CEF8B96011461A460B46FB801346BB80FA886A
S3150800CF08BB889A4201D9BB88FB80BB88002B01D114
S3150800CF180123BB80FA8813461B029A1ABB8892FB20
S3150800CF28F3F3FB82FB681B781A46FB8AC3F1FF03F7
S3150800CF3803FB02F2BB681B781946FB8A01FB03F35D
S3150800CF481344204A82FB03121A44D211DB17D31A58
S3150800CF58DAB23B6A1A70FB685B781A46FB8AC3F131
S3150800CF68FF0303FB02F2BB685B781946FB8A01FBE1
S3150800CF7803F31344134A82FB03121A44D211DB172C
S3150800CF88D31ADAB23B6A5A70FB689B781A46FB8A48
S3150800CF98C3F1FF0303FB02F2BB689B781946FB8AB9
S3150800CFA801FB03F31344074A82FB03121A44D211FE
S3150800CFB8DB17D31ADAB23B6A9A7000BF1C37BD462C
S3150800CFC880BC70478180808080B483B000AF786069
S3150800CFD87B681B781A46642302FB03F3174A82FB0D
S3150800CFE803121A44D211DB17D21A154B1B689A6317
S3150800CFF87B685B781A46642302FB03F30F4A82FBB5
S3150800D00803121A44D211DB17D21A0D4B1B68DA63BE
S3150800D0187B689B781A46642302FB03F3074A82FB5C
S3150800D02803121A44D211DB17D21A054B1B681A6465
S3150800D03800BF0C37BD4680BC704700BF8180808022
S3150800D048F80C002080B483B000AF7860054B7A6886
S3150800D0581068516803C312891A8000BF0C37BD4689
S3150800D06880BC70475C0A002080B582B000AF0023F8
S3150800D0783B7100237B710023BB710421094804F026
S3150800D088DFFD0821074804F0DBFD0C21054804F0FC
S3150800D098D7FD3B1D1846FFF797FF00BF0837BD4663
S3150800D0A880BD00BFF80C002080B582B002AF01F041
S3150800D0B88BFB0246464B1B68D31A142B40F2858015
S3150800D0C801F082FB0346424A1360424B5B880133F0
S3150800D0D89AB2404B5A803F4B1B78032B67D801A25C
S3150800D0E852F823F0FDD000082FD100085BD10008BC
S3150800D0F88DD10008374B5A88374BDB781946374B9A
S3150800D10800930B4634493648FFF7EEFE314B5B88E9
S3150800D118314AD27893424ED92E4B01221A702D4B9A
S3150800D12800225A8047E02B4B2B4A043312681146D3
S3150800D13819800233120C1A70264B5B88264A127914
S3150800D14893423AD9234B02221A70224B00225A805C
S3150800D15833E0204B5A88204B5B7919461F4B0093BE
S3150800D1680B461F491C48FFF7BFFE1A4B5B881A4A2D
S3150800D1785279934223D9174B03221A70154B00226A
S3150800D1885A801CE0134B144A0433073211889278E4
S3150800D19819809A700F4B5B880F4A9279934210D977
S3150800D1A80C4B00221A700B4B00225A8009E0094BD7
S3150800D1B800221A7006E000BF04E000BF02E000BFC4
S3150800D1C800E000BF0548FFF7FFFE00BFBD4680BD6B
S3150800D1D8680A0020540A00205C0A0020580A002021
S3150800D1E8630A002080B500AF0A4B0B4A1A60094B40
S3150800D1F84FF0FF325A60074B4FF480729A60054821
S3150800D20804F06EFB0346002B01D0FFF769F800BF50
S3150800D21880BD00BF6C0A00200028004080B584B095
S3150800D22800AF78607B681B680B4A934210D103F0FD
S3150800D238EBFA0A4BDB69094A43F00063D361074BEB
S3150800D248DB6903F00063FB60FB68054B01221A6083
S3150800D25800BF1037BD4680BD0028004000100240B8
S3150800D2683C04424280B400AF0E4B1B681B689AB256
S3150800D2780D4B1A800B4B1B685A790B4B9A70094B46
S3150800D2881B681A79084BDA70074B01229A80064BF5
S3150800D2980022DA80044B01221A8100BFBD4680BCF1
S3150800D2A8704700BF00000020E80C002080B500AFDA
S3150800D2B84FF404720021024806F0E6FE00BF80BD5E
S3150800D2C8800A002080B500AF254B93F84230DBB2C0
S3150800D2D8202B0AD1234B93F80832DBB2002B04D152
S3150800D2E8FF2221491E4805F084FA1D4B93F8413060
S3150800D2F8DBB2212B19D11B4BD3F80C32002B14D0D7
S3150800D30801F062FA0246174BD3F80C32D31A642B8B
S3150800D3180BD9134805F0CAFA00221021134803F05E
S3150800D3285AFA104B0022C3F80C220E4B93F808320F
S3150800D338DBB2002B11D00A4B93F84130DBB2212B14
S3150800D3480BD00B4800F024FAFF220749044805F0D9
S3150800D35850FA044B002283F8082200BF80BD00BF9C
S3150800D368D00D0020800A0020800B00200014014000
S3150800D378800C002080B582B000AF78600B467B80B1
S3150800D3887B681A680A4B1B689A420CD17B8819462F
S3150800D398084800F08FF90346002B04D1142200210F
S3150800D3A8002000F04BF900BF0837BD4680BD00BF16
S3150800D3B8D00D0020800B002080B582B000AF7860C1
S3150800D3C87B681A68084B1B689A4208D10022102104
S3150800D3D8064803F000FA064B0022C3F80C2200BFE1
S3150800D3E80837BD4680BD00BFD00D00200014014097
S3150800D3F8800A002080B485B000AF78600023FB60FF
S3150800D4080023BB607A68BB6822FA03F303F00103BA
S3150800D418FA681343FB600123BB600EE0FB685B00F8
S3150800D428FB607A68BB6822FA03F303F00103FA681B
S3150800D4381343FB60BB680133BB60BB681F2BEDD980
S3150800D448FB6818461437BD4680BC704780B586B059
S3150800D45800AF7860396000237B610023FB603B6876
S3150800D4689B087B613D4B5B693C4A43F0400353612B
S3150800D4783A4B5B6903F04003BB60BB68384B1B68D3
S3150800D4889A68374B1B6842F001029A6023E007F155
S3150800D4980C037A6812781A7007F10C0301337A6854
S3150800D4A852781A7007F10C0302337A6892781A7060
S3150800D4B807F10C0303337A68D2781A707B68043349
S3150800D4C87B60FB681846FFF795FF0346FB60244B0D
S3150800D4D81B68FA681A607B695A1E7A61002BD6D1CE
S3150800D4E81F4B1B681B681846FFF784FF0346FB603B
S3150800D4F83B6803F003037B611EE07B685A1C7A606D
S3150800D5081B781A46FB685340FB6000233B6110E012
S3150800D518FB6803F00103002B05D0FB685A08114B7A
S3150800D5285340FB6002E0FB685B08FB603B6901331C
S3150800D5383B613B69072BEBD97B695A1E7A61002B3D
S3150800D548DBD1064B5B69054A23F040035361FB6848
S3150800D558DB4318461837BD4680BD00BF0010024099
S3150800D568D00300202083B8ED80B582B000AF78607C
S3150800D5780B467B807B8819467868FFF767FF034662
S3150800D58818460837BD4680BD80B588B000AFF86034
S3150800D5987A601A460B467B8113467B720023FB8307
S3150800D5A8FB8B5A1CFA831A467B6813447A7A1A70D4
S3150800D5B8FB68002B19D00023BB8312E0BB8BFA68E3
S3150800D5C81A44FB8B591CF98319467B680B44127855
S3150800D5D81A70FB8BFA2B01D900232AE0BB8B01337F
S3150800D5E8BB83BA8B7B899A42E8D3FB8B1946786842
S3150800D5F8FFF7BAFF03463B6107F110037B61002377
S3150800D608BB6112E0BB697A691A44FB8B591CF9831A
S3150800D61819467B680B4412781A70FB8BFE2B01D9C6
S3150800D628002306E0BB690133BB61BB69032BE9DD4F
S3150800D638FB8B18462037BD4680BD000080B584B0F0
S3150800D64800AF78600B467B8013467B707B787988B9
S3150800D658154A7868FFF798FF0346FB81FB89002B74
S3150800D6681ED0124B93F84130DBB2212B07D10F4855
S3150800D67805F01CF9002210210D4803F0ACF8012228
S3150800D68810210B4803F0A7F8FB891A4606490748EC
S3150800D69805F07AF801F098F80346034AC2F80C32FE
S3150800D6A800BF1037BD4680BD800A0020D00D002077
S3150800D6B80014014080B586B000AF78600B467B80C1
S3150800D6C87B88042B01D8002346E07B88B3F5807F46
S3150800D6D801D9002340E07B88043BFB82FB8A7A68F1
S3150800D6E813441B781946FB8A01337A6813441B7856
S3150800D6F81B0241EA0302FB8A023379680B441B784A
S3150800D7081B041A43FB8A033379680B441B781B06E8
S3150800D71813433B61FB8A19467868FFF725FFF860CB
S3150800D7283A69FB689A4201D0002315E07B68013301
S3150800D7380B4AC2F804327B681A78094B83F8002228
S3150800D748FB8ADBB2013BDAB2054B83F80122044BAC
S3150800D758012283F80822012318461837BD4680BDDA
S3150800D768800A002080B400AFBFF34F8F00BF064B76
S3150800D778DB6803F4E0620449044B1343CB60BFF348
S3150800D7884F8F00BF00BFFDE700ED00E00400FA0573
S3150800D79880B584B000AF78601323FB737B681B7869
S3150800D7A8C22B00F3B080B02B09DA602B3CD0602B73
S3150800D7B800F3A980402B2FD0502B3BD0A3E0B03BD9
S3150800D7C8122B00F2A08001A252F823F043D80008D1
S3150800D7D80FD900080FD900080FD900080FD9000873
S3150800D7E8F3D800080FD900080FD900080FD9000880
S3150800D7F80FD900080FD900080FD900080FD9000853
S3150800D8080FD900080FD900080FD9000889D80008C9
S3150800D818EDD80008C1D8000800F096F8402258212B
S3150800D8283F48FFF70BFF77E060220A213D48FFF7DC
S3150800D83805FF71E0FDF7B0FD6EE07B685B780B2BA2
S3150800D8481BD17B685A68384B1068516803C311891D
S3150800D858927A19809A70FCF7C7FA344B01221A7023
S3150800D868FCF7C2FA304BD3F803302F4A3049072061
S3150800D878FDF7F4FD1223FB7348E01323FB7345E019
S3150800D8887B685B78012B14D17B685B681B781A4622
S3150800D8984FF47A7302FB03F31A46264B5A61254B53
S3150800D8A85B691A4624490720FDF7D8FD1223FB733E
S3150800D8B82CE01323FB7329E07B685B78012B0ED1D8
S3150800D8C87B685B681A781D4B1A701C4B1B781A46BE
S3150800D8D81B490720FDF7C2FD1223FB7316E0132325
S3150800D8E8FB7313E01323FB7310E0122200210020B8
S3150800D8F8FFF7A4FE00BF134B93F84130DBB2212B88
S3150800D908F9D0FFF72FFF1323FB7300BFFB7B1A46DB
S3150800D91800210020FFF792FE1037BD4680BD00BFE4
S3150800D928900C0020E80C002060000020F20C002073
S3150800D9388C6B0108FC090020A06B0108E80200208E
S3150800D948B46B0108D00D0020B0B500AF9D4B9A788E
S3150800D9589D4B9A709B4BD3F807309B4AC2F8033005
S3150800D968984BB3F80F309AB2974BA3F80720954B04
S3150800D978B3F81B309AB2944BA3F80920914BB3F825
S3150800D98813309AB2904BA3F80B208E4BB3F8153088
S3150800D9989AB28D4BA3F80D208A4B1A7E8A4BDA73F6
S3150800D9A8884B5A7F884B5A70864B5A78864B1A701A
S3150800D9B8854B00221A7400225A74834B00229A74E3
S3150800D9C8814B0022DA7400221A750420FBF7EEFE52
S3150800D9D8034603F00103D9B27B4A537D61F300037A
S3150800D9E853750320FBF7E2FE034603F00103D9B299
S3150800D9F8754A537D61F3410353750020FBF7D6FE3C
S3150800DA08034603F00103D9B26F4A537D61F38203D3
S3150800DA185375FEF7B1F9034603F00103D9B26A4A0A
S3150800DA28537D61F3C30353750320FBF7CFFE034603
S3150800DA38002B0CBF01230023D9B2634A537D61F337
S3150800DA4804135375FDF794FC0346002B14BF0123F2
S3150800DA580023D9B25C4A537D61F3451353755B4B72
S3150800DA681B7803F00103D9B2574A537D61F386132D
S3150800DA785375574B1B7A03F00103D9B2524A537DA3
S3150800DA8861F3C71353750020FBF784FF03465AB2A0
S3150800DA984D4B5A760120FBF77DFF03465AB24A4B8F
S3150800DAA89A764B4BDB695AB2474BDA76494B5B7821
S3150800DAB85AB2454B1A77474BDB785AB2424B5A77D4
S3150800DAC8454B9B889AB2404BDA83424B9A793E4B30
S3150800DAD883F82020414B9B689AB23B4BA3F8212038
S3150800DAE83E4BDB689AB2384BA3F823203B4B1B699D
S3150800DAF89AB2354BA3F82520334B394A27331832BF
S3150800DB08156854689068D1681D605C609860D9602B
S3150800DB18127C1A74324BDA782B4B83F83820304B40
S3150800DB289B889AB2284BA3F839202D4BDB889AB2E2
S3150800DB38254BA3F83B202A4B9B681A46224BC3F869
S3150800DB483D20274BDB68204AC2F84130244B9A7C93
S3150800DB581D4B83F84720224B5A7C1B4B83F84620DB
S3150800DB681F4B1A7C184B83F845201D4BDA7C197D08
S3150800DB7809020A435B7D1B0413439AB2124BA3F8A6
S3150800DB884820174B9A7D104B83F84A200E4B144AA7
S3150800DB984B3329321168526819605A600A4B0022B9
S3150800DBA883F85320084B002283F85420002283F870
S3150800DBB85520054B002283F85620002283F8572063
S3150800DBC800BFB0BDE8020020900C00201903002011
S3150800DBD8FC0900209403002088030020D0090020AF
S3150800DBE83403002080B500AF024800F0A5F80346C4
S3150800DBF8184680BD6C0A002080B582B000AF7860F0
S3150800DC087968034800F0C8F800BF0837BD4680BDE4
S3150800DC186C0A002080B483B000AF78607B680F4A2E
S3150800DC2882FB03129210DB17D31A5BB21B0158B298
S3150800DC387A680A4B83FB02139910D317C91A0B463D
S3150800DC489B000B445B00D11A4BB203435BB2DBB2B1
S3150800DC5818460C37BD4680BC704700BF67666666BF
S3150800DC6890B587B000AF78603960796800200A46B1
S3150800DC780346C7E9022307F10803184606F00CFA13
S3150800DC8878617B691B681846FFF7C4FF03461A467E
S3150800DC983B681A707B695A683B685C1C1046FFF734
S3150800DCA8B9FF034623707B699A683B689C1C104633
S3150800DCB8FFF7B0FF034623707B69DA683B68DC1C0C
S3150800DCC81046FFF7A7FF034623707B691B695A1C92
S3150800DCD83B681C1D1046FFF79DFF034623707B69AA
S3150800DCE85B6903F26C73134A82FB03125111DA1744
S3150800DCF88A1A642101FB02F29A1A3B685C1D1046CF
S3150800DD08FFF788FF034623707B695B6903F26C7328
S3150800DD18084A82FB03125211DB17D21A3B689C1D6C
S3150800DD281046FFF777FF0346237000BF1C37BD462A
S3150800DD3890BD00BF1F85EB5180B487B000AF7860EF
S3150800DD4800237B8200233B820023FB8100237B611F
S3150800DD587B681B689B697B827B681B68DB69FB8120
S3150800DD687B681B689B693B827A8A3B8A9A4208D0F9
S3150800DD783B8A1A047B681B68DB699BB213437B6181
S3150800DD8804E07B8A1A04FB8913437B617B6918467E
S3150800DD981C37BD4680BC704780B584B000AF786034
S3150800DDA839600023FB73786800F01DF80346002BDA
S3150800DDB802D00123FB7311E07B681B683A68120CD2
S3150800DDC89A617B681B683A6892B2DA61786800F0EB
S3150800DDD832F80346002B01D00123FB73FB7B184658
S3150800DDE81037BD4680BD80B584B000AF7860002383
S3150800DDF8FB6000F0E9FCF86009E000F0E5FC024683
S3150800DE08FB68D31AB3F57A7F01D903230FE07B6839
S3150800DE181B685B6803F02003002BEED07B681B6841
S3150800DE285A687B681B6842F010025A600023184635
S3150800DE381037BD4680BD80B584B000AF7860002332
S3150800DE48FB607B681B685A687B681B6822F01002AF
S3150800DE585A6000F0B9FCF86009E000F0B5FC024623
S3150800DE68FB68D31AB3F57A7F01D9032307E07B68E1
S3150800DE781B685B6803F02003002BEED000231846C6
S3150800DE881037BD4680BD000080B485B000AF154B7D
S3150800DE989B69144A43F001039361124B9B6903F08B
S3150800DEA80103BB60BB680F4BDB690E4A43F080531E
S3150800DEB8D3610C4BDB6903F080537B607B680A4BA4
S3150800DEC85B68FB60FB6823F0E063FB60FB6843F074
S3150800DED80073FB60044AFB68536000BF1437BD46ED
S3150800DEE880BC7047001002400000014080B400AFB3
S3150800DEF800BFFDE780B400AF00BFFDE780B400AF00
S3150800DF0800BFFDE780B400AF00BFFDE780B400AFEF
S3150800DF1800BFFDE780B400AF00BFBD4680BC7047B0
S3150800DF2880B400AF00BFBD4680BC704780B400AF60
S3150800DF3800BFBD4680BC704780B500AF00F032FC14
S3150800DF4800BF80BD80B500AF024801F023FE00BFC0
S3150800DF5880BD00BF9402002080B500AF024804F0D7
S3150800DF68B9FD00BF80BD00BF880D002080B500AF91
S3150800DF78024804F0AFFD00BF80BD00BFD00D0020E9
S3150800DF8880B500AF024804F0A5FD00BF80BD00BFFC
S3150800DF98180E002080B500AF024801F0FBFD00BF4F
S3150800DFA880BD00BFBC02002080B500AF024801F062
S3150800DFB8F1FD00BF80BD00BFBC02002080B400AFE1
S3150800DFC801231846BD4680BC704780B582B000AFAD
S3150800DFD87860396006F026F9034616221A604FF06B
S3150800DFE8FF3318460837BD4680BD80B582B000AFF6
S3150800DFF878604FF0FF317868FFF7E7FF00BFFDE765
S3150800E00880B586B000AFF860B9607A6000237B6196
S3150800E0180AE0AFF300800146BB685A1CBA60CAB268
S3150800E0281A707B6901337B617A697B689A42F0DBEF
S3150800E0387B6818461837BD4680BD80B483B000AFE4
S3150800E04878604FF0FF3318460C37BD4680BC7047DA
S3150800E05880B483B000AF786039603B684FF40052EB
S3150800E0685A60002318460C37BD4680BC704780B4F2
S3150800E07883B000AF7860012318460C37BD4680BCCC
S3150800E088704780B485B000AFF860B9607A6000233D
S3150800E09818461437BD4680BC7047000080B586B060
S3150800E0A800AF7860144A154BD31A7B617B693B61CC
S3150800E0B8134B1B68002B02D1114B124A1A60104BDE
S3150800E0C81A687B6813443A699A4207D206F0AAF88E
S3150800E0D803460C221A604FF0FF3309E0084B1B6809
S3150800E0E8FB60074B1A687B681344054A1360FB688C
S3150800E0F818461837BD4680BD0000012000040000F8
S3150800E108F40C0020B00F002080B400AF00BFBD4655
S3150800E11880BC704780B58EB000AF07F1280300228F
S3150800E1281A605A609A60DA6007F1200300221A60BA
S3150800E1385A603B1D00221A605A609A60DA601A61B2
S3150800E1485A619A61374B384A1A60364B4FF434721B
S3150800E1585A60344B00229A60324B6422DA60314B9B
S3150800E16800221A612F4B00229A612E4803F0C1FC3F
S3150800E1780346002B01D0FEF7B3F84FF48053BB6271
S3150800E18807F128031946274803F0C6FE0346002B5D
S3150800E19801D0FEF7A5F8234803F0FAFC0346002B3E
S3150800E1A801D0FEF79DF800233B6200237B6207F146
S3150800E1B8200319461B4804F031FA0346002B01D000
S3150800E1C8FEF78EF860237B600023BB600023FB60A4
S3150800E1D800237B613B1D04221946124803F0DAFD29
S3150800E1E80346002B01D0FEF77BF83B1D082219468B
S3150800E1F80C4803F0CFFD0346002B01D0FEF770F854
S3150800E2083B1D0C221946074803F0C4FD0346002B9C
S3150800E21801D0FEF765F8034800F026F800BF38373E
S3150800E228BD4680BDF80C00200008004080B485B0C3
S3150800E23800AF78607B681B68094A93420BD1094B83
S3150800E248DB69084A43F00403D361064BDB6903F02C
S3150800E2580403FB60FB6800BF1437BD4680BC7047E3
S3150800E268000800400010024080B588B000AF78600A
S3150800E27807F10C0300221A605A609A60DA607B6814
S3150800E2881B68174A934226D1164B9B69154A43F0D1
S3150800E29820039361134B9B6903F02003BB60BB689B
S3150800E2A84FF46043FB6002233B610223BB6107F11D
S3150800E2B80C0319460C4802F0F3F80C4B5B68FB6133
S3150800E2C8FB6943F0E063FB61FB6943F48053FB6138
S3150800E2D8064AFB69536000BF2037BD4680BD00BFAC
S3150800E2E800080040001002400014014000000140E8
S3150800E2F880B500AF114B124A1A60104B4FF4E13241
S3150800E3085A600E4B00229A600C4B0022DA600B4BBF
S3150800E31800221A61094B0C225A61084B00229A619D
S3150800E328064B0022DA61054804F0DEF90346002B9D
S3150800E33801D0FDF7D5FF00BF80BD00BF400D002006
S3150800E3480050004080B500AF114B124A1A60104BB6
S3150800E3584FF4E1325A600E4B00229A600C4B0022A9
S3150800E368DA600B4B00221A61094B0C225A61084BDA
S3150800E37800229A61064B0022DA61054804F0B4F9CE
S3150800E3880346002B01D0FDF7ABFF00BF80BD00BFD9
S3150800E398880D00200038014080B500AF114B124A9D
S3150800E3A81A60104B4FF4E1325A600E4B00229A60FD
S3150800E3B80C4B0022DA600B4B00221A61094B0C221F
S3150800E3C85A61084B00229A61064B0022DA61054811
S3150800E3D804F08AF90346002B01D0FDF781FF00BF38
S3150800E3E880BD00BFD00D00200044004080B500AFB6
S3150800E3F8114B124A1A60104B4FF4E1325A600E4B11
S3150800E40800229A600C4B0022DA600B4B00221A6134
S3150800E418094B0C225A61084B00229A61064B0022C6
S3150800E428DA61054804F060F90346002B01D0FDF7C8
S3150800E43857FF00BF80BD00BF180E002000480040E7
S3150800E44880B592B000AF786007F1300300221A60F1
S3150800E4585A609A60DA607B681B68914A93423DD194
S3150800E468904BDB698F4A43F48013D3618D4BDB6984
S3150800E47803F48013FB62FB6A8A4B9B69894A43F05B
S3150800E48810039361874B9B6903F01003BB62BB6A51
S3150800E498844B9B69834A43F020039361814B9B69AC
S3150800E4A803F020037B627B6A4FF480533B630223A5
S3150800E4B87B630323FB6307F1300319467A4801F0A7
S3150800E4C8EFFF04233B6300237B630023BB6307F149
S3150800E4D830031946754801F0E3FFDCE07B681B68E2
S3150800E4E8734A93423AD16F4B9B696E4A43F4804309
S3150800E4F893616C4B9B6903F480433B623B6A694BA7
S3150800E5089B69684A43F004039361664B9B6903F069
S3150800E5180403FB61FB694FF400733B6302237B63C7
S3150800E5280323FB6307F130031946624801F0B8FF75
S3150800E5384FF480633B6300237B630023BB6307F1C7
S3150800E548300319465B4801F0ABFF0022002125205D
S3150800E55801F011FE252001F02AFE9CE07B681B6865
S3150800E568554A934246D14F4BDB694E4A43F400332A
S3150800E578D3614C4BDB6903F40033BB61BB69494B78
S3150800E5889B69484A43F020039361464B9B6903F00D
S3150800E59820037B617B6920233B6302237B63032378
S3150800E5A8FB6307F130031946404801F079FF402319
S3150800E5B83B6300237B630023BB6307F130031946DB
S3150800E5C83A4801F06DFF3D4B5B683B643B6C43F092
S3150800E5D8E0633B643B6C43F008033B64374A3B6C97
S3150800E5E8536000220021262001F0C5FD262001F0EF
S3150800E5F8DEFD50E07B681B68314A93424BD1294BB4
S3150800E608DB69284A43F48023D361264BDB6903F484
S3150800E61880233B613B69234B9B69224A43F01003DD
S3150800E6289361204B9B6903F01003FB60FB684FF46A
S3150800E63880633B6302237B630323FB6307F1300391
S3150800E6481946194801F02CFF4FF400633B63002371
S3150800E6587B630023BB6307F130031946124801F0B0
S3150800E6681FFF164B5B687B647B6C23F030037B6467
S3150800E6787B6C43F0E0637B647B6C43F010037B643C
S3150800E6880E4A7B6C536000220021272001F073FD97
S3150800E698272001F08CFD00BF4837BD4680BD00BF66
S3150800E6A800500040001002400010014000140140CC
S3150800E6B800380140000801400044004000000140BD
S3150800E6C800480040DFF834D0FFF71EFD0C480D4916
S3150800E6D80D4A002302E0D458C4500433C4188C42A7
S3150800E6E8F9D30A4A0A4C002301E013600432A2420D
S3150800E6F8FBD305F09DFDFDF705FD704700000120D9
S3150800E7080000002040020020047001084002002092
S3150800E718B00F0020FEE7000080B500AF084B1B6865
S3150800E728074A43F010031360032001F019FD0F2070
S3150800E73800F008F8FFF7A8FB0023184680BD00BFBD
S3150800E7480020024080B582B000AF7860124B1A6884
S3150800E758124B1B7819464FF47A73B3FBF1F3B2FBE5
S3150800E768F3F3184601F031FD0346002B01D00123C7
S3150800E7780EE07B680F2B0AD8002279684FF0FF3025
S3150800E78801F0F9FC064A7B681360002300E00123C0
S3150800E79818460837BD4680BD6C0000207400002066
S3150800E7A87000002080B400AF054B1B781A46054B4D
S3150800E7B81B681344034A136000BFBD4680BC7047F4
S3150800E7C874000020600E002080B400AF024B1B685E
S3150800E7D81846BD4680BC7047600E002080B584B0D8
S3150800E7E800AF7860FFF7F0FFB8607B68FB60FB68EE
S3150800E7F8B3F1FF3F05D00A4B1B781A46FB6813444A
S3150800E808FB6000BFFFF7E0FF0246BB68D31AFA6849
S3150800E8189A42F7D800BF00BF1037BD4680BD00BF73
S3150800E8287400002080B586B000AF78600023FB75B9
S3150800E83800233B610023BB600023FB607B68002B39
S3150800E84801D10123BEE07B689B68002B7B689B6A25
S3150800E858002B09D17B680022DA627B68002283F8DC
S3150800E86824207868FAF7EAFE786800F0F1FB034690
S3150800E878FB757B689B6A03F01003002B40F09980B0
S3150800E888FB7D002B40F095807B689B6A23F48853B0
S3150800E89823F0020343F002027B689A627B685A688F
S3150800E8A87B68DB691A437B681B7B5B001343BA6882
S3150800E8B81343BB607B689B68B3F5807F03D07B688E
S3150800E8C89B68012B02D14FF4807300E000233A6954
S3150800E8D813433B617B681B7D012B19D17B681B7B26
S3150800E8E8002B09D17B689B69013B5A033B69134393
S3150800E8F843F400633B610BE07B689B6A43F02002A4
S3150800E9087B689A627B68DB6A43F001027B68DA6295
S3150800E9187B681B685B6823F469417B681B683A69EE
S3150800E9280A435A607B681B689A68284B13407A68BA
S3150800E9381268B9680B4393607B689B68B3F5807F58
S3150800E94803D07B689B68012B04D17B681B69013B54
S3150800E9581B05FB607B681B68DB6A23F470017B6810
S3150800E9681B68FA680A43DA627B681B689A68184B58
S3150800E9781340BA689A420BD17B680022DA627B6830
S3150800E9889B6A23F0030343F001027B689A6218E046
S3150800E9987B689B6A23F0120343F010027B689A622D
S3150800E9A87B68DB6A43F001027B68DA620123FB7540
S3150800E9B807E07B689B6A43F010027B689A6201232A
S3150800E9C8FB75FB7D18461837BD4680BDFDF7E1FF88
S3150800E9D8FE0E1FFF80B584B000AF78600023FB7376
S3150800E9E87B6893F82430012B01D1022398E07B68D1
S3150800E9F8012283F82420786800F0D0FA0346FB73CE
S3150800EA08FB7B002B40F087807B689B6A23F4407366
S3150800EA1823F0010343F480727B689A627B681B685B
S3150800EA28414A934205D1414B5B6803F47023002B96
S3150800EA3815D17B689B6A23F480127B689A627B6887
S3150800EA481B685B6803F48063002B26D07B689B6A87
S3150800EA5823F4405343F480527B689A621DE07B682E
S3150800EA689B6A43F480127B689A627B681B682F4A04
S3150800EA78934204D07B681B682B4A93420DD12B4BD3
S3150800EA885B6803F48063002B07D07B689B6A23F4D2
S3150800EA98405343F480527B689A627B689B6A03F406
S3150800EAA88053002B06D07B68DB6A23F006027B6856
S3150800EAB8DA6202E07B680022DA627B68002283F861
S3150800EAC824207B681B686FF002021A607B681B6843
S3150800EAD89B6803F46023B3F5602F13D17B681B6822
S3150800EAE8114A934205D1114B5B6803F47023002B36
S3150800EAF808D17B681B689A687B681B6842F4A00281
S3150800EB089A600CE07B681B689A687B681B6842F405
S3150800EB1880129A6003E07B68002283F82420FB7B36
S3150800EB2818461037BD4680BD00280140002401401C
S3150800EB3880B584B000AF78600023FB737B6893F8D0
S3150800EB482430012B01D102231AE07B68012283F8BD
S3150800EB582420786800F07CFA0346FB73FB7B002BBD
S3150800EB6809D17B689B6A23F4885323F0010343F091
S3150800EB7801027B689A627B68002283F82420FB7B63
S3150800EB8818461037BD4680BD90B587B000AF786087
S3150800EB98396000237B610023FB6000233B61FFF794
S3150800EBA813FE78617B681B689B6803F48073002BE7
S3150800EBB80BD07B689B6A43F020027B689A627B6865
S3150800EBC8002283F824200123D3E07B681B685B684E
S3150800EBD803F48073002B31D17B681B68DB6A03F466
S3150800EBE87003002B2AD121E03B68B3F1FF3F1DD003
S3150800EBF83B68002B07D0FFF7E7FD02467B69D31A67
S3150800EC083A689A4212D27B681B681B6803F00203AB
S3150800EC18002B0BD17B689B6A43F004027B689A62D7
S3150800EC287B68002283F824200323A2E07B681B68FC
S3150800EC381B6803F00203002BD6D070E04F4B1C6804
S3150800EC48022002F0FBFC0346B4FBF3F27B681B6860
S3150800EC5819694B4B0B40002B18D17B681B68D96880
S3150800EC68484B0B40002B11D17B681B681969464B2A
S3150800EC780B40002B08D17B681B68D968434B0B40AF
S3150800EC88002B01D1142320E029231EE07B681B688A
S3150800EC9819693D4B0B40002B06D17B681B68D96860
S3150800ECA83A4B0B40002B0DD07B681B681969384B0B
S3150800ECB80B40002B08D17B681B68D968344B0B407E
S3150800ECC8002B01D1542300E0FC2302FB03F33B612C
S3150800ECD821E03B68B3F1FF3F1AD03B68002B07D009
S3150800ECE8FFF772FD02467B69D31A3A689A420FD231
S3150800ECF8FB683A699A420BD97B689B6A43F0040217
S3150800ED087B689A627B68002283F82420032330E014
S3150800ED18FB680133FB60FB683A699A42D9D87B6875
S3150800ED281B686FF012021A607B689B6A43F40072CC
S3150800ED387B689A627B681B689B6803F46023B3F553
S3150800ED48602F15D17B681B7B002B11D17B689B6ACA
S3150800ED5823F480727B689A627B689B6A03F4805303
S3150800ED68002B05D17B689B6A43F001027B689A628F
S3150800ED78002318461C37BD4690BD00BF6C0000200E
S3150800ED88244992242449920092244912922449003B
S3150800ED984992240080B483B000AF78607B681B680A
S3150800EDA8DB6C18460C37BD4680BC704780B485B006
S3150800EDB800AF786039600023FB730023BB607B686B
S3150800EDC893F82430012B01D10223DCE07B68012269
S3150800EDD883F824203B685B68062B1CD87B681B686D
S3150800EDE8596B3B685A6813469B001344053B1F2218
S3150800EDF802FA03F3DB4319403B6818683B685A680C
S3150800EE0813469B001344053B00FA03F27B681B680C
S3150800EE180A435A633CE03B685B680C2B1CD87B6842
S3150800EE281B68196B3B685A6813469B001344233BB7
S3150800EE381F2202FA03F3DB4319403B6818683B684C
S3150800EE485A6813469B001344233B00FA03F27B686F
S3150800EE581B680A431A631BE07B681B68D96A3B6808
S3150800EE685A6813469B001344413B1F2202FA03F3D0
S3150800EE78DB4319403B6818683B685A6813469B0089
S3150800EE881344413B00FA03F27B681B680A43DA62BB
S3150800EE983B681B68092B1CD97B681B68D9683B68C3
S3150800EEA81A6813465B0013441E3B072202FA03F34B
S3150800EEB8DB4319403B6898683B681A6813465B0049
S3150800EEC813441E3B00FA03F27B681B680A43DA60A0
S3150800EED819E07B681B6819693B681A6813465B0062
S3150800EEE81344072202FA03F3DB4319403B68986880
S3150800EEF83B681A6813465B00134400FA03F27B68FA
S3150800EF081B680A431A613B681B68102B03D03B68C9
S3150800EF181B68112B32D17B681B681D4A934225D181
S3150800EF287B681B689B6803F40003002B26D17B6863
S3150800EF381B689A687B681B6842F400029A603B68FB
S3150800EF481B68102B1AD1134B1B68134AA2FB032301
S3150800EF589A0C13469B0013445B00BB6002E0BB682F
S3150800EF68013BBB60BB68002BF9D107E07B689B6A4D
S3150800EF7843F020027B689A620123FB737B680022B0
S3150800EF8883F82420FB7B18461437BD4680BC704797
S3150800EF98002401406C00002083DE1B4380B584B042
S3150800EFA800AF78600023FB600023BB607B681B68A2
S3150800EFB89B6803F00103012B40D07B681B689A689D
S3150800EFC87B681B6842F001029A601F4B1B681F4A40
S3150800EFD8A2FB03239B0CBB6002E0BB68013BBB603A
S3150800EFE8BB68002BF9D1FFF7EFFBF8601FE0FFF7C6
S3150800EFF8EBFB0246FB68D31A022B18D97B681B68F9
S3150800F0089B6803F00103012B11D07B689B6A43F0C8
S3150800F01810027B689A627B68DB6A43F001027B68A8
S3150800F028DA627B68002283F82420012307E07B68DC
S3150800F0381B689B6803F00103012BD8D100231846E7
S3150800F0481037BD4680BD00BF6C00002083DE1B4319
S3150800F05880B584B000AF78600023FB607B681B68C6
S3150800F0689B6803F00103012B2ED17B681B689A68FD
S3150800F0787B681B6822F001029A60FFF7A5FBF86017
S3150800F0881BE0FFF7A1FB0246FB68D31A022B14D92B
S3150800F0987B681B689B6803F00103012B0DD17B680D
S3150800F0A89B6A43F010027B689A627B68DB6A43F0C6
S3150800F0B801027B68DA62012307E07B681B689B68A4
S3150800F0C803F00103012BDCD0002318461037BD4690
S3150800F0D880BD000090B587B000AF78600023FB7547
S3150800F0E80023FB607B6893F82430012B01D10223A7
S3150800F0F897E07B68012283F824207868FFF7A8FF41
S3150800F1080346FB757868FFF749FF0346FB75FB7DE1
S3150800F118002B40F081807B689B6A23F4885323F090
S3150800F128020343F002027B689A62404B1C6802207D
S3150800F13802F084FA0346B4FBF3F35B00FB6002E0D3
S3150800F148FB68013BFB60FB68002BF9D17B681B68F1
S3150800F1589A687B681B6842F008029A60FFF734FBD6
S3150800F16838611BE0FFF730FB02463B69D31A0A2BC6
S3150800F17814D97B681B689B6803F00803002B0DD01D
S3150800F1887B689B6A23F0120343F010027B689A6235
S3150800F1987B68002283F82420012342E07B681B68E9
S3150800F1A89B6803F00803002BDCD17B681B689A6808
S3150800F1B87B681B6842F004029A60FFF705FB386112
S3150800F1C81BE0FFF701FB02463B69D31A0A2B14D941
S3150800F1D87B681B689B6803F00403002B0DD07B68CB
S3150800F1E89B6A23F0120343F010027B689A627B68D5
S3150800F1F8002283F82420012313E07B681B689B6898
S3150800F20803F00403002BDCD17B689B6A23F0030315
S3150800F21843F001027B689A627B68002283F82420FF
S3150800F228FB7D18461C37BD4690BD00BF6C00002004
S3150800F23880B584B000AF78607B68002B01D10123C4
S3150800F248EDE07B6893F82030DBB2002B02D17868B2
S3150800F258FAF76EFC7B681B681A687B681B6842F0BD
S3150800F26801021A60FFF7B0FAF86012E0FFF7ACFA85
S3150800F2780246FB68D31A0A2B0BD97B685B6A43F4E8
S3150800F28800327B685A627B68052283F820200123AE
S3150800F298C5E07B681B685B6803F00103002BE5D0B3
S3150800F2A87B681B681A687B681B6822F002021A606A
S3150800F2B8FFF78AFAF86012E0FFF786FA0246FB6853
S3150800F2C8D31A0A2B0BD97B685B6A43F400327B682E
S3150800F2D85A627B68052283F8202001239FE07B6811
S3150800F2E81B685B6803F00203002BE5D17B681B7E6D
S3150800F2F8012B08D17B681B681A687B681B6842F073
S3150800F30880021A6007E07B681B681A687B681B68B6
S3150800F31822F080021A607B685B7E012B08D17B6825
S3150800F3281B681A687B681B6842F040021A6007E087
S3150800F3387B681B681A687B681B6822F040021A609B
S3150800F3487B689B7E012B08D17B681B681A687B68DB
S3150800F3581B6842F020021A6007E07B681B681A6877
S3150800F3687B681B6822F020021A607B68DB7E012B0B
S3150800F37808D17B681B681A687B681B6822F010022C
S3150800F3881A6007E07B681B681A687B681B6842F086
S3150800F39810021A607B681B7F012B08D17B681B68E3
S3150800F3A81A687B681B6842F008021A6007E07B68DF
S3150800F3B81B681A687B681B6822F008021A607B6853
S3150800F3C85B7F012B08D17B681B681A687B681B68FA
S3150800F3D842F004021A6007E07B681B681A687B68B3
S3150800F3E81B6822F004021A607B689A687B68DB68E7
S3150800F3F81A437B681B691A437B685B6942EA0301FF
S3150800F4087B685B685A1E7B681B680A43DA617B68F7
S3150800F41800225A627B68012283F8202000231846B6
S3150800F4281037BD4680BD000080B487B000AF78604D
S3150800F43839607B681B687B617B6893F82030FB74AE
S3150800F448FB7C012B03D0FB7C022B40F0BE80654B6E
S3150800F4587B617B69D3F8003243F001027B69C3F804
S3150800F46800227B69D3F8003223F47C527B69C3F8FF
S3150800F47800227B69D3F800223B685B6A1B021A43A1
S3150800F4887B69C3F800223B685B6903F01F03012206
S3150800F49802FA03F3FB607B69D3F81C22FB68DB439B
S3150800F4A81A407B69C3F81C223B68DB69002B23D109
S3150800F4B87B69D3F80C22FB68DB431A407B69C3F8DF
S3150800F4C80C223B68DB6819043B685B689BB23A68A0
S3150800F4D8526919437B69483243F832103B689B687E
S3150800F4E819043B681B689AB23B685B690A437969E1
S3150800F4F84833DB000B445A603B68DB69012B22D191
S3150800F5087B69D3F80C22FB681A437B69C3F80C227B
S3150800F5183B681B6819043B685B689BB23A68526982
S3150800F52819437B69483243F832103B689B681904CB
S3150800F5383B68DB689AB23B685B690A437969483372
S3150800F548DB000B445A603B689B69002B09D17B6931
S3150800F558D3F80422FB68DB431A407B69C3F8042204
S3150800F56807E07B69D3F80422FB681A437B69C3F86A
S3150800F57804223B681B69002B09D17B69D3F814223E
S3150800F588FB68DB431A407B69C3F8142207E07B69EA
S3150800F598D3F81422FB681A437B69C3F814223B681C
S3150800F5A81B6A012B07D17B69D3F81C22FB681A430F
S3150800F5B87B69C3F81C227B69D3F8003223F0010261
S3150800F5C87B69C3F80022002306E07B685B6A43F47C
S3150800F5D880227B685A62012318461C37BD4680BCC0
S3150800F5E8704700BF0064004080B584B000AF7860FB
S3150800F5F87B6893F82030DBB2012B2ED17B68022278
S3150800F60883F820207B681B681A687B681B6822F0C9
S3150800F61801021A60FFF7D8F8F86012E0FFF7D4F885
S3150800F6280246FB68D31A0A2B0BD97B685B6A43F434
S3150800F63800327B685A627B68052283F820200123FA
S3150800F64812E07B681B685B6803F00103002BE5D1B1
S3150800F6587B6800225A62002306E07B685B6A43F4EB
S3150800F66800227B685A62012318461037BD4680BDBA
S3150800F67880B584B000AF78607B6893F82030DBB239
S3150800F688022B33D17B681B681A687B681B6842F0B3
S3150800F69801021A60FFF798F8F86012E0FFF794F885
S3150800F6A80246FB68D31A0A2B0BD97B685B6A43F4B4
S3150800F6B800327B685A627B68052283F8202001237A
S3150800F6C81BE07B681B685B6803F00103002BE5D029
S3150800F6D87B681B681A687B681B6822F002021A6036
S3150800F6E87B68012283F82020002306E07B685B6A92
S3150800F6F843F480127B685A62012318461037BD46C0
S3150800F70880BD80B489B000AFF860B9607A603B60A4
S3150800F718FB6893F82030FB77FB681B689B68BB611E
S3150800F728FB7F012B03D0FB7F022B40F0AD80BB6922
S3150800F73803F08063002B0AD1BB6903F00063002B32
S3150800F74805D1BB6903F08053002B00F09580BB698F
S3150800F7581B0E03F003037B6101227B699A403B6811
S3150800F7681A60BB689B68002B0DD1BB681B685A05D5
S3150800F778BB68DB68F96809681A437B6918331B0193
S3150800F7880B441A600FE0BB685B68DA00BB689B68C5
S3150800F7981A43BB68DB68F96809681A437B69183332
S3150800F7A81B010B441A60FB681968BB681A697B69F0
S3150800F7B818331B010B4404331A60BB681B7D012BE5
S3150800F7C811D1FB681A687B6918331B011344043383
S3150800F7D81B68FA68116843F480727B6918331B0141
S3150800F7E80B4404331A607B6807331B781A067B6850
S3150800F7F806331B781B041A437B6805331B781B02E0
S3150800F80813437A68043212781046FA68116843EA8C
S3150800F81800027B691B010B4403F5C6731A607B68F3
S3150800F82803331B781A067B6802331B781B041A43B2
S3150800F8387B6801331B781B0213437A6812781046D3
S3150800F848FA68116843EA00027B691B010B4403F551
S3150800F858C4731A60FB681A687B6918331B0113445A
S3150800F8681B68FA68116843F001027B6918331B01A3
S3150800F8780B441A6000230EE0FB685B6A43F4001227
S3150800F888FB685A62012306E0FB685B6A43F4802238
S3150800F898FB685A62012318462437BD4680BC704760
S3150800F8A880B485B000AF78600023FB607B6893F866
S3150800F8B82030FB72FB7A012B02D0FB7A022B1DD172
S3150800F8C87B681B689B6803F08063002B02D0FB6883
S3150800F8D80133FB607B681B689B6803F00063002B99
S3150800F8E802D0FB680133FB607B681B689B6803F0E2
S3150800F8F88053002B02D0FB680133FB60FB6818466F
S3150800F9081437BD4680BC704780B487B000AFF8602E
S3150800F918B9607A603B60FB6893F82030FB75FB7D1D
S3150800F928012B03D0FB7D022B40F00381BB68002B1B
S3150800F9380ED1FB681B68DB6803F00303002B16D19E
S3150800F948FB685B6A43F40012FB685A620123F7E016
S3150800F958FB681B681B6903F00303002B07D1FB68C8
S3150800F9685B6A43F40012FB685A620123E8E0FB6805
S3150800F9781A68BB681B331B0113441B6803F004028F
S3150800F9887B689A607B689B68002B0CD1FB681A68B1
S3150800F998BB681B331B0113441B685B0DC3F30A02C0
S3150800F9A87B681A600BE0FB681A68BB681B331B0187
S3150800F9B813441B68DB0823F060427B685A60FB68BF
S3150800F9C81A68BB681B331B0113441B6803F0020241
S3150800F9D87B68DA60FB681A68BB681B331B0113442B
S3150800F9E804331B6803F00803002B03D07B6808223E
S3150800F9F81A610BE0FB681A68BB681B331B011344C2
S3150800FA0804331B6803F00F027B681A61FB681A68DF
S3150800FA18BB681B331B01134404331B681B0ADAB281
S3150800FA287B689A61FB681A68BB681B331B01134419
S3150800FA3804331B681B0C9AB27B685A61FB681A6800
S3150800FA48BB681B01134403F5DC731B68DAB23B6811
S3150800FA581A70FB681A68BB681B01134403F5DC7344
S3150800FA681B681A0A3B680133D2B21A70FB681A680F
S3150800FA78BB681B01134403F5DC731B681A0C3B6847
S3150800FA880233D2B21A70FB681A68BB681B011344A2
S3150800FA9803F5DC731B681A0E3B680333D2B21A7077
S3150800FAA8FB681A68BB681B01134403F5DE731A68FA
S3150800FAB83B680433D2B21A70FB681A68BB681B0124
S3150800FAC8134403F5DE731B681A0A3B680533D2B27A
S3150800FAD81A70FB681A68BB681B01134403F5DE73C2
S3150800FAE81B681A0C3B680633D2B21A70FB681A6888
S3150800FAF8BB681B01134403F5DE731B681A0E3B68C3
S3150800FB080733D2B21A70BB68002B08D1FB681B688A
S3150800FB18DA68FB681B6842F02002DA6007E0FB68CF
S3150800FB281B681A69FB681B6842F020021A610023E1
S3150800FB3806E0FB685B6A43F48022FB685A62012385
S3150800FB4818461C37BD4680BC704780B485B000AFE0
S3150800FB58786039607B6893F82030FB73FB7B012B50
S3150800FB6802D0FB7B022B09D17B681B6859697B6825
S3150800FB781B683A680A435A61002306E07B685B6A91
S3150800FB8843F480227B685A62012318461437BD4617
S3150800FB9880BC704780B58AB000AF786000237B6266
S3150800FBA87B681B685B693B627B681B685B68FB61F3
S3150800FBB87B681B689B68BB617B681B68DB687B6125
S3150800FBC87B681B681B693B617B681B689B69FB60D4
S3150800FBD83B6A03F00103002B7CD0BB6903F00103E1
S3150800FBE8002B23D07B681B6801229A60BB6903F047
S3150800FBF80203002B03D0786800F083F916E0BB6986
S3150800FC0803F00403002B04D07B6A43F400637B6289
S3150800FC180CE0BB6903F00803002B04D07B6A43F4A5
S3150800FC2880537B6202E0786800F086F9BB6903F4C2
S3150800FC388073002B24D07B681B684FF480729A6007
S3150800FC48BB6903F40073002B03D0786800F062F9E7
S3150800FC5816E0BB6903F48063002B04D07B6A43F47F
S3150800FC6800537B620CE0BB6903F40063002B04D0E5
S3150800FC787B6A43F480437B6202E0786800F065F9A2
S3150800FC88BB6903F48033002B24D07B681B684FF4C8
S3150800FC9880329A60BB6903F40033002B03D0786876
S3150800FCA800F041F916E0BB6903F48023002B04D061
S3150800FCB87B6A43F400437B620CE0BB6903F40023C8
S3150800FCC8002B04D07B6A43F480337B6202E07868B1
S3150800FCD800F044F93B6A03F00803002B0CD07B6953
S3150800FCE803F01003002B07D07B6A43F400737B628A
S3150800FCF87B681B681022DA603B6A03F00403002B52
S3150800FD080BD07B6903F00803002B06D07B681B68B9
S3150800FD180822DA60786800F02AF93B6A03F00203D9
S3150800FD28002B09D07B681B68DB6803F00303002BEC
S3150800FD3802D07868FBF7ACFD3B6A03F04003002B5A
S3150800FD480CD03B6903F01003002B07D07B6A43F4F9
S3150800FD5880637B627B681B6810221A613B6A03F022
S3150800FD682003002B0BD03B6903F00803002B06D0B1
S3150800FD787B681B6808221A61786800F001F93B6AF3
S3150800FD8803F01003002B09D07B681B681B6903F076
S3150800FD980303002B02D07868FCF732FB3B6A03F4AE
S3150800FDA80033002B0BD0FB6903F01003002B06D099
S3150800FDB87B681B6810225A60786800F0EAF83B6A84
S3150800FDC803F48033002B0BD0FB6903F00803002BE0
S3150800FDD806D07B681B6808225A60786800F0E2F843
S3150800FDE83B6A03F40043002B7BD0FB6903F004034A
S3150800FDF8002B72D03B6A03F48073002B08D0FB688B
S3150800FE0803F00103002B03D07B6A43F001037B62EE
S3150800FE183B6A03F40073002B08D0FB6803F002035F
S3150800FE28002B03D07B6A43F002037B623B6A03F428
S3150800FE388063002B08D0FB6803F00403002B03D06B
S3150800FE487B6A43F004037B623B6A03F40063002B76
S3150800FE5843D0FB6803F07003002B3ED0FB6803F021
S3150800FE687003602B2BD0602B2ED8502B22D0502B0A
S3150800FE782AD8402B19D0402B26D8302B10D0302B17
S3150800FE8822D8102B02D0202B05D01DE07B6A43F020
S3150800FE9808037B6219E07B6A43F010037B6214E06F
S3150800FEA87B6A43F020037B620FE07B6A43F04003DA
S3150800FEB87B620AE07B6A43F080037B6205E07B6A23
S3150800FEC843F480737B6200E000BF7B681B689A690D
S3150800FED87B681B6822F070029A617B681B6804229B
S3150800FEE85A607B6A002B08D07B685A6A7B6A1A4371
S3150800FEF87B685A62786800F05EF800BF2837BD4606
S3150800FF0880BD80B483B000AF786000BF0C37BD46AB
S3150800FF1880BC704780B483B000AF786000BF0C37E8
S3150800FF28BD4680BC704780B483B000AF786000BF18
S3150800FF380C37BD4680BC704780B483B000AF786084
S3150800FF4800BF0C37BD4680BC704780B483B000AF8D
S3150800FF58786000BF0C37BD4680BC704780B483B054
S3150800FF6800AF786000BF0C37BD4680BC704780B4C8
S3150800FF7883B000AF786000BF0C37BD4680BC7047B9
S3150800FF8880B483B000AF786000BF0C37BD4680BC2C
S3150800FF98704780B483B000AF786000BF0C37BD46A1
S3150800FFA880BC704780B483B000AF786000BF0C3758
S3150800FFB8BD4680BC704780B483B000AF786000BF88
S3150800FFC80C37BD4680BC704780B485B000AF7860F2
S3150800FFD87B6803F00703FB600C4BDB68BB60BA68F9
S3150800FFE84FF6FF031340BB60FB681A02BB6813434E
S3150800FFF843F0BF6343F40033BB60044ABB68D3606D
S3150801000800BF1437BD4680BC704700BF00ED00E04D
S3150801001880B400AF044BDB681B0A03F007031846D4
S31508010028BD4680BC704700BF00ED00E080B483B0D0
S3150801003800AF0346FB7197F90730002B0BDBFB79F9
S3150801004803F01F02064997F907305B09012000FAF0
S3150801005802F241F8232000BF0C37BD4680BC704721
S3150801006800E100E080B483B000AF03463960FB7154
S3150801007897F90730002B0ADB3B68DAB20C4997F97E
S3150801008807301201D2B20B4483F800230AE03B6811
S31508010098DAB20849FB7903F00F03043B1201D2B21D
S315080100A80B441A7600BF0C37BD4680BC704700BFA3
S315080100B800E100E000ED00E080B489B000AFF86027
S315080100C8B9607A60FB6803F00703FB61FB69C3F152
S315080100D80703042B28BF0423BB61FB690433062BDA
S315080100E802D9FB69033B00E000237B614FF0FF322D
S315080100F8BB6902FA03F3DA43BB681A407B699A407B
S315080101084FF0FF317B6901FA03F3D9437B680B404A
S31508010118134318462437BD4680BC704780B582B05C
S3150801012800AF78607B68013BB3F1807F01D3012377
S315080101380FE00A4A7B68013B53600F214FF0FF30F5
S31508010148FFF790FF054B00229A60044B07221A60B5
S31508010158002318460837BD4680BD00BF10E000E0F9
S3150801016880B582B000AF78607868FFF72DFF00BFC9
S315080101780837BD4680BD80B586B000AF0346B9606D
S315080101887A60FB7300237B61FFF742FF78617A681F
S31508010198B9687869FFF790FF024697F90F30114653
S315080101A81846FFF75FFF00BF1837BD4680BD80B503
S315080101B882B000AF0346FB7197F907301846FFF777
S315080101C835FF00BF0837BD4680BD80B582B000AF90
S315080101D878607868FFF7A2FF034618460837BD46D0
S315080101E880BD80B582B000AF78607B68002B01D1ED
S315080101F801230EE07B685B79DBB2002B05D17B68AE
S3150801020800221A717868FBF725F87B6801225A716A
S31508010218002318460837BD4680BD80B485B000AFAF
S3150801022878600023FB737B6893F82130DBB2022BD5
S3150801023808D07B6804229A637B68002283F8202009
S31508010248012320E07B681B681A687B681B6822F013
S315080102580E021A607B681B681A687B681B6822F09D
S3150801026801021A607B681A6C7B68DB6B012101FA4B
S3150801027802F25A607B68012283F821207B680022F2
S3150801028883F82020FB7B18461437BD4680BC704787
S3150801029880B584B000AF78600023FB737B6893F858
S315080102A82130DBB2022B05D07B6804229A6301232D
S315080102B8FB73D6E07B681B681A687B681B6822F0A3
S315080102C80E021A607B681B681A687B681B6822F02D
S315080102D801021A607B681B681A46644B9A4258D908
S315080102E87B681B68624A93424FD07B681B68614AE0
S315080102F8934248D07B681B685F4A934240D07B6823
S315080103081B685E4A934238D07B681B685C4A9342ED
S3150801031830D07B681B685B4A934228D07B681B6888
S31508010328524A934220D07B681B68574A934219D090
S315080103387B681B68554A934212D07B681B68544AE6
S3150801034893420AD07B681B68524A934202D14FF4FA
S3150801035880531BE04FF4803318E04FF4807315E09F
S31508010368102313E0012311E04FF080730EE04FF4D8
S3150801037880130BE04FF4803308E04FF4805305E00F
S315080103884FF4807302E0102300E00123424A5360C8
S3150801039857E07B681B68364A93424FD07B681B68CF
S315080103A8344A934248D07B681B68334A934240D003
S315080103B87B681B68314A934238D07B681B68304A88
S315080103C8934230D07B681B682E4A934228D07B68B3
S315080103D81B68264A934220D07B681B682A4A93429F
S315080103E819D07B681B68294A934212D07B681B6817
S315080103F8274A93420AD07B681B68264A934202D148
S315080104084FF480531BE04FF4803318E04FF48073A0
S3150801041815E0102313E0012311E04FF080730EE075
S315080104284FF480130BE04FF4803308E04FF4805300
S3150801043805E04FF4807302E0102300E00123174A10
S3150801044853607B68012283F821207B68002283F8A0
S3150801045820207B685B6B002B03D07B685B6B786815
S315080104689847FB7B18461037BD4680BD8000024079
S31508010478080002401C0002403000024044000240C5
S31508010488580002406C000240080402401C0402405D
S3150801049830040240440402400004024000000240BD
S315080104A880B48BB000AF7860396000237B62002383
S315080104B83B6269E101227B6A02FA03F3FB613B6845
S315080104C81B68FA691340BB61BA69FB699A4240F02D
S315080104D858813B685B689A4A93425ED0984A934228
S315080104E875D8984A934258D0964A93426FD8964AED
S315080104F8934252D0944A934269D8944A93424CD02B
S31508010508924A934263D8924A934246D0904A934272
S315080105185DD8122B2AD8122B59D801A252F823F0E2
S31508010528A30501087D0501088F050108D1050108FC
S31508010538D7050108D7050108D7050108D705010810
S31508010548D7050108D7050108D7050108D705010800
S31508010558D7050108D7050108D7050108D7050108F0
S31508010568D70501088505010899050108794A9342BD
S3150801057813D02CE03B68DB683B6229E03B68DB6803
S3150801058804333B6224E03B68DB6808333B621FE0BF
S315080105983B68DB680C333B621AE03B689B68002BB7
S315080105A802D104233B6213E03B689B68012B05D102
S315080105B808233B627B68FA691A6109E008233B62EA
S315080105C87B68FA695A6103E000233B6200E000BFD1
S315080105D8BB69FF2B01D87B6801E07B6804337B6123
S315080105E8BB69FF2B02D87B6A9B0002E07B6A083B42
S315080105F89B003B617B691A680F213B6901FA03F382
S31508010608DB431A40396A3B6901FA03F31A437B69E2
S315080106181A603B685B6803F08053002B00F0B180D1
S315080106284D4B9B694C4A43F0010393614A4B9B69BD
S3150801063803F00103BB60BB68484A7B6A9B0802331F
S3150801064852F82330FB607B6A03F003039B000F22F1
S3150801065802FA03F3DB43FA681340FB607B68404AF6
S31508010668934213D07B683F4A93420DD07B683E4A32
S31508010678934207D07B683D4A934201D1032306E09A
S31508010688042304E0022302E0012300E000237A6A36
S3150801069802F0030292009340FA681343FB602F495C
S315080106A87B6A9B080233FA6841F823203B685B6832
S315080106B803F48013002B06D02D4B9A682C49BB6985
S315080106C813438B6006E02A4B9A68BB69DB432849C2
S315080106D813408B603B685B6803F40013002B06D054
S315080106E8234BDA682249BB691343CB6006E0204BE2
S315080106F8DA68BB69DB431E491340CB603B685B6814
S3150801070803F40033002B06D0194B5A681849BB69FC
S3150801071813434B6006E0164B5A68BB69DB43144919
S3150801072813404B603B685B6803F48033002B21D088
S315080107380F4B1A680E49BB6913430B6021E000BFCA
S3150801074800003210000031100000221000002110AC
S3150801075800001210000011100010024000000140AC
S3150801076800080140000C0140001001400014014036
S31508010778000401400B4B1A68BB69DB43094913405E
S315080107880B607B6A01337B623B681A687B6A22FACB
S3150801079803F3002B7FF48EAE00BF00BF2C37BD468E
S315080107A880BC70470004014080B485B000AF78600A
S315080107B80B467B807B689A687B881340002B02D09E
S315080107C80123FB7301E00023FB73FB7B18461437EF
S315080107D8BD4680BC704780B483B000AF78600B46CD
S315080107E87B8013467B707B78002B03D07A887B68DD
S315080107F81A6103E07B881A047B681A6100BF0C3703
S31508010808BD4680BC7047000080B400AF034B012287
S315080108181A6000BFBD4680BC704700BF20000E4263
S3150801082880B582B000AFFDF7CFFF7860604B1B68D3
S315080108385F4A43F00103136008E0FDF7C5FF024666
S315080108487B68D31A022B01D90323ACE0584B1B68E2
S3150801085803F00203002BF0D0554B1B6823F0F8036D
S31508010868534A43F080031360FDF7AEFF7860504B97
S3150801087800225A600AE0FDF7A7FF02467B68D31AE9
S3150801088841F28832934201D903238CE0484B5B68CD
S3150801089803F00C03002BEED1464B474A1A60474B27
S315080108A81B681846FDF74EFF0346002B01D00123A6
S315080108B879E0FDF789FF78603D4B1B683C4A23F0D0
S315080108C88073136008E0FDF77FFF02467B68D31A39
S315080108D8022B01D9032366E0354B1B6803F0007325
S315080108E8002BF0D1324B00225A60FDF76DFF786074
S315080108F82F4B1B682E4A23F41023136008E0FDF7D3
S3150801090863FF02467B68D31A642B01D903234AE09D
S31508010918274B1B6803F40033002BF0D1244B1B68C3
S31508010928234A23F480231360FDF74EFF7860204B92
S315080109381B681F4A23F08063136008E0FDF744FF2C
S3150801094802467B68D31A642B01D903232BE0184B7B
S315080109581B6803F00063002BF0D1FDF735FF7860BB
S31508010968134B1B68124A23F08053136008E0FDF7FE
S315080109782BFF02467B68D31A642B01D9032312E09D
S315080109880B4B1B6803F00053002BF0D1084B0022D0
S31508010998DA62074B5B6A064A43F080735362044B73
S315080109A800229A60002318460837BD4680BD00BF55
S315080109B8001002406C00002000127A007000002026
S315080109C880B586B000AF78607B68002B01D101231A
S315080109D804E37B681B6803F00103002B00F087809A
S315080109E8924B5B6803F00C03042B0CD08F4B5B68A6
S315080109F803F00C03082B12D18C4B5B6803F4803384
S31508010A08B3F5803F0BD1894B1B6803F40033002BE0
S31508010A186CD07B689B68002B68D10123DEE27B6872
S31508010A289B68B3F5803F06D1804B1B687F4A43F420
S31508010A38803313602EE07B689B68002B0CD17B4BB7
S31508010A481B687A4A23F480331360784B1B68774A04
S31508010A5823F4802313601DE07B689B68B3F5A02FF8
S31508010A680CD1724B1B68714A43F4802313606F4B90
S31508010A781B686E4A43F4803313600BE06B4B1B68A3
S31508010A886A4A23F480331360684B1B68674A23F460
S31508010A98802313607B689B68002B13D0FDF794FEAF
S31508010AA8386108E0FDF790FE02463B69D31A642BC4
S31508010AB801D9032392E25D4B1B6803F40033002B2B
S31508010AC8F0D014E0FDF780FE386108E0FDF77CFEFA
S31508010AD802463B69D31A642B01D903237EE2534B99
S31508010AE81B6803F40033002BF0D100E000BF7B68D4
S31508010AF81B6803F00203002B63D04C4B5B6803F0B9
S31508010B080C03002B0BD0494B5B6803F00C03082B2D
S31508010B181CD1464B5B6803F48033002B16D1434B33
S31508010B281B6803F00203002B05D07B685B69012B60
S31508010B3801D0012352E23D4B1B6823F0F8027B687A
S31508010B489B69DB00394913430B603AE07B685B69AB
S31508010B58002B20D0364B01221A60FDF735FE386185
S31508010B6808E0FDF731FE02463B69D31A022B01D983
S31508010B78032333E22D4B1B6803F00203002BF0D045
S31508010B882A4B1B6823F0F8027B689B69DB00274917
S31508010B9813430B6015E0264B00221A60FDF714FE75
S31508010BA8386108E0FDF710FE02463B69D31A022BA5
S31508010BB801D9032312E21D4B1B6803F00203002B1C
S31508010BC8F0D17B681B6803F00803002B3AD07B68D1
S31508010BD8DB69002B19D0174B01221A60FDF7F4FDC2
S31508010BE8386108E0FDF7F0FD02463B69D31A022B86
S31508010BF801D90323F2E10D4B5B6A03F00203002BCB
S31508010C08F0D0012000F0CAFB1CE00A4B00221A604A
S31508010C18FDF7DAFD38610FE0FDF7D6FD02463B69B7
S31508010C28D31A022B08D90323D8E100BF00100240C2
S31508010C3800004242800442429B4B5B6A03F002036E
S31508010C48002BE9D17B681B6803F00403002B00F02D
S31508010C58A6800023FB75944BDB6903F08053002BB0
S31508010C680DD1914BDB69904A43F08053D3618E4B82
S31508010C78DB6903F08053BB60BB680123FB758B4BAB
S31508010C881B6803F48073002B18D1884B1B68874AA5
S31508010C9843F480731360FDF797FD386108E0FDF7A3
S31508010CA893FD02463B69D31A642B01D9032395E1BF
S31508010CB87E4B1B6803F48073002BF0D07B681B6995
S31508010CC8012B06D1784B1B6A774A43F00103136255
S31508010CD82DE07B681B69002B0CD1734B1B6A724A82
S31508010CE823F001031362704B1B6A6F4A23F004034E
S31508010CF813621CE07B681B69052B0CD16A4B1B6ABE
S31508010D08694A43F004031362674B1B6A664A43F050
S31508010D18010313620BE0644B1B6A634A23F0010360
S31508010D281362614B1B6A604A23F0040313627B68EA
S31508010D381B69002B15D0FDF747FD38610AE0FDF759
S31508010D4843FD02463B69D31A41F28832934201D9D7
S31508010D58032343E1544B1B6A03F00203002BEED02D
S31508010D6814E0FDF731FD38610AE0FDF72DFD02466D
S31508010D783B69D31A41F28832934201D903232DE1FB
S31508010D88494B1B6A03F00203002BEED1FB7D012BAD
S31508010D9805D1454BDB69444A23F08053D3617B6807
S31508010DA8DB6A002B00F08C803F4B5B6803F48033C9
S31508010DB8B3F5803F0ED13C4B5B6803F00C03082B57
S31508010DC808D1394BDB6A03F48033B3F5803F01D187
S31508010DD8012303E17B68DB6A022B4ED1324B1B6880
S31508010DE803F08053002B09D02F4BDB6A03F0F0027E
S31508010DF87B685B6B9A4201D00123EFE02C4B0022FA
S31508010E081A60FDF7E1FC386108E0FDF7DDFC0246EA
S31508010E183B69D31A642B01D90323DFE0224B1B68EC
S31508010E2803F00063002BF0D11F4BDB6A23F0F002B5
S31508010E387B685B6B1C491343CB621B4BDB6A23F448
S31508010E4870627B681B6B18491343CB62184B0122E6
S31508010E581A60FDF7B9FC386108E0FDF7B5FC0246EA
S31508010E683B69D31A642B01D90323B7E00E4B1B68D8
S31508010E7803F00063002BF0D022E00B4BDB6A0A4A29
S31508010E8823F48033D3620A4B00221A60FDF79CFCCF
S31508010E9838610FE0FDF798FC02463B69D31A642BC3
S31508010EA808D903239AE000BF0010024000700040E9
S31508010EB8680042424B4B1B6803F00063002BE9D1DB
S31508010EC87B681B6A002B00F08880464B5B6803F039
S31508010ED80C03082B68D07B681B6A022B4DD1424B41
S31508010EE800221A60FDF770FC386108E0FDF76CFC12
S31508010EF802463B69D31A022B01D903236EE0394B03
S31508010F081B6803F00073002BF0D17B685B6AB3F5A5
S31508010F18803F0FD1334BDA6A7B685B6831491343E3
S31508010F28CB62304BDB6A23F00F027B68DB682D49FD
S31508010F381343CB622B4B5B6823F474127B68596A9B
S31508010F487B689B6A0B43274913434B60264B01224F
S31508010F581A60FDF739FC386108E0FDF735FC0246E9
S31508010F683B69D31A022B01D9032337E01D4B1B68AA
S31508010F7803F00073002BF0D02FE01B4B00221A60F8
S31508010F88FDF722FC386108E0FDF71EFC02463B69BD
S31508010F98D31A022B01D9032320E0124B1B6803F04D
S31508010FA80073002BF0D118E07B681B6A012B01D16D
S31508010FB8012313E00B4B5B68FB60FB6803F4803283
S31508010FC87B685B6A9A4206D1FB6803F470127B68F0
S31508010FD89B6A9A4201D0012300E000231846183774
S31508010FE8BD4680BD001002406000424280B584B00B
S31508010FF800AF786039607B68002B01D10123D0E006
S315080110086A4B1B6803F007033A689A4210D9674B7B
S315080110181B6823F0070265493B6813430B60634B5A
S315080110281B6803F007033A689A4201D00123B8E01E
S315080110387B681B6803F00203002B20D07B681B68BA
S3150801104803F00403002B05D0594B5B68584A43F44F
S31508011058E06353607B681B6803F00803002B05D01F
S31508011068534B5B68524A43F460535360504B5B6871
S3150801107823F0F0027B689B684D4913434B607B68F4
S315080110881B6803F00103002B40D07B685B68012BC2
S3150801109807D1474B1B6803F40033002B15D10123ED
S315080110A87FE07B685B68022B07D1414B1B6803F01D
S315080110B80073002B09D1012373E03D4B1B6803F02C
S315080110C80203002B01D101236BE0394B5B6823F03E
S315080110D803027B685B68364913434B60FDF774FB6B
S315080110E8F8600AE0FDF770FB0246FB68D31A41F27D
S315080110F88832934201D9032353E02D4B5B6803F0E9
S315080111080C027B685B689B009A42EBD1274B1B68EC
S3150801111803F007033A689A4210D2244B1B6823F056
S31508011128070222493B6813430B60204B1B6803F0EF
S3150801113807033A689A4201D0012332E07B681B68A3
S3150801114803F00403002B08D0194B5B6823F4E0620B
S315080111587B68DB68164913434B607B681B6803F099
S315080111680803002B09D0124B5B6823F460527B688D
S315080111781B69DB000E4913434B6000F021F8024650
S315080111880B4B5B681B0903F00F030A49CB5C22FA70
S3150801119803F3094A1360094B1B681846FDF7D2FA87
S315080111A8002318461037BD4680BD00BF00200240FF
S315080111B800100240CC6B01086C000020700000206A
S315080111C82DE9B04F8EB000AF0023FB620023BB6246
S315080111D800237B6300237B6200233B6300233B6276
S315080111E80023FB614E4B5B68FB62FB6A03F00C0349
S315080111F8042B02D0082B03D089E04A4B3B6389E0CC
S31508011208FB6A9B0C03F00F02474B9B5C7B62FB6AEC
S3150801121803F48033002B72D0414BDB6A03F00F02CB
S31508011228424B9B5CBB623E4BDB6A03F48033002B63
S3150801123853D03B4BDB6A1B0903F00F0301333B62AF
S31508011248374BDB6A1B0A03F00F030233FB61FB69A1
S3150801125800229A4693467B6A00223B617A613B697A
S3150801126803FB0BF27B690AFB03F313443A69AAFBEE
S3150801127802010B4419462B4B03FB01F2002300FB21
S3150801128803F31344274AA0FB02452B441D463B6A30
S315080112980022BB60FA60BB6A00223B607A60D7E924
S315080112A802010B46D7E900AB524602FB03F25B463D
S315080112B884460CFB03F3134402465146A2FB0189F3
S315080112C84B44994642464B4620462946F7F7DEFFE0
S315080112D802460B4613467B6307E07B6A114A03FB02
S315080112E802F2BB6AB2FBF3F37B630F4B5B7B1A46CD
S315080112F87B6A934208D17B6B5B087B6304E07B6A54
S315080113080B4A02FB03F37B637B6B3B6302E0094BE6
S315080113183B6300BF3B6B18463837BD46BDE8B08FFF
S315080113280010024040787D01E46B0108F46B01085E
S3150801133800093D0000127A0080B400AF024B1B6811
S315080113481846BD4680BC70476C00002080B500AFC2
S31508011358FFF7F2FF0246054B5B681B0A03F0070312
S315080113680349CB5C22FA03F3184680BD00100240F4
S31508011378DC6B010880B500AFFFF7DEFF0246054BB7
S315080113885B68DB0A03F007030349CB5C22FA03F31C
S31508011398184680BD00100240DC6B010880B485B090
S315080113A800AF78600A4B1B680A4AA2FB03235B0A4B
S315080113B87A6802FB03F3FB6000BFFB685A1EFA60F2
S315080113C8002BF9D100BF00BF1437BD4680BC704752
S315080113D86C000020D34D621080B588B000AF7860E4
S315080113E800237B6100233B610023FB617B681B6843
S315080113F803F00103002B7DD00023FB768B4BDB69B9
S3150801140803F08053002B0DD1884BDB69874A43F0DB
S315080114188053D361854BDB6903F08053FB60FB6816
S315080114280123FB76824B1B6803F48073002B18D1C2
S315080114387F4B1B687E4A43F480731360FDF7C4F932
S31508011448786108E0FDF7C0F902467B69D31A642B6F
S3150801145801D90323E5E0764B1B6803F48073002B57
S31508011468F0D0724B1B6A03F440733B613B69002B4E
S315080114782ED07B685B6803F440733A699A4227D091
S315080114886A4B1B6A23F440733B616A4B01221A6053
S31508011498684B00221A60654A3B6913623B6903F087
S315080114A80103002B14D0FDF78FF978610AE0FDF7DF
S315080114B88BF902467B69D31A41F28832934201D9DC
S315080114C80323AEE0594B1B6A03F00203002BEED047
S315080114D8564B1B6A23F440727B685B68534913436E
S315080114E80B62FB7E012B05D1504BDB694F4A23F072
S315080114F88053D3617B681B6803F00203002B08D06D
S315080115084A4B5B6823F440427B689B684749134307
S315080115184B607B681B6803F00403002B08D0434B18
S31508011528DB6A23F400327B68DB6840491343CB62E4
S315080115387B681B6803F00803002B08D03B4BDB6A62
S3150801154823F480227B681B6938491343CB62374BDE
S31508011558DB6A03F40033002B05D1344BDB6A03F449
S315080115688023002B01D00123FB61FB69012B48D19C
S315080115782E4B1B6803F08053002B38D12B4B1B6865
S3150801158803F08063002B09D0284BDB6A03F0F002CD
S315080115987B689B699A4201D0012342E0234BDB6AA7
S315080115A823F0F0027B689B6920491343CB621F4BE2
S315080115B8DB6A23F470427B685B691C491343CB6277
S315080115C81D4B01221A60FDF7FFF8786108E0FDF75F
S315080115D8FBF802467B69D31A642B01D9032320E059
S315080115E8124B1B6803F00053002BF0D009E00F4B90
S315080115F8DB6A03F470427B685B699A4201D001236E
S315080116080FE07B681B6803F01003002B08D0074B13
S315080116185B6823F480027B68DB69044913434B60E2
S31508011628002318462037BD4680BD00BF001002407A
S3150801163800700040400442427000424280B58AB0B8
S3150801164800AF78600023FB6100237B620023BB613E
S3150801165800237B6100233B610023FB600023BB60F9
S3150801166800233B627B68013B0F2B00F21D8101A217
S3150801167852F823F03118010895180108B11801081C
S315080116888F170108B1180108B1180108B11801081E
S31508011698E1170108B1180108B1180108B1180108BC
S315080116A8B1180108B1180108B1180108B1180108DB
S315080116B8BD160108834B5B68BB60824B1B6803F048
S315080116C88073002B00F0F280BB689B0C03F00F03B4
S315080116D87D4AD35CBB61BB6803F48033002B3BD0DE
S315080116E8784BDB6A03F00F03784AD35CFB61754BC9
S315080116F8DB6A03F48033002B1CD0724BDB6A1B09A7
S3150801170803F00F030133FB606E4BDB6A1B0A03F018
S315080117180F0302337B616E4AFB68B2FBF3F37A69FE
S3150801172803FB02F2FB69B2FBF3F2BB6902FB03F3A3
S315080117387B6207E0664AFB69B2FBF3F2BB6902FB07
S3150801174803F37B62604B5B7B1A46BB69934208D1FC
S315080117587B6A5B087B6204E0BB695E4A02FB03F3AA
S315080117687B62584B5B6803F48003B3F5800F02D19B
S315080117787B6A3B629AE07B6A5B00574AA2FB0323B2
S315080117885B083B6292E04F4BDB6A03F40033002B9C
S3150801179803D1FFF715FD38628AE04A4B1B6803F047
S315080117A88053002B00F08480464BDB6A1B0903F043
S315080117B80F030133FB60434BDB6A1B0B03F00F0373
S315080117C802333B61424AFB68B2FBF3F33A6902FB0F
S315080117D803F35B003B626BE03A4BDB6A03F4802355
S315080117E8002B03D1FFF7ECFC386263E0354B1B6825
S315080117F803F08053002B5DD0324BDB6A1B0903F0DB
S315080118080F030133FB602F4BDB6A1B0B03F00F0336
S3150801181802333B612E4AFB68B2FBF3F33A6902FBD2
S3150801182803F35B003B6245E0264B1B6ABB60BB685A
S3150801183803F44073B3F5807F08D1BB6803F002034C
S31508011848002B03D04FF400433B621EE0BB6803F448
S315080118584073B3F5007F09D11A4B5B6A03F002039B
S31508011868002B03D049F640433B620EE0BB6803F4FC
S315080118784073B3F5407F1FD1124B1B6803F400333D
S31508011888002B19D0154B3B6216E015E0FFF772FDE0
S3150801189802460C4B5B689B0B03F0030301335B00A1
S315080118A8B2FBF3F33B6208E000BF06E000BF04E0C1
S315080118B800BF02E000BF00E000BF3B6A18462837B0
S315080118C8BD4680BD00100240046C0108146C01086D
S315080118D840787D0100093D00ABAAAAAAF0FA0200E0
S315080118E880B584B000AF78600023FB607B68002B65
S315080118F801D101237AE07B685B7CDBB2002B05D139
S315080119087B6800221A747868FBF788FC7B680222D0
S315080119185A74786800F070F80346002B04D07B687F
S3150801192804225A74012361E0786800F092F80346A4
S31508011938002B04D07B6804225A74012356E07B687D
S315080119481B685A687B681B6822F007025A607B681D
S315080119589B68002B05D0274B1B6B264A23F00103EE
S315080119681363244BDB6A23F460727B689B682149FD
S315080119781343CB627B685B68B3F1FF3F03D07B688F
S315080119885B68FB600EE00120FFF758FEF860FB680C
S31508011998002B04D17B6804225A74012326E0FB68CC
S315080119A8013BFB60FB681A0C7B681B6802F00F0297
S315080119B89A607B681B68FA6892B2DA60786800F000
S315080119C870F80346002B04D07B6804225A74012355
S315080119D80CE07B680022DA737B6801225A737B68FC
S315080119E801229A737B6801225A7400231846103714
S315080119F8BD4680BD006C004080B584B000AF7860F4
S31508011A080023FB607B68002B01D101231DE07B685D
S31508011A181B685A687B681B6822F008025A60FCF73B
S31508011A28D3FEF86009E0FCF7CFFE0246FB68D31A35
S31508011A38B3F57A7F01D9032307E07B681B685B68DE
S31508011A4803F00803002BEED0002318461037BD46CD
S31508011A5880BD80B584B000AF78600023FB60FCF7D1
S31508011A68B3FEF86009E0FCF7AFFE0246FB68D31A35
S31508011A78B3F57A7F01D903230FE07B681B685B6896
S31508011A8803F02003002BEED07B681B685A687B6835
S31508011A981B6842F010025A60002318461037BD46E3
S31508011AA880BD80B584B000AF78600023FB607B6891
S31508011AB81B685A687B681B6822F010025A60FCF793
S31508011AC883FEF86009E0FCF77FFE0246FB68D31A35
S31508011AD8B3F57A7F01D9032307E07B681B685B683E
S31508011AE803F02003002BEED0002318461037BD4615
S31508011AF880BD80B582B000AF78607B68002B01D1C4
S31508011B08012341E07B6893F83D30DBB2002B06D10F
S31508011B187B68002283F83C207868FCF787FB7B689A
S31508011B28022283F83D207B681A687B6804331946C4
S31508011B38104600F0B9FA7B68012283F846207B68CB
S31508011B48012283F83E207B68012283F83F207B68BF
S31508011B58012283F840207B68012283F841207B68AB
S31508011B68012283F842207B68012283F843207B6897
S31508011B78012283F844207B68012283F845207B6883
S31508011B88012283F83D20002318460837BD4680BD43
S31508011B9880B582B000AF78607B68002B01D101233C
S31508011BA841E07B6893F83D30DBB2002B06D17B68B0
S31508011BB8002283F83C20786800F039F87B6802220D
S31508011BC883F83D207B681A687B68043319461046F2
S31508011BD800F06AFA7B68012283F846207B680122AD
S31508011BE883F83E207B68012283F83F207B6801221F
S31508011BF883F840207B68012283F841207B6801220B
S31508011C0883F842207B68012283F843207B680122F6
S31508011C1883F844207B68012283F845207B680122E2
S31508011C2883F83D20002318460837BD4680BD80B491
S31508011C3883B000AF786000BF0C37BD4680BC7047DB
S31508011C4880B584B000AF786039603B68002B09D14C
S31508011C587B6893F83E30DBB2012B14BF01230023BE
S31508011C68DBB222E03B68042B09D17B6893F83F3045
S31508011C78DBB2012B14BF01230023DBB215E03B6855
S31508011C88082B09D17B6893F84030DBB2012B14BFC6
S31508011C9801230023DBB208E07B6893F84130DBB205
S31508011CA8012B14BF01230023DBB2002B01D001232A
S31508011CB863E03B68002B04D17B68022283F83E2047
S31508011CC813E03B68042B04D17B68022283F83F2082
S31508011CD80BE03B68082B04D17B68022283F8402075
S31508011CE803E07B68022283F841207B681B6801228E
S31508011CF83968184600F06EFC7B681B68214A9342CE
S31508011D0807D17B681B685A6C7B681B6842F40042DA
S31508011D185A647B681B681B4A934213D07B681B6805
S31508011D28B3F1804F0ED07B681B68174A934209D0D6
S31508011D387B681B68154A934204D07B681B68144A5A
S31508011D48934211D17B681B689B6803F00703FB6004
S31508011D58FB68062B10D07B681B681A687B681B68AA
S31508011D6842F001021A6007E07B681B681A687B68FB
S31508011D781B6842F001021A60002318461037BD464F
S31508011D8880BD00BF002C0140000400400008004047
S31508011D98000C004080B586B000AFF860B9607A607B
S31508011DA80023FB75FB6893F83C30012B01D102230C
S31508011DB8AEE0FB68012283F83C207B680C2B00F215
S31508011DC89F8001A252F823F0051E0108091F010880
S31508011DD8091F0108091F0108451E0108091F0108ED
S31508011DE8091F0108091F0108871E0108091F01089B
S31508011DF8091F0108091F0108C71E0108FB681B6896
S31508011E08B968184600F0C8F9FB681B689A69FB683F
S31508011E181B6842F008029A61FB681B689A69FB68A5
S31508011E281B6822F004029A61FB681B689969BB68FA
S31508011E381A69FB681B680A439A6164E0FB681B68B0
S31508011E48B968184600F00EFAFB681B689A69FB68B8
S31508011E581B6842F400629A61FB681B689A69FB6809
S31508011E681B6822F480629A61FB681B689969BB68DA
S31508011E781B691A02FB681B680A439A6143E0FB68F7
S31508011E881B68B968184600F057FAFB681B68DA69CF
S31508011E98FB681B6842F00802DA61FB681B68DA69A5
S31508011EA8FB681B6822F00402DA61FB681B68D969BA
S31508011EB8BB681A69FB681B680A43DA6123E0FB6891
S31508011EC81B68B968184600F0A1FAFB681B68DA6945
S31508011ED8FB681B6842F40062DA61FB681B68DA6909
S31508011EE8FB681B6822F48062DA61FB681B68D9699A
S31508011EF8BB681B691A02FB681B680A43DA6102E0B8
S31508011F080123FB7500BFFB68002283F83C20FB7D93
S31508011F1818461837BD4680BD80B584B000AF7860CD
S31508011F2839600023FB737B6893F83C30012B01D198
S31508011F380223B4E07B68012283F83C207B680222ED
S31508011F4883F83D207B681B689B68BB60BB6823F0E8
S31508011F587703BB60BB6823F47F43BB607B681B6858
S31508011F68BA689A603B681B68B3F5005F3ED0B3F55B
S31508011F78005F00F28780B3F5805F00F08680B3F5CD
S31508011F88805F7FD8702B1AD0702B7BD8602B50D0E6
S31508011F98602B77D8502B3CD0502B73D8402B58D070
S31508011FA8402B6FD8302B64D0302B6BD8202B60D0C0
S31508011FB8202B67D8002B5CD0102B5AD062E07B689F
S31508011FC818683B6899683B685A683B68DB6800F09B
S31508011FD8E2FA7B681B689B68BB60BB6843F07703BA
S31508011FE8BB607B681B68BA689A604FE07B681868AB
S31508011FF83B6899683B685A683B68DB6800F0CBFA26
S315080120087B681B689A687B681B6842F480429A60F9
S315080120183CE07B6818683B6859683B68DB681A4680
S3150801202800F042FA7B681B685021184600F099FAB5
S315080120382CE07B6818683B6859683B68DB681A4670
S3150801204800F060FA7B681B686021184600F089FA77
S315080120581CE07B6818683B6859683B68DB681A4660
S3150801206800F022FA7B681B684021184600F079FAC5
S315080120780CE07B681A683B681B681946104600F02D
S3150801208870FA03E00123FB7300E000BF7B680122B5
S3150801209883F83D207B68002283F83C20FB7B1846A1
S315080120A81037BD4680BD000080B485B000AF7860A2
S315080120B839607B681B68FB607B68334A93420FD09B
S315080120C87B68B3F1804F0BD07B68304A934207D0BF
S315080120D87B682F4A934203D07B682E4A934208D1DC
S315080120E8FB6823F07003FB603B685B68FA68134377
S315080120F8FB607B68244A93420FD07B68B3F1804F13
S315080121080BD07B68214A934207D07B68204A9342C1
S3150801211803D07B681F4A934208D1FB6823F44073AE
S31508012128FB603B68DB68FA681343FB60FB6823F0CE
S3150801213880023B685B691343FB607B68FA681A602F
S315080121483B689A687B68DA623B681A687B689A62B0
S315080121587B680D4A934203D13B681A697B681A63FF
S315080121687B6801225A617B681B6903F00103002B0E
S3150801217805D07B681B6923F001027B681A6100BFD9
S315080121881437BD4680BC7047002C01400004004046
S3150801219800080040000C004080B487B000AF7860A2
S315080121A839607B681B6A7B617B681B6A23F00102BD
S315080121B87B681A627B685B683B617B689B69FB6025
S315080121C8FB6823F07003FB60FB6823F00303FB60DD
S315080121D83B681B68FA681343FB607B6923F00203B3
S315080121E87B613B689B687A6913437B617B681C4AF8
S315080121F893420CD17B6923F008037B613B68DB6852
S315080122087A6913437B617B6923F004037B617B68E5
S31508012218134A934211D13B6923F480733B613B69A5
S3150801222823F400733B613B685B693A6913433B6175
S315080122383B689B693A6913433B617B683A695A600B
S315080122487B68FA689A613B685A687B685A637B684F
S315080122587A691A6200BF1C37BD4680BC704700BF41
S31508012268002C014080B487B000AF786039607B687C
S315080122781B6A7B617B681B6A23F010027B681A62FA
S315080122887B685B683B617B689B69FB60FB6823F439
S31508012298E043FB60FB6823F44073FB603B681B68FB
S315080122A81B02FA681343FB607B6923F020037B61F1
S315080122B83B689B681B017A6913437B617B681D4AE6
S315080122C893420DD17B6923F080037B613B68DB6808
S315080122D81B017A6913437B617B6923F040037B61A0
S315080122E87B68144A934213D13B6923F480633B61A3
S315080122F83B6923F400633B613B685B699B003A6968
S3150801230813433B613B689B699B003A6913433B61ED
S315080123187B683A695A607B68FA689A613B685A68C1
S315080123287B689A637B687A691A6200BF1C37BD465F
S3150801233880BC7047002C014080B487B000AF786034
S3150801234839607B681B6A7B617B681B6A23F4807228
S315080123587B681A627B685B683B617B68DB69FB6043
S31508012368FB6823F07003FB60FB6823F00303FB603B
S315080123783B681B68FA681343FB607B6923F400739F
S315080123887B613B689B681B027A6913437B617B689F
S315080123981D4A93420DD17B6923F400637B613B682F
S315080123A8DB681B027A6913437B617B6923F48063C3
S315080123B87B617B68144A934213D13B6923F48053A2
S315080123C83B613B6923F400533B613B685B691B012D
S315080123D83A6913433B613B689B691B013A69134395
S315080123E83B617B683A695A607B68FA68DA613B68D7
S315080123F85A687B68DA637B687A691A6200BF1C3790
S31508012408BD4680BC704700BF002C014080B487B028
S3150801241800AF786039607B681B6A3B617B681B6A19
S3150801242823F480527B681A627B685B687B617B68E8
S31508012438DB69FB60FB6823F4E043FB60FB6823F474
S315080124484073FB603B681B681B02FA681343FB6011
S315080124583B6923F400533B613B689B681B033A6954
S3150801246813433B617B680F4A934209D17B6923F47D
S3150801247880437B613B685B699B017A6913437B618E
S315080124887B687A695A607B68FA68DA613B685A68D0
S315080124987B681A647B683A691A6200BF1C37BD46AD
S315080124A880BC7047002C014080B487B000AFF86043
S315080124B8B9607A60FB681B6A7B61FB681B6A23F053
S315080124C80102FB681A62FB689B693B613B6923F059
S315080124D8F0033B617B681B013A6913433B617B69DE
S315080124E823F00A037B617A69BB6813437B61FB683E
S315080124F83A699A61FB687A691A6200BF1C37BD4650
S3150801250880BC704780B487B000AFF860B9607A605C
S31508012518FB681B6A7B61FB681B6A23F01002FB6870
S315080125281A62FB689B693B613B6923F470433B610B
S315080125387B681B033A6913433B617B6923F0A00354
S315080125487B61BB681B017A6913437B61FB683A693E
S315080125589A61FB687A691A6200BF1C37BD4680BC56
S31508012568704780B485B000AF786039607B689B682E
S31508012578FB60FB6823F07003FB603A68FB6813434A
S3150801258843F00703FB607B68FA689A6000BF143753
S31508012598BD4680BC704780B487B000AFF860B960A3
S315080125A87A603B60FB689B687B617B6923F47F43A0
S315080125B87B613B681A027B681A43BB6813437A69CD
S315080125C813437B61FB687A699A6000BF1C37BD466D
S315080125D880BC704780B487B000AFF860B9607A608C
S315080125E8BB6803F01F03012202FA03F37B61FB6848
S315080125F81A6A7B69DB431A40FB681A62FB681A6A1E
S31508012608BB6803F01F03796801FA03F31A43FB68E9
S315080126181A6200BF1C37BD4680BC704780B485B0B6
S3150801262800AF786039607B6893F83C30012B01D19B
S3150801263802234BE07B68012283F83C207B6802224F
S3150801264883F83D207B681B685B68FB607B681B68B1
S315080126589B68BB60FB6823F07003FB603B681B68DB
S31508012668FA681343FB607B681B68FA685A607B68DB
S315080126781B68194A934213D07B681B68B3F1804FCC
S315080126880ED07B681B68154A934209D07B681B687C
S31508012698134A934204D07B681B68124A93420CD1A9
S315080126A8BB6823F08003BB603B685B68BA68134361
S315080126B8BB607B681B68BA689A607B68012283F8E5
S315080126C83D207B68002283F83C20002318461437EE
S315080126D8BD4680BC704700BF002C0140000400407D
S315080126E800080040000C004080B582B000AF786051
S315080126F87B68002B01D1012342E07B6893F84130BE
S31508012708DBB2002B06D17B68002283F84020786863
S31508012718FBF796FE7B68242283F841207B681B68B1
S31508012728DA687B681B6822F40052DA60786800F078
S31508012738B3FE7B681B681A697B681B6822F490429A
S315080127481A617B681B685A697B681B6822F02A022A
S315080127585A617B681B68DA687B681B6842F4005211
S31508012768DA607B6800225A647B68202283F8412054
S315080127787B68202283F842207B6800225A6300235B
S3150801278818460837BD4680BD80B485B000AFF860E5
S31508012798B9601346FB80FB6893F84130DBB2202BFE
S315080127A821D1BB68002B02D0FB88002B01D101235C
S315080127B81AE0FB68BA681A62FB68FA889A84FB68A1
S315080127C8FA88DA84FB6800225A64FB68212283F8AE
S315080127D84120FB681B68DA68FB681B6842F08002BF
S315080127E8DA60002300E0022318461437BD4680BC88
S315080127F8704780B58CB000AFF860B9601346FB80A6
S31508012808FB6893F84230DBB2202B4AD1BB68002B10
S3150801281802D0FB88002B01D1012343E0FB68012282
S315080128281A63FB6800225A63FB881A46B968F8686E
S3150801283800F0FDFB034687F82F3097F82F30002B59
S315080128482CD1FB681B6B012B25D100233B61FB6847
S315080128581B681B683B61FB681B685B683B613B69D6
S31508012868FB681B680C33BB61BB6953E8003F7B6196
S315080128787B6943F01003BB62FB681B680C33BA6AB1
S315080128887A623B62396A7A6A41E80023FB61FB6925
S31508012898002BE5D102E0012387F82F3097F82F306E
S315080128A800E0022318463037BD4680BD80B5A2B080
S315080128B800AF78600123C7F884307B681B680C333E
S315080128C83B663B6E53E8003FFB65FB6D23F4F073EB
S315080128D8C7F880307B681B680C33D7F88020FA66FE
S315080128E8BB66B96EFA6E41E800237B667B6E002BE0
S315080128F8E3D17B681B681433FB64FB6C53E8003F20
S31508012908BB64BB6C23F00103FB677B681B68143344
S31508012918FA6FBA657B65796DBA6D41E800233B653F
S315080129283B6D002BE5D17B681B6B012B19D17B68A5
S315080129381B680C33BB63BB6B53E8003F7B637B6B3C
S3150801294823F01003BB677B681B680C33BA6F7A647C
S315080129583B64396C7A6C41E80023FB63FB6B002BFB
S31508012968E5D17B689B6B002B0FD07B681B685B697D
S3150801297803F08003002B04D07B689B6B534A5A6388
S3150801298803E07B689B6B00225A637B68DB6B002B31
S315080129980FD07B681B685B6903F04003002B04D0E2
S315080129A87B68DB6B4A4A5A6303E07B68DB6B002268
S315080129B85A637B681B685B6903F08003002B2DD07B
S315080129C87B681B6814337B627B6A53E8003F3B626A
S315080129D83B6A23F080037B677B681B6814337A6F2D
S315080129E83A63FB62F96A3A6B41E80023BB62BB6A40
S315080129F8002BE5D17B689B6B002B0FD07B689B6B03
S31508012A081846FDF745FC0346002B04D07B689B6BEB
S31508012A1800225A6302E00023C7F884307B681B68E2
S31508012A285B6903F04003002B30D07B681B681433BD
S31508012A383B613B6953E8003FFB60FB6823F04003B1
S31508012A483B677B681B6814333A6FFA61BB61B969DE
S31508012A58FA6941E800237B617B69002BE5D17B682C
S31508012A68DB6B002B12D07B68DB6B1846FDF710FC75
S31508012A780346002B07D07B68DB6B00225A630123C8
S31508012A88C7F8843002E00023C7F88430D7F88430C1
S31508012A98012B16D17B680022DA847B680022DA8545
S31508012AA87B6800225A647B68202283F841207B6868
S31508012AB8202283F842207B6800221A63786800F08E
S31508012AC8ADFA002318468837BD4680BD95310108F9
S31508012AD8F531010880B5BAB000AF78607B681B6824
S31508012AE81B68C7F8E4307B681B68DB68C7F8E03001
S31508012AF87B681B685B69C7F8DC300023C7F8D830E0
S31508012B080023C7F8D430D7F8E43003F00F03C7F821
S31508012B18D830D7F8D830002B0FD1D7F8E43003F0DE
S31508012B282003002B09D0D7F8E03003F02003002B47
S31508012B3803D0786800F0F1FB5BE2D7F8D830002BB0
S31508012B4800F0DE80D7F8DC3003F00103002B06D14C
S31508012B58D7F8E03003F49073002B00F0D180D7F84A
S31508012B68E43003F00103002B0BD0D7F8E03003F467
S31508012B788073002B05D07B685B6C43F001027B6888
S31508012B885A64D7F8E43003F00403002B0BD0D7F8BE
S31508012B98DC3003F00103002B05D07B685B6C43F03E
S31508012BA802027B685A64D7F8E43003F00203002B63
S31508012BB80BD0D7F8DC3003F00103002B05D07B686E
S31508012BC85B6C43F004027B685A64D7F8E43003F077
S31508012BD80803002B11D0D7F8E03003F02003002BA7
S31508012BE805D1D7F8DC3003F00103002B05D07B6843
S31508012BF85B6C43F008027B685A647B685B6C002B44
S31508012C0800F0F281D7F8E43003F02003002B08D04E
S31508012C18D7F8E03003F02003002B02D0786800F0DB
S31508012C287CFB7B681B685B6903F04003002B14BFB8
S31508012C3801230023DBB2C7F8D4307B685B6C03F049
S31508012C480803002B03D1D7F8D430002B4FD0786866
S31508012C5800F026FA7B681B685B6903F04003002BC2
S31508012C6841D07B681B681433C7F89C30D7F89C3069
S31508012C7853E8003FC7F89830D7F8983023F040034F
S31508012C88C7F8D0307B681B681433D7F8D020C7F843
S31508012C98A820C7F8A430D7F8A410D7F8A82041E87F
S31508012CA80023C7F8A030D7F8A030002BD9D17B6804
S31508012CB8DB6B002B13D07B68DB6B7E4A5A637B6818
S31508012CC8DB6B1846FDF7E4FA0346002B16D07B683A
S31508012CD8DB6B5B6B7A68D26B104698470EE07868AF
S31508012CE800F093F90AE0786800F08FF906E0786849
S31508012CF800F08BF97B6800225A6475E100BF73E11D
S31508012D087B681B6B012B40F04F81D7F8E43003F041
S31508012D181003002B00F04881D7F8E03003F01003C0
S31508012D28002B00F041810023BB607B681B681B6888
S31508012D38BB607B681B685B68BB60BB687B681B6894
S31508012D485B6903F04003002B00F0B6807B68DB6BF8
S31508012D581B685B68A7F8BE30B7F8BE30002B00F0D1
S31508012D6845817B689B8DB7F8BE209A4280F03E81E3
S31508012D787B68B7F8BE20DA857B68DB6B9B69202BF5
S31508012D8800F088807B681B680C33C7F88830D7F849
S31508012D98883053E8003FC7F88430D7F8843023F4DD
S31508012DA88073C7F8B8307B681B680C33D7F8B82026
S31508012DB8C7F89420C7F89030D7F89010D7F8942018
S31508012DC841E80023C7F88C30D7F88C30002BD9D1C5
S31508012DD87B681B6814337B677B6F53E8003F3B6747
S31508012DE83B6F23F00103C7F8B4307B681B681433BB
S31508012DF8D7F8B420C7F88020FB67F96FD7F8802081
S31508012E0841E80023BB67BB6F002BE1D17B681B68D0
S31508012E1814333B663B6E53E8003FFB65FB6D23F0B5
S31508012E284003C7F8B0307B681B681433D7F8B0205D
S31508012E38FA66BB66B96EFA6E41E800237B667B6E55
S31508012E48002BE3D17B68202283F842207B68002285
S31508012E581A637B681B680C33FB64FB6C53E8003FF9
S31508012E68BB64BB6C23F01003C7F8AC307B681B68DE
S31508012E780C33D7F8AC20BA657B65796DBA6D41E82C
S31508012E8800233B653B6D002BE3D17B68DB6B18465A
S31508012E98FDF7C3F97B6802225A637B689A8D7B68BA
S31508012EA8DB8D9BB2D31A9BB219467868FAF762FA90
S31508012EB89CE000BF6D3101087B689A8D7B68DB8DC4
S31508012EC89BB2D31AA7F8CE307B68DB8D9BB2002B51
S31508012ED800F08E80B7F8CE30002B00F089807B6829
S31508012EE81B680C33BB63BB6B53E8003F7B637B6B87
S31508012EF823F49073C7F8C8307B681B680C33D7F876
S31508012F08C8207A643B64396C7A6C41E80023FB6310
S31508012F18FB6B002BE3D17B681B6814337B627B6AE6
S31508012F2853E8003F3B623B6A23F00103C7F8C43004
S31508012F387B681B681433D7F8C4203A63FB62F96ABD
S31508012F483A6B41E80023BB62BB6A002BE3D17B6875
S31508012F58202283F842207B6800221A637B681B6853
S31508012F680C333B613B6953E8003FFB60FB6823F080
S31508012F781003C7F8C0307B681B680C33D7F8C02024
S31508012F88FA61BB61B969FA6941E800237B617B6922
S31508012F98002BE3D17B6802225A63B7F8CE3019466B
S31508012FA87868FAF7E7F923E0D7F8E43003F08003FD
S31508012FB8002B09D0D7F8E03003F08003002B03D0A3
S31508012FC8786800F043F914E0D7F8E43003F04003D1
S31508012FD8002B0ED0D7F8E03003F04003002B08D0B9
S31508012FE8786800F082F904E000BF02E000BF00E05B
S31508012FF800BFE837BD4680BD80B483B000AF7860AE
S3150801300800BF0C37BD4680BC704780B483B000AF9B
S31508013018786000BF0C37BD4680BC704780B483B062
S3150801302800AF786000BF0C37BD4680BC704780B4D6
S3150801303885B000AFF860B9601346FB80FB68BA68CB
S315080130489A62FB68FA889A85FB68FA88DA85FB68C2
S3150801305800225A64FB68222283F84220FB681B690E
S31508013068002B07D0FB681B68DA68FB681B6842F403
S315080130788072DA60FB681B685A69FB681B6842F04C
S3150801308801025A61FB681B68DA68FB681B6842F02B
S315080130982002DA60002318461437BD4680BC7047FB
S315080130A880B495B000AF78607B681B680C337B6386
S315080130B87B6B53E8003F3B633B6B23F49073FB64DC
S315080130C87B681B680C33FA6C3A64FB63F96B3A6CD8
S315080130D841E80023BB63BB6B002BE5D17B681B6802
S315080130E814333B623B6A53E8003FFB61FB6923F0F3
S315080130F80103BB647B681B681433BA6CFA62BB624A
S31508013108B96AFA6A41E800237B627B6A002BE5D132
S315080131187B681B6B012B19D17B681B680C33FB6019
S31508013128FB6853E8003FBB60BB6823F010037B6468
S315080131387B681B680C337A6CBA617B617969BA69F1
S3150801314841E800233B613B69002BE5D17B682022D6
S3150801315883F842207B6800221A6300BF5437BD46AC
S3150801316880BC704780B584B000AF78607B685B6ABD
S31508013178FB60FB680022DA85FB680022DA84F868B6
S31508013188FFF743FF00BF1037BD4680BD80B584B041
S3150801319800AF78607B685B6AFB60FB689B6B002203
S315080131A85A63FB68DB6B002B04D0FB68DB6B5B6B34
S315080131B8002B17D1FB680022DA84FB680022DA851E
S315080131C8FB6800225A64FB68202283F84120FB68C1
S315080131D8202283F84220FB6800221A63F868FFF761
S315080131E81DFF00E000BF1037BD4680BD80B584B01D
S315080131F800AF78607B685B6AFB60FB68DB6B002263
S315080132085A63FB689B6B002B04D0FB689B6B5B6B53
S31508013218002B17D1FB680022DA84FB680022DA85BD
S31508013228FB6800225A64FB68202283F84120FB6860
S31508013238202283F84220FB6800221A63F868FFF700
S31508013248EDFE00E000BF1037BD4680BD80B485B0ED
S3150801325800AF78607B6893F84130DBB2212B3ED109
S315080132687B689B68B3F5805F14D17B681B69002B63
S3150801327810D17B681B6AFB60FB681B881A467B684A
S315080132881B68C2F308025A607B681B6A9A1C7B682A
S315080132981A6208E07B681B6A591C7A6811621A78EF
S315080132A87B681B685A607B68DB8C9BB2013B9BB2C7
S315080132B87A681946D184002B0FD17B681B68DA68AE
S315080132C87B681B6822F08002DA607B681B68DA680B
S315080132D87B681B6842F04002DA60002300E002239B
S315080132E818461437BD4680BC704780B582B000AF12
S315080132F878607B681B68DA687B681B6822F040027D
S31508013308DA607B68202283F841207868FAF754F84E
S31508013318002318460837BD4680BD80B58CB000AF76
S3150801332878607B6893F84230DBB2222B40F0AE8096
S315080133387B689B68B3F5805F17D17B681B69002B8F
S3150801334813D10023FB627B689B6ABB627B681B6897
S315080133585B689BB2C3F308039AB2BB6A1A807B6897
S315080133689B6A9A1C7B689A6226E07B689B6AFB6261
S315080133780023BB627B689B68B3F5805F07D07B68CF
S315080133889B68002B0AD17B681B69002B06D17B68D1
S315080133981B685B68DAB2FB6A1A7008E07B681B6807
S315080133A85B68DBB203F07F03DAB2FB6A1A707B68E3
S315080133B89B6A5A1C7B689A627B68DB8D9BB2013BC8
S315080133C89BB27A681946D185002B5DD17B681B6843
S315080133D8DA687B681B6822F02002DA607B681B685A
S315080133E8DA687B681B6822F48072DA607B681B6876
S315080133F85A697B681B6822F001025A617B68202298
S3150801340883F842207B6800225A637B681B6B012B71
S3150801341835D17B6800221A637B681B680C337B618C
S315080134287B6953E8003F3B613B6923F010037B62E4
S315080134387B681B680C337A6A3A62FB61F9693A6AEE
S3150801344841E80023BB61BB69002BE5D17B681B6892
S315080134581B6803F01003102B0AD10023FB607B6855
S315080134681B681B68FB607B681B685B68FB60FB68FD
S315080134787B689B8D19467868F9F77CFF02E07868BE
S31508013488FFF7BAFD002302E0002300E002231846ED
S315080134983037BD4680BD000080B584B000AF78607E
S315080134A87B681B681B6923F440517B68DA687B686B
S315080134B81B680A431A617B689A687B681B691A4301
S315080134C87B685B691343BB607B681B68DB6823F40D
S315080134D8B05323F00C037A681268B9680B43D360B2
S315080134E87B681B685B6923F440717B689A697B680A
S315080134F81B680A435A617B681B682C4A934203D1A5
S31508013508FDF738FFF86002E0FDF720FFF860FA6872
S3150801351813469B0013449A001A447B685B689B0010
S31508013528B2FBF3F3224AA2FB03235B091901FA68E2
S3150801353813469B0013449A001A447B685B689B00F0
S31508013548B2FBF3F21A4BA3FB02035B09642000FBE7
S3150801355803F3D31A1B013233154AA2FB03235B096A
S3150801356803F0F0031944FA6813469B0013449A00BA
S315080135781A447B685B689B00B2FBF3F20C4BA3FB0E
S3150801358802035B09642000FB03F3D31A1B013233D8
S31508013598074AA2FB03235B0903F00F027B681B6832
S315080135A80A449A6000BF1037BD4680BD00380140FD
S315080135B81F85EB51002B2DE9F0471D46BBBF03F1CB
S315080135C800431D4600232D2388B01446B8BF144668
S315080135D8129A109E1370149BDDF84CA023F020084C
S315080135E8B8F1460F05D0B8F1450F00D101360223C7
S315080135F800E0032307AA049206AACDE902A2CDE9A7
S31508013608003622462B4600F003FFB8F1470F074656
S3150801361819D1119BDB070ED500EB060900220023F9
S3150801362820462946F5F728FA08B1CDF81C90302224
S31508013638079B4B451ED33846079B159ADB1B136018
S3150801364808B0BDE8F087B8F1460F00EB0609E5D1E1
S315080136580378302B0AD10022002320462946F5F79C
S315080136680BFA18B9C6F10106CAF80060DAF800308B
S315080136789944D3E7591C07911A70D9E7F7B5002970
S31508013688B6BF2D232B23494209290270437029DD28
S315080136980DF107031D460A27B1FBF7F61A4607FB7C
S315080136A81614303402F8014C0C46632C314603F1E2
S315080136B8FF33F1DC3031941E03F8011C2346411C03
S315080136C8AB420AD30DF109039B1AAC4288BF002302
S315080136D802330344181A03B0F0BD13F8016B01F855
S315080136E8016FEDE7302330318370C170031DF1E7AF
S315080136F82DE9F04F91B00C46DDF8688016461F464D
S31508013708054600F0BDFD036818460893F4F788FDD9
S3150801371800230E93D8F800300990073323F00703DE
S3150801372803F1080294F818A0D4F800B0C8F80020E4
S31508013738D3E9008929F000430B93CDF828804FF087
S31508013748FF32DDE90A01C4E912899C4BF5F7C6F986
S3150801375870BBDDE90A014FF0FF32984BF5F7A0F97E
S3150801376830BB0022002340464946F5F78FF910B1C8
S315080137782D2384F84330924A924BBAF1470F8CBFEE
S315080137889046984603234FF0000923612BF004035A
S31508013798236033462146284600970FAA00F0D4F934
S315080137A8013040F090804FF0FF3011B0BDE8F08F3E
S315080137B842464B4640464946F5F790F948B14B46C5
S315080137C8002BB8BF2D23804AB8BF84F843307F4BF6
S315080137D8D3E763680AF0DF015A1C3FD10623636001
S315080137E800224BF48063236006920EAACDE904A24F
S315080137F80DAA03920DF13302CDE9013263684246F7
S31508013808009328464B460A91FFF7D4FE0A99804643
S3150801381847290D9928D1C81C02DB6368994240DDFE
S31508013828AAF1020A5FFA8AFA5246013904F15000E6
S315080138380D91FFF723FF0E9A81461318012A236172
S3150801384802DC2268D20701D5013323619DF833309A
S31508013858002B9ED02D2384F843309AE74729BFD1F8
S31508013868002BBDD10123BAE7BAF1650FDCD9BAF144
S31508013878660F18D1002963680BDD216113B922681F
S31508013888D00702D501330B4423614FF00009A1651E
S31508013898DCE713B92268D20701D50233F4E7012315
S315080138A8F2E74FF0670A0E9B994205DB2368216107
S315080138B8D807EAD54B1CE7E70029CCBF0122C1F195
S315080138C802021344E0E723685A0507D423694246E6
S315080138D831462846B84701302BD164E7BAF1650F56
S315080138E840F2DC80D4E9120100220023F5F7C4F876
S315080138F8002833D0012331462846354AB8470130CE
S315080139083FF451AFDDE90D38434502DB2368D80793
S315080139180FD5DDE9082331462846B84701303FF473
S3150801392842AF4FF0000908F1FF3804F11A0AC845F1
S3150801393809DC23689B0700F10281E0680F9B98421E
S31508013948B8BF184631E70123524631462846B847D3
S3150801395801303FF428AF09F10109E8E70D9B002B6F
S3150801396838DC012331462846194AB84701303FF45D
S315080139781AAFDDE90D3959EA030302D12368D907D4
S31508013988D7D5DDE9082331462846B84701303FF43B
S315080139980AAF4FF0000A04F11A0B0D9B5B42534517
S315080139A801DC4B4693E701235A4631462846B84770
S315080139B801303FF4F8AE0AF1010AEEE7FFFFEF7F9F
S315080139C8286C0108246C0108306C01082C6C010864
S315080139D8346C0108A36DDDF838A05345A8BF5346D2
S315080139E8002B994636DC4FF0000B29EAE97904F1F0
S315080139F81A02A36D0A93A3EB09035B4531DC0D9BF8
S31508013A089A453ADC2368DA0737D40D9BAAEB0309EA
S31508013A180A9BAAEB03039945A8BF9946B9F1000F72
S31508013A2833DC4FF0000829EAE97904F11A0B0D9BF2
S31508013A38AAEB0303A3EB090343457FF77AAF0123EF
S31508013A485A4631462846B84701303FF4ACAE08F124
S31508013A580108ECE7424631462846B8470130C2D143
S31508013A68A1E60123314628460A92B84701303FF4B0
S31508013A789AAE0A9A0BF1010BBBE73146DDE9082331
S31508013A882846B8470130C0D18DE60A9A4B463146D1
S31508013A9828464244B8470130C3D184E6DDF838A040
S31508013AA8BAF1010F01DCDB0736D501234246314657
S31508013AB82846B84701303FF476AEDDE90823314692
S31508013AC82846B84701303FF46EAED4E91201002200
S31508013AD800230AF1FF3AF4F7CFFFC0B9534608F1B4
S31508013AE8010231462846B84701300CD15BE6012365
S31508013AF85A4631462846B84701303FF454AE08F1CC
S31508013B080108D045F3DB4B4604F15002E0E64FF0D5
S31508013B18000804F11A0BF4E701234246E1E70123F9
S31508013B284A4631462846B84701303FF43CAE08F1C3
S31508013B380108E3680F995B1A4345F0DCFDE64FF087
S31508013B48000804F11909F4E72DE9F04716469846DD
S31508013B588A680B6907469342B8BF1346336091F8DA
S31508013B6843200C46DDF820900AB1013333602368F7
S31508013B78990642BF336802333360256815F006058E
S31508013B8806D104F1190AE36832689B1AAB422BDCA1
S31508013B9894F843302268003B18BF0123920630D4B3
S31508013BA84146384604F14302C847013023D0236801
S31508013BB8226903F00603042B14BF002533684FF066
S31508013BC8000608BFE56804F11A0408BFED1A54F897
S31508013BD8123C08BF25EAE5759342C4BF9B1AED183E
S31508013BE8B5421AD1002008E0012352464146384613
S31508013BF8C847013003D14FF0FF30BDE8F0870135DA
S31508013C08C1E73020E11881F843005A1C94F8451099
S31508013C182244023382F84310C2E701232246414669
S31508013C283846C8470130E6D00136D9E72DE9FF47B6
S31508013C380F7E9146782F80460C469A460C9E01F1CE
S31508013C48430207D8622F0AD8002F00F0D180582FCF
S31508013C5800F0B88004F1420684F842703AE0A7F108
S31508013C686303152BF6D801A151F823F0CD3C0108B9
S31508013C78E13C01085D3C01085D3C01085D3C010821
S31508013C885D3C0108E13C01085D3C01085D3C010811
S31508013C985D3C01085D3C0108DF3D01080B3D010853
S31508013CA8993D01085D3C01085D3C0108013E010892
S31508013CB85D3C01080B3D01085D3C01085D3C0108B6
S31508013CC8A13D010833681A1D1B68326004F14206D2
S31508013CD884F8423001239CE033682068191D316055
S31508013CE8060601D51D6803E04506FBD5B3F900505C
S31508013CF8002D03DA2D236D4284F843300A235848E8
S31508013D0811E021683368080653F8045B02D44906AA
S31508013D1848BFADB26F2F336014BF0A230823504832
S31508013D28002184F843106668002EA66005DB216821
S31508013D382E4321F0040121604BD01646B5FBF3F159
S31508013D4803FB1157C75D06F8017D2F46BB420D4691
S31508013D58F4D9082B0BD12368DF0708D523696168CD
S31508013D689942DEBF302306F8013C06F1FF36921B5D
S31508013D7822614B4621464046CDF800A003AAFFF723
S31508013D88E3FE01304AD14FF0FF3004B0BDE8F087B1
S31508013D98236843F0200323607827324884F845705E
S31508013DA8236831681F0651F8045B02D45F0648BFC9
S31508013DB8ADB23160D90744BF43F0200323601DB172
S31508013DC81023ADE72648E9E7236823F02003236093
S31508013DD8F6E71646BDE733682568181D6169306038
S31508013DE82E061B6801D5196002E06806FBD51980FD
S31508013DF8002316462361BCE7336800211A1D326081
S31508013E081E686268304600F03FFA08B1801B606098
S31508013E1863682361002384F84330AAE73246494692
S31508013E2840462369D0470130ADD023689B0713D490
S31508013E38E068039B9842B8BF1846A6E701233246AD
S31508013E4849464046D04701309DD00135E368039974
S31508013E585B1AAB42F2DCEBE7002504F11906F5E734
S31508013E68366C0108476C0108002310B50446C0E9F9
S31508013E780033C0E90433836081814366C281836163
S31508013E88194608225C3000F0FFF80D4B246263627C
S31508013E980C4BA3620C4BE3620C4B23630C4B9C4201
S31508013EA806D003F16802944202D0D0339C4205D168
S31508013EB804F15800BDE8104000F0DEB910BD00BF96
S31508013EC8A15E0108C35E0108FB5E01081F5F0108C0
S31508013ED8640E0020024A0349034800F0A5B800BF4A
S31508013EE878000020455701088800002041680C4BD6
S31508013EF810B59942044601D001F020FCA168094B86
S31508013F08994202D0204601F019FCE168064B99420C
S31508013F1804D02046BDE8104001F010BC10BD00BF12
S31508013F28640E0020CC0E0020340F002010B50B4B70
S31508013F380B4C0C4A20461A6004210022FFF794FF0D
S31508013F4804F1680001220921FFF78EFF04F1D00068
S31508013F580222BDE810401221FFF786BF9C0F0020F8
S31508013F68640E0020DD3E0108014800F086B900BF4D
S31508013F78A10F0020014800F081B900BFA10F002058
S31508013F8810B50446FFF7F0FF236A1BB1BDE81040D8
S31508013F98FFF7F0BF044B2362044B1B68002BF5D1CE
S31508013FA8FFF7C4FFF2E700BFF53E01089C0F0020A2
S31508013FB830B51446002C05461A469BB005DA8B23FC
S31508013FC803604FF0FF301BB030BD4FF40273ADF8F4
S31508013FD80C304FF0000319930CBF234604F1FF3345
S31508013FE8029305934FF6FF7300910491ADF80E30CD
S31508013FF869461E9B01F03CF8431CBCBF8B232B600A
S31508014008002CE0D00022009B1A70DCE707B5009364
S3150801401813460A46014603480068FFF7C9FF03B075
S315080140285DF804FB840000202DE9F8430746884615
S3150801403814460026D4E90195B9F1010905D524687C
S31508014048002CF7D13046BDE8F883AB89012B07D98F
S31508014058B5F90E30013303D029463846C047064319
S315080140686835E9E70FB407B5064904AB086853F894
S31508014078042B8168019301F01FF903B05DF804EB7D
S3150801408804B070478400002003460244934200D1D5
S31508014098704703F8011BF9E738B50B4B04461D6849
S315080140A86B6B53B9242001F01FFA0246686320B9DD
S315080140B83D21064B064800F003F92046696BBDE821
S315080140C8384000F007B800BF84000020586C010882
S315080140D86F6C01082DE9F04100230C46D0E900016F
S315080140E84C4AF5F783F84FF46161002ABCBF02F51B
S315080140F8A83202F5C072B2FBF1F301FB13224FF0A5
S315080141083C01A360B2FBF1F301FB132222604FF0D5
S31508014118070200F52F20ACBF00F66C2000F66B20CD
S315080141286360C31C93FBF2F2C2EBC2029B1A3A49BB
S3150801413855D50733A361A0F50E33A3F52C7393FB65
S31508014148F1F1364B40F2B45C03FB010048F6AC6367
S31508014158B0FBF3F3B0FBFCF203449B1A304A40F276
S315080141686D17B0FBF2F29B1AB3FBF7F26426B3FBA1
S31508014178FCF3B2FBF6F5EB1A0344992007FB123355
S3150801418803EB83070237B7FBF0FC4FF0050800FB82
S315080141980CF00230B0FBF8F003F1010EAEEB0000AB
S315080141A840F2F95E77458CBF6FF009070227674425
S315080141B84FF4C87C0CFB0121012F98BF0131B3F5D7
S315080141C8997F12D3A3F59973E3610023A1F26C7160
S315080141D8E060C4E9047120462362BDE8F08100283D
S315080141E8A361A8DB90FBF1F1ABE712F0030F02D14B
S315080141F806FB15255DB94FF4C875B2FBF5F605FB3F
S315080142081622B2FA82F252093B331344DCE7012239
S31508014218FAE700BF80510100B13A02004FC5FDFF18
S31508014228B03A0200014B1868704700BF84000020A5
S3150801423870B500260C4D0D4C641BA410A64209D175
S3150801424802F006F900260A4D0A4C641BA410A64278
S3150801425805D170BD55F8043B98470136EEE755F880
S31508014268043B98470136F2E7FC6F0108FC6F010821
S31508014278FC6F010800700108704770477047000015
S3150801428800487047C4010020034610B5C9B2024464
S315080142989342184601D1002003E0047801338C4281
S315080142A8F6D110BD0A44914200F1FF3300D1704797
S315080142B810B511F8014B914203F8014FF9D110BD18
S315080142C81FB514461A46094B05461B68D8684CB1EA
S315080142D8074BCDE9013400912B46064901F020FE2A
S315080142E801F0E6FF044B1C46F3E700BF84000020F3
S315080142F8C76C0108D46C0108026D01082DE9F74F4E
S3150801430803690C690746A3427EDB013CA30000F159
S31508014318140501F11408009305EB8403019358F871
S31508014328243055F8242001339A42B2FBF3F608EBF8
S3150801433884092ED34FF0000AC446AE46D3465CF824
S31508014348043B98B206FB00A01B0C020C06FB0323D0
S31508014358DEF8002080B292B2121A5A44DEF800003A
S315080143684FEA134A9BB2C3EB224303EB104392B2BB
S3150801437842EA0342E1454FEA234B4EF8042BDED2C3
S31508014388009BEB582BB9019B043B9D421A462FD338
S315080143983C61384601F078FC002825DB29460020CF
S315080143A858F8042BD1F800C01FFA82FE1FFA8CF3BD
S315080143B8A3EB0E030344120CC2EB234202EB1C4285
S315080143C89BB243EA0243C1454FEA224041F8043BFE
S315080143D8E6D255F8242005EB840322B9043B9D420D
S315080143E81A460BD33C610136304603B0BDE8F08F57
S315080143F81268043B002ACBD1013CC6E71268043B84
S31508014408002AEFD1013CEAE70020EEE700000000A8
S315080144182DE9F04F14461D46C76997B08146CDE97F
S315080144280645239E7FB9102001F05EF80246C9F8B1
S315080144381C0020B9EF21AC4BAC48FFF741FFC0E996
S3150801444801770760C760D9F81C30196859B15A68E5
S31508014458012393404A608B60484601F0E3F900223C
S31508014468D9F81C301A602B1EAFBF0023012223F08E
S3150801447800430793A8BF3360DDF81C809C4BB8BF7F
S31508014488326033EA080312D142F20F73229A136093
S31508014498C8F31303234300F05E85249BDFF854A26F
S315080144A8002B00F060850AF1030300F05ABDDDE927
S315080144B80623CDE90C23DDE90C0100220023F4F7D4
S315080144C8DBFA074658B10123229A1360249B13B1D4
S315080144D8894B249A1360DFF824A200F044BD14AB73
S315080144E8019315AB00934846DDE90C2301F07CFCE2
S315080144F8C8F30A560390002E78D0DDE90C010D9B06
S31508014508A6F2FF36C3F3130343F07F5343F440136C
S315080145181297194600227A4BF3F78EFE6CA3D3E954
S315080145280023F4F741F86CA3D3E90023F3F786FED1
S31508014538044630460D46F3F7CDFF69A3D3E90023B0
S31508014548F4F732F802460B4620462946F3F776FE73
S3150801455804460D46F4F7D8FA0022074600232046F2
S315080145682946F4F793FA40B13846F3F7B3FF2246DA
S315080145782B46F4F781FA00B9013F162F54D8DDE91D
S315080145880C01604B03EBC703D3E90023F4F77EFA62
S3150801459800284BD00023013F0F93149B9B1B5A1EDF
S315080145A849BFC3F10103002304930023099254BFA9
S315080145B804930993002F3BDB099B0E973B44099308
S315080145C800230A93209B092B65D8052BC4BF043BF6
S315080145D82093209BC8BF0024A3F10203D8BF012456
S315080145E8032B64D8DFE803F05355382CDDE9146347
S315080145F81E4406F23243202BC1BFC3F1400308FA11
S3150801460803F806F2124324FA03F3D6BFC3F12003CB
S3150801461848EA030004FA03F0F3F74CFF0122A1F173
S31508014628F873013E129274E70123B5E70F90B4E7D0
S31508014638049BDB1B04937B420A9300230E93C1E771
S3150801464801230B93219B07EB030B0BF10103012BA9
S315080146580893B8BF012306E001230B93219B002B7E
S3150801466828DD9B46089300210422D9F81C0002F18B
S3150801467814059D4226D94160484601F093F88246B9
S31508014688002843D1024640F2AF111F4BD4E6002356
S31508014698E3E70023D5E7012400230B9420934FF081
S315080146A8FF3B00221223CDF820B02192DBE7012334
S315080146B80B93F4E74FF0010B5B46CDF820B0CDF824
S315080146C884B0D0E701315200D1E700BFAFF30080CB
S315080146D861436F63A787D23FB3C8608B288AC63FF1
S315080146E8FB799F501344D33F586C0108106D010894
S315080146F80000F07F0C6D0108356C0108346C01085F
S315080147080000F83F286E0108686D0108D9F81C30C1
S315080147181860089B0E2B00F2A180002C00F09E80E1
S31508014728002F33DD9C4B07F00F0203EBC203F80594
S31508014738D3E90034CDE910344FEA271416D5DDE953
S315080147480C01964B0326D3E90823F4F757F8CDE964
S31508014758060104F00F04914D54B9DDE91023DDE98A
S315080147680601F4F74BF8CDE9060128E00226F2E737
S31508014778E10708D5DDE91001D5E90023F3F714FFA8
S31508014788CDE91001013664100835E5E700F0AF8078
S31508014798DDE90C017C42804B04F00F0203EBC203EE
S315080147A8D3E90023F3F700FF02260023CDE9060122
S315080147B87A4D2411002C40F08F80002BD3D1DDE9E6
S315080147C806450F9B002B00F09480002220462946B7
S315080147D8734BF4F75BF9002800F08B80089B002BD4
S315080147E800F08780BBF1000F34DD204600222946F8
S315080147F86C4BF3F7D9FE5C46CDE9060107F1FF389C
S3150801480801363046F3F766FEDDE90623F3F7CCFEF3
S315080148180022654BF3F712FD0546A1F15076002CE7
S315080148286AD1DDE906010022604BF3F705FD024668
S315080148380B46CDE906232A463346F4F745F90028F7
S3150801484840F09882DDE906012A4606F10043F4F7A5
S315080148581DF938BBDDE90C34CDE90634159B002B67
S31508014868C0F257810E2F00F354814B4B03EBC70354
S31508014878D3E90034CDE90434219B002B80F2E58085
S31508014888089B002B00F3E1800CD1DDE90401002225
S31508014898464BF3F789FEDDE90623F4F70BF90028F9
S315080148A800F0668200242546219B56466FEA0308CE
S315080148B800272146484600F0B5FF002D00F0BD80C7
S315080148C82FB1AF4203D03946484600F0ABFF294617
S315080148D8484600F0A7FFB0E0E20705D5D5E9002369
S315080148E8F3F762FE012301366410083562E70226EA
S315080148F865E7B846089C84E7274B0B9903EBC4037D
S3150801490853E902235444002954D000202849F3F7CF
S3150801491875FF33462A46F3F78FFC5646CDE910014B
S31508014928DDE90601F4F7F0F80546F3F7D3FD024683
S315080149380B46DDE90601F3F77FFC02460B463035DF
S31508014948CDE90623DDE9102306F8015BF4F79EF89D
S31508014958002872D1DDE9062300201149F3F76CFC1A
S31508014968DDE91023F4F792F8002840F0B480A6424E
S315080149783FF470AFDDE9100100220A4BF3F714FE84
S315080149880022CDE91001DDE90601064BF3F70CFE15
S31508014998CDE90601C4E700BF286E0108006E0108C3
S315080149A80000F03F0000244000001C4000001440AD
S315080149B80000E03F31462846F3F7F6FD5646CDE9AD
S315080149C810011394DDE90601F4F79EF80546F3F795
S315080149D881FD02460B46DDE90601F3F72DFC024681
S315080149E80B46303506F8015BA642CDE906234FF09A
S315080149F8000224D1DDE91001AE4BF3F71FFC02468C
S31508014A080B46DDE90601F4F75FF8002863D1DDE90D
S31508014A1810230020A749F3F70FFC02460B46DDE9E8
S31508014A280601F4F733F800283FF414AF139E731EF2
S31508014A38139316F8013C302BF8D047463BE09E4BBA
S31508014A48F3F7B2FDCDE90601BCE75646DDE90645A9
S31508014A58DDE9042320462946F3F7D0FEF4F754F88E
S31508014A688046F3F737FDDDE90423F3F79DFD024692
S31508014A780B4620462946F3F7DFFB08F13004089D63
S31508014A8806F8014BA6EB0A04A54202460B4633D1A2
S31508014A98F3F7D4FBDDE9042304460D46F4F714F8C5
S31508014AA8C0B9DDE9042320462946F3F7E5FF10B125
S31508014AB818F0010F0ED14846039900F0B3FE0023FA
S31508014AC83370229B01371F60249B002B00F04B8211
S31508014AD81E6048E2B84633461E4613F8012D392AA0
S31508014AE806D19A45F8D1302208F101088AF800203A
S31508014AF81A7801321A70A0E700226F4BF3F754FDB2
S31508014B080022002304460D46F3F7B6FF00289FD076
S31508014B18D1E70B9A002A00F0EA80209A012A00F3C5
S31508014B28CD80129A002A00F0C18003F233430A9C09
S31508014B38049E049A01211A440492099A48461A4479
S31508014B48099200F023FF054666B1099B002B09DD8A
S31508014B58B342A8BF3346049AF61AD21A0492099A96
S31508014B68D31A09930A9B0BB30B9B002B00F0C6803B
S31508014B78002C00F0C08029462246484600F0BEFFB0
S31508014B88039A01460546484600F016FF03998046EA
S31508014B98484600F047FE0A9B1B1B0A9300F0B180A2
S31508014BA841460A9A484600F0A9FF0390012148465A
S31508014BB800F0ECFE0E9B0446002B00F0D8811A463D
S31508014BC80146484600F09AFF209B0446012B00F34C
S31508014BD89F80069B002B40F09780079BC3F313031E
S31508014BE8002B40F09380079B23F000431B0D1B0500
S31508014BF833B1049B01330493099B013309930123B8
S31508014C080A930E9B002B00F0B881236904EB8303F2
S31508014C18186900F06FFEC0F12000099B184410F0CE
S31508014C281F0000F08280C0F12003042B73DD049B6A
S31508014C38C0F11C0003440493099B064403440993E1
S31508014C48049B002B05DD1A464846039900F0B0FF78
S31508014C580390099B002B05DD21461A46484600F0B4
S31508014C68A7FF04460F9B002B61D02146039801F044
S31508014C780BF800285BDA00230A224846039900F054
S31508014C88F3FD0B9B07F1FF380390002B00F07781A2
S31508014C98294600230A22484600F0E6FDBBF1000F23
S31508014CA805466FDC209B022B49DC6BE0149BC3F19C
S31508014CB836033CE70000E03F00002440089B5C1EE1
S31508014CC80A9BA34209DB1C1B089B002BBFF630AFC6
S31508014CD8049B089A9E1A00232BE70A9B0E9AE31A45
S31508014CE81A440A94049E0024089B0E9221E70A9CFA
S31508014CF8049E0B9D28E7DDF80C8051E70A9A03996B
S31508014D0850E7CDF80C8051E7002379E7069B77E74A
S31508014D1800230A9379E793D0049A1C331A44049218
S31508014D28099A1E441A4409928AE70346F4E7089B36
S31508014D38B846002B20DC9B46209B022B1EDDBBF1C7
S31508014D48000F7FF4B1AD21465B460522484600F0BF
S31508014D588BFD01460446039800F096FF00287FF765
S31508014D68A3AD5646312308F1010806F8013B9FE52C
S31508014D78B846089C2546F4E7DDF820B00B9B002BBE
S31508014D8800F00181002E05DD29463246484600F025
S31508014D980FFF05460A9B002B5CD04846696800F058
S31508014DA801FD064628B9024640F2EF21804BFFF776
S31508014DB843BB2A6905F10C01023292000C30FFF750
S31508014DC871FA01223146484600F0F2FE2F46054699
S31508014DD80AF1010304930AEB0B030A93069B03F0F2
S31508014DE801030993049B2146039803F1FF3BFFF747
S31508014DF885FA034639463033069003980B9300F033
S31508014E0843FF2A4608902146484600F059FFC268DA
S31508014E1806460B9B02BB0146039800F035FF02467E
S31508014E280B9B31464846CDE90B3200F0FBFC209B2B
S31508014E380C9A049E42EA0301099B19430B9B0DD15F
S31508014E48392B27D0089A002A01DD069B31338BF8BE
S31508014E5800302EE52846B9E70122E2E70899002934
S31508014E6804DB209801430998014320D1002AEEDD85
S31508014E78012203994846049300F09AFE21460390B5
S31508014E8800F002FF0028049B02DCE0D1DA07DED530
S31508014E98392BDAD139238BF8003033461E4616F8F2
S31508014EA8012C013B392A4ED001321A7001E5002A34
S31508014EB803DD392BEED00133C9E7049A0A9902F8BA
S31508014EC8013C8A4228D000230A220399484600F061
S31508014ED8CBFCAF4203904FF000034FF00A02394664
S31508014EE8484607D100F0C0FC07460546049B01332E
S31508014EF8049377E700F0B8FC2946074600230A22F7
S31508014F08484600F0B1FC0546F0E7BBF1000FCCBFF7
S31508014F185E4601260027564401220399484604930A
S31508014F2800F046FE2146039000F0AEFE0028B4DCE8
S31508014F3802D1049BDB07B0D433461E4613F8012D6C
S31508014F48302AFAD0B5E49A45A8D1312308F10108DF
S31508014F588AF80030ADE4249BDFF858A01BB10AF1A2
S31508014F680803249A1360504617B0BDE8F08F209BB2
S31508014F78012B7FF72EAE0E9B0A9301204DE6BBF156
S31508014F88000F7FF7D9AE564621460398FFF7B6F9BB
S31508014F9800F1300306F8013BA6EB0A029345B4DD96
S31508014FA800230A224846039900F05EFC0390EBE7C2
S31508014FB8686D0108036D01082DE9F0471F468E68DB
S31508014FC88246BE420C4690460B682DD8B1F90C208C
S31508014FD812F4906F26D06569096905EB4505A3EBB7
S31508014FE8010905EBD5757B1C4B446D109D4238BFED
S31508014FF81D46530527D5294600F0A0FA064660B38B
S315080150084A462169FFF74EF9A38923F4906343F0C9
S315080150188003A38126614E4426603E466561A5EB59
S315080150280905A560BE4200D93E4632464146206872
S3150801503801F0ABF80020A3689B1BA36023683344DF
S315080150482360BDE8F0872A4600F07CFF064600285B
S31508015058E0D15046216901F047F90C23CAF8003016
S31508015068A3894FF0FF3043F04003A381E9E7000025
S315080150782DE9F04F98468B8907461B060D461446B7
S315080150889DB010D50B6973B9402100F057FA28600D
S31508015098286130B90C233B604FF0FF301DB0BDE8DD
S315080150A8F08F40236B610023099320238DF829305B
S315080150B830234FF00109CDF80C80DFF898818DF877
S315080150C82A3023469A4613F8012B0AB1252AF9D11B
S315080150D8BAEB040B0BD05B46224629463846FFF73E
S315080150E86BFF013000F0A780099A5A4409929AF889
S315080150F80030002B00F09F8000234FF0FF32CDE9E6
S3150801510805230AF1010A049307938DF853301A9374
S315080151185446052214F8011B4E48FFF7B5F8049AB8
S31508015128D8B9D00644BF20238DF85330110744BF98
S315080151382B238DF853309AF800302A2B15D054466C
S3150801514800204FF00A0C079A214611F8013B303B1B
S31508015158092B4BD9B0B1079214E0A0EB080309FA59
S3150801516803F31343A2460493D2E7039B191D1B684D
S315080151780391002BBBBF5B4242F0020207930793D8
S31508015188B8BF049223782E2B0AD163782A2B32D1F9
S31508015198039B02341A1D1B68039243EAE3730593BA
S315080151A8DFF8B4A0032250462178FFF76DF838B125
S315080151B84022049BA0EB0A0082401343013404935E
S315080151C814F8011B062225488DF82810FFF75CF804
S315080151D8002836D0224B1BBB039B073323F0070352
S315080151E808330393099B334409936AE70C4601205C
S315080151F80CFB0232A8E700234FF00A0C19460134C2
S315080152080593204610F8012B303A092A03D9002BB1
S31508015218C6D00591C4E7044601230CFB0121F0E732
S3150801522803AB00932A4638460E4B04A9FEF760FAE3
S31508015238421C0646D6D1AB895B063FF52DAF0998C0
S315080152482CE703AB00932A463846064B04A9FEF712
S31508015258EDFCEDE7796D01087F6D0108836D01089D
S31508015268F9360108C14F0108936810B4013B002BB0
S31508015278936007DA9469A34201DB0A2902D110BCB3
S3150801528800F08EBE1368581C10601970084610BCC9
S315080152987047F8B506460F461446D518AC4201D1EB
S315080152A8002007E03A46304614F8011BFFF7DCFFF1
S315080152B8431CF3D1F8BD00002DE9F04F0D461446FD
S315080152C8984606469DB018B1036A0BB9FEF758FE0B
S315080152D86B6ED90705D4AB899A0502D4A86DFEF772
S315080152E8CCFFAB891B0701D52B699BB929463046E3
S315080152F800F094FE70B16B6EDC0704D54FF0FF30F1
S315080153081DB0BDE8F08FAB899805F7D4A86DFEF7EF
S31508015318B5FFF3E70023099320238DF829303023B5
S315080153284FF00109CDF80C80DFF8A8818DF82A30ED
S3150801533823469A4613F8012B0AB1252AF9D1BAEB5D
S31508015348040B0BD05B46224629463046FFF7A1FFD8
S31508015358013000F0A780099A5A4409929AF8003050
S31508015368002B00F09F8000234FF0FF32CDE905237B
S315080153780AF1010A049307938DF853301A93544690
S31508015388052214F8011B5348FEF77EFF049AD8B97B
S31508015398D10644BF20238DF85330130744BF2B2366
S315080153A88DF853309AF800302A2B15D05446002028
S315080153B84FF00A0C079A214611F8013B303B092B95
S315080153C84BD9B0B1079214E0A0EB080309FA03F325
S315080153D81343A2460493D2E7039B191D1B6803913D
S315080153E8002BBBBF5B4242F0020207930793B8BF83
S315080153F8049223782E2B0AD163782A2B32D1039B60
S3150801540802341A1D1B68039243EAE3730593DFF80E
S31508015418C8A0032250462178FEF736FF38B1402244
S31508015428049BA0EB0A00824013430134049314F841
S31508015438011B062229488DF82810FEF725FF0028A2
S315080154483FD0274B1BBB039B073323F007030833BE
S315080154580393099B3B4409936AE70C4601200CFB15
S315080154680232A8E700234FF00A0C194601340593BE
S31508015478204610F8012B303A092A03D9002BC6D041
S315080154880591C4E7044601230CFB0121F0E703ABA8
S3150801549800932A463046134B04A9FEF729F907460D
S315080154A8781CD6D16B6ED90705D4AB899A0502D46F
S315080154B8A86DFEF7E3FEAB895B063FF51FAF0998B2
S315080154C81EE703AB00932A463046064B04A9FEF7A6
S315080154D8ADFBE4E7796D01087F6D0108836D010865
S315080154E8F93601089B520108024B0146186800F073
S315080154F825B800BF8400002070B50F4E0C463168E8
S31508015508054611B900F090FE30602146284600F09C
S315080155188BFE431C03D14FF0FF34204670BDC41CD3
S3150801552824F00304A042F8D0211A284600F07CFE8C
S315080155380130F2D1EFE700BFA40F00202DE9F843A7
S31508015548CD1C25F0030508350C2D38BF0C25002D73
S31508015558064601DBA94204D90C2333600020BDE8BD
S31508015568F883DFF8D48000F011F9D8F800301C4622
S3150801557844BB29463046FFF7BFFF431C044658D1AA
S31508015588D8F800402746002F43D1002C4BD0236872
S315080155983946304604EB030900F046FE814542D1F7
S315080155A8216830466D1A2946FFF7A6FF01303AD019
S315080155B823682B442360D8F800305A6862BBC8F8B8
S315080155C800700FE02268521B20D40B2A17D96119DB
S315080155D8A342256018BF5960636808BFC8F8001058
S315080155E862514B60304600F0D7F804F10B00231DD1
S315080155F820F00700C21A1CBF1B1AA350AFE762683E
S31508015608A3420CBFC8F800205A60EBE72346646832
S31508015618AEE73C467F68B6E71A465B68A342FBD104
S3150801562800235360DEE70C233046336000F0B4F8F4
S3150801563894E70560D6E700BFA80F0020B1F90C204A
S31508015648F8B5160705460C4654D44B68002B02DCF8
S315080156580B6C002B48DDE66A002E45D0002312F4B0
S3150801566880522F68216A2B6030D0626DA389590749
S3150801567805D56368D21A636B0BB1236CD21A00235A
S315080156882846E66A216AB047431CA38906D12968D0
S315080156981D292BD8284ACA40D60727D50022626071
S315080156A82269D904226004D5421C01D12B6803B9A1
S315080156B86065616B2F60B9B104F14403994202D060
S315080156C8284600F011FE002363630DE001232846EE
S315080156D8B0470246501CC9D12B68002BC6D01D2BD2
S315080156E801D0162B1DD12F60002021E043F040037D
S315080156F81BB21AE00F69002FF6D0930718BF0023CB
S315080157080E6808BF4B69F61B0F608B60002EEBDD30
S3150801571833463A462846216AD4F828C0E04700287D
S3150801572807DCB4F90C3043F040034FF0FF30A3818E
S31508015738F8BD0744361AE9E70100402038B50B6970
S3150801574805460C4613B90025284638BD18B1036A1B
S315080157580BB9FEF715FCB4F90C30002BF3D0626EC1
S31508015768D00704D4990502D4A06DFEF786FD28460C
S315080157782146FFF763FF636E0546DA07E4D4A38972
S315080157889B05E1D4A06DFEF779FDDDE70148FEF733
S3150801579874BD00BFA00F00200148FEF76FBD00BF0A
S315080157A8A00F002070B5C66904460D4676B91020C3
S315080157B8FFF79AFE0246E06120B96B21174B184894
S315080157C8FEF77EFDC0E901660660C660E669F3680C
S315080157D883B1E369DB6853F82500B8B9012101FAF1
S315080157E805F6721D2046920000F069FD60B1C0E910
S315080157F801560EE021220421204600F060FDE369E6
S31508015808F060DB68002BE4D1002070BD026843F81C
S3150801581825200023C0E90333F7E700BF586C0108C0
S315080158288A6D010870B5C66905460C4676B9102011
S31508015838FFF75AFE0246E86120B98F21084B094845
S31508015848FEF73EFDC0E901660660C6603CB1EB6934
S315080158586268DB6853F82210216043F8224070BD5C
S31508015868586C01088A6D01082DE9F04107460C466E
S315080158781E4600200D6901F1140CDCF800300130D0
S3150801588899B202FB01611E0C0B0C02FB063389B2A5
S3150801589801EB034185424FEA13464CF8041BECDC3D
S315080158A80EB3A368AB4219DC616838460131FFF7C4
S315080158B879FF804628B90246BA210C4B0C48FEF7EF
S315080158C8FFFC226904F10C01023292000C30FEF742
S315080158D8E9FC21463846FFF7A5FF444604EB85034C
S315080158E801355E6125612046BDE8F081686D0108CC
S315080158F88A6D01080346B0F5803F3ABF03041020B4
S315080159080020B3F1807F3CBF1B020830B3F1805FEA
S315080159183CBF1B010430B3F1804F3CBF9B000230EA
S31508015928002B05DB13F0804F00F1010008BF20208A
S3150801593870470368024613F007000BD0D90721D42C
S31508015948980749BF5B089B08012013605CBF0220C2
S315080159581360704799B209B910201B0CD9B209B955
S3150801596808301B0A190704BF1B090430990704BF25
S315080159789B080230D90703D45B0800F1010003D05C
S3150801598813607047002070472020704710B50C46F1
S315080159980121FFF707FF024628B940F24511044BD2
S315080159A80448FEF78DFC01234461036110BD00BF5D
S315080159B8686D01088A6D01082DE9F04F17460A69CD
S315080159C83B6989469A42A2BF3B460F4699463D69B5
S315080159D8D9F810A0BB68796805EB0A06B34285B001
S315080159E8B8BF0131FFF7DEFE30B902464FF4B1718F
S315080159F8404B4148FEF764FC00F114042346002293
S31508015A0804EB860E734520D307F1140809F114012E
S31508015A1808EB850501EB8A030293EB1B153B23F07B
S31508015A28030304331537BD4238BF04230193029B88
S31508015A3803918B420CD8002E03DD5EF8043D002B3A
S31508015A4855D0066105B0BDE8F08F43F8042BD9E7B0
S31508015A58B1F800A0BAF1000F1FD0C446A146002725
S31508015A685CF8042BD9F800301FFA82FB9BB20AFBB3
S31508015A780B333B44D9F80070120C3F0C0AFB02722F
S31508015A8802EB13429BB243EA024365454FEA1247C2
S31508015A9849F8043BE4D8019BE750039B0431B3F862
S31508015AA80290B9F1000F20D04746A4464FF0000AE4
S31508015AB82368B7F800B0BCF802209BB209FB0B2291
S31508015AC8524443EA02434CF8043B57F8043B4FEA6D
S31508015AD8134ABCF80030BD4209FB0A3303EB1243EB
S31508015AE84FEA134AE5D8019AA35004349FE7013EC1
S31508015AF8A1E700BF686D01088A6D01082DE9F84319
S31508015B08154612F0030207460E4607D0254C013AF8
S31508015B18002354F82220FFF7A7FE0646AD103DD00C
S31508015B28FC697CB91020FFF7DFFC0246F86128B941
S31508015B3840F2B3111C4B1D48FEF7C2FBC0E90144EC
S31508015B480460C460D7F81C80D8F808404CB940F2FC
S31508015B5871213846FFF71AFF00230446C8F80800DA
S31508015B6803604FF00009EB070AD531462246384645
S31508015B78FFF722FF804631463846FFF753FE464669
S31508015B886D100BD0206838B9224621463846FFF7EA
S31508015B9813FF2060C0F800900446E4E73046BDE8E4
S31508015BA8F88300BFF06D0108586C01088A6D010871
S31508015BB82DE9F0470C46074691462369496803EBE0
S31508015BC86218A3684FEA621A08F10106B3420BDBA9
S31508015BD83846FFF7E7FD054648B902464FF4EF711F
S31508015BE8274B2848FEF76CFB01315B00EEE70023DB
S31508015BF800F1140100F110021846534533DB2069F8
S31508015C082AEAEA7A04F1140319F01F0901EB8A0151
S31508015C1803EB800C2BD08A460022C9F1200E18689E
S31508015C2800FA09F010434AF8040B53F8042B9C456B
S31508015C3822FA0EF2F3D8ACEB0403153B23F003035F
S31508015C48043304F11500604588BF0423CA500AB114
S31508015C5808F10206013E384621462E61FFF7E2FDA4
S31508015C682846BDE8F08742F8040F0133C5E7043929
S31508015C7853F8042B9C4541F8042FF9D8EAE700BFE5
S31508015C88686D01088A6D010803460A69006930B515
S31508015C98801A0ED11433143103EB820401EB820105
S31508015CA854F8045D51F8042D954203D005D24FF0F6
S31508015CB8FF3030BDA342F3D3FBE70120F9E7000023
S31508015CC82DE9F74F89460646114648461446FFF711
S31508015CD8DBFF051E12D129463046FFF763FD02464A
S31508015CE828B940F237213E4B3E48FEF7E9FA012327
S31508015CF8C0E90435104603B0BDE8F08FBCBF4B4672
S31508015D08A1463046D9F80410BABF1C460125002514
S31508015D18FFF748FD024618B940F24521304BE3E73B
S31508015D2800F1140BD9F8107009F11003C5604FF08A
S31508015D38000C09F11405D946266904F1140E05EB78
S31508015D4887080EEB86060193019B5EF8040B53F848
S31508015D5804AF81B201931FFA8AF35B1A000C6344F4
S31508015D68C0EB1A4000EB23409BB243EA0043764551
S31508015D784FEA204C49F8043BE6D8331B153B23F078
S31508015D88030315340433A64238BF04231D445B4470
S31508015D981E462C4644450ED308F10301491B21F03A
S31508015DA80301033DA84538BF00210B4453F8041DD8
S31508015DB899B117619EE7E64654F8041B1FFA81FC58
S31508015DC8F444080C714400EB2C4089B241EA0041BD
S31508015DD84FEA204C46F8041BDCE7013FE6E700BF1B
S31508015DE8686D01088A6D01082DE9734301219046FA
S31508015DF89946089EFFF7D6FC044630B9024640F292
S31508015E080F31234B2348FEF75BFAC9F30A55C9F341
S31508015E1813030DB143F480130193B8F1000324D099
S31508015E2868460093FFF785FDDDE90012D8B1C0F190
S31508015E38200302FA03F30B43C24063610192019BF3
S31508015E48002B0CBF01220222A3612261ADB1A5F282
S31508015E58334505443560C0F13500099B186020466D
S31508015E6802B0BDE870836161E9E701A8FFF761FD42
S31508015E78019B012263612030E7E7A0F2324004EB77
S31508015E88820330601869FFF735FDC0EB4210E4E775
S31508015E98686D01088A6D010810B50C46B1F90E102E
S31508015EA800F0B0F90028ABBF636DA3891B1823F46A
S31508015EB88053ACBF6365A38110BD2DE9F0411F4628
S31508015EC88B890546DB050C46164605D502230022AD
S31508015ED8B1F90E1000F084F9A389324623F48053E8
S31508015EE8A38128463B46B4F90E10BDE8F04100F0F7
S31508015EF8ABB910B50C46B1F90E1000F071F9431C8F
S31508015F08A38915BF606523F4805343F48053A3819D
S31508015F1818BFA38110BDB1F90E1000F0A7B900008A
S31508015F280EB403B5014603AB054853F8042B0068BC
S31508015F380193FFF7C1F902B05DF804EB03B07047A6
S31508015F48840000202DE9F041074614460D4621B97B
S31508015F581146BDE8F041FFF7F1BA2AB900F0C4F9CC
S31508015F6825462846BDE8F08100F018FA8442064617
S31508015F7802D8B4EB500FF4D821463846FFF7DEFAB3
S31508015F88804608B94546ECE7B4422246294628BF61
S31508015F983246FEF787F92946384600F0A5F9F1E7AA
S31508015FA8F8B50E461446054618B1036A0BB9FDF746
S31508015FB8E7FFA369A360A3891A0701D5236943B92A
S31508015FC82146284600F02AF818B14FF0FF37384617
S31508015FD8F8BD23682269F6B2981A63693746834277
S31508015FE805DC21462846FFF7A9FB0028EDD1A36859
S31508015FF8013BA36023685A1C22601E706269431C10
S315080160089A4204D0A389DB07E1D50A2EDFD12146B6
S315080160182846FFF793FB0028D9D0D6E738B5294B88
S31508016028054618680C4618B1036A0BB9FDF7A8FFA7
S31508016038B4F90C30190722D4DA0607D409222A60DA
S3150801604843F040034FF0FF30A38133E0580712D5D8
S31508016058616B41B104F14403994202D0284600F024
S3150801606843F900236363A38923F02403A381002347
S31508016078636023692360A38943F00803A38123691D
S315080160884BB9A38903F42073B3F5007F03D02146DE
S31508016098284600F03EF8B4F90C3013F001020AD08C
S315080160A80022A26062695242A261226942B913F0CA
S315080160B88000C5D138BD990758BF6269A260F4E75F
S315080160C80020F7E78400002070B50C46B1F90E10D8
S315080160D8154600291E4696B00CDAA389002113F045
S315080160E8800F14BF40234FF48063002031602B6072
S315080160F816B070BD6A4600F0C9F80028EDDB0199AB
S3150801610801F47041A1F50053594259414FF480638E
S31508016118EBE78B89F7B59D0706460C4607D504F1C3
S315080161284703236023610123636103B0F0BD6A460F
S3150801613801ABFFF7C9FF009F054639463046FFF709
S31508016148FDF948B9B4F90C309A05EED423F00303DE
S3150801615843F00203A381E2E7A389C4E9040743F0EC
S315080161688003A381019B20605BB13046B4F90E1008
S3150801617800F026F828B1A38923F0030343F00103A5
S31508016188A381A3891D43A581CFE7884210B501EBF1
S31508016198020402D98442234607D8431EA14208D0DD
S315080161A811F8012B03F8012FF8E7014602448A4240
S315080161B800D110BD13F8014D02F8014DF7E70000AB
S315080161C838B50023054D044608462B60F7F74FFFF7
S315080161D8431C02D12B6803B1236038BDAC0F0020DC
S315080161E838B50446084611460022054D2A601A465E
S315080161F8F7F747FF431C02D12B6803B1236038BD63
S31508016208AC0F002038B50446084611460022054D4C
S315080162182A601A46F7F7F4FE431C02D12B6803B124
S31508016228236038BDAC0F002038B50023054D044658
S3150801623808462B60F7F732FF431C02D12B6803B1D6
S31508016248236038BDAC0F002038B504460846114608
S315080162580022054D2A601A46F5F71AF8431C02D199
S315080162682B6803B1236038BDAC0F002038B500236D
S31508016278054D044608462B60F7F7DFFE431C02D195
S315080162882B6803B1236038BDAC0F002038B500234D
S31508016298064D0446084611462B60F7F7D9FE431CF6
S315080162A802D12B6803B1236038BD00BFAC0F0020AB
S315080162B8062008B500F0B0F80120F7F796FE70B584
S315080162C8A1FB025434B92946FFF738F9064628B915
S315080162D8304670BD0C2200260260F9E72A46214697
S315080162E8FDF7D2FEF4E7000038B50546002940D087
S315080162F851F8043C0C1F002BB8BFE418FFF746FAFF
S315080163081C4A136833B9636014602846BDE83840E7
S31508016318FFF742BAA34208D9206821188B4201BF60
S3150801632819685B6809182160EDE71A465B680BB1BD
S31508016338A342FAD911685018A0420BD12068014422
S31508016348501883421160E0D118685B6808441060E8
S315080163585360DAE702D90C232B60D6E7206821189F
S315080163688B4201BF19685B6809182160636054602C
S31508016378CBE738BDA80F002082B001B901A942B1FF
S315080163884BB113780B601278101E18BF012002B0A2
S3150801639870471046FBE76FF00100F8E751F8043C2F
S315080163A8181F002BBCBF0B58C01870470346084670
S315080163B841B1FF2A04D98A224FF0FF301A60704783
S315080163C801200A7070471F2938B505460C4604D9B5
S315080163D8162303604FF0FF3038BDC26B12B152F86D
S315080163E821304BB9284600F031F82246014628469D
S315080163F8BDE8384000F018B8012B0AD0591C03D15A
S31508016408162303600120E7E70021204642F82410F5
S3150801641898470020E0E70000024B01461868FFF795
S31508016428D2BF00BF8400002038B50023064D0446B4
S31508016438084611462B60F7F7C8FD431C02D12B689D
S3150801644803B1236038BD00BFAC0F0020F7F7B6BD0E
S31508016458F8B500BFF8BC08BC9E467047F8B500BF3A
S30D08016468F8BC08BC9E4670470A
S31508016470434F4E4E2564204572726F723A20256449
S315080164800A000000434F4E4E256420436861726737
S31508016490696E672046696E69736865643A0A000021
S315080164A04368617267696E6720456E657267793AF6
S315080164B02025640A0000000042484D2054696D6594
S315080164C06F75740A000000005053552072656164A7
S315080164D0792074696D656F75742C2073746F70708B
S315080164E0696E672E2E2E0A00505355206F6E207442
S315080164F0696D656F75742C2073746F7070696E673A
S315080165002E2E2E0A00000000505355206F66662075
S3150801651074696D656F75742C2073746F7070696E0C
S31508016520672E2E2E0A000000455620696E666F3AC0
S315080165300A0000004742545F766572205625642E8C
S31508016540256425640A000000426174746572792025
S31508016550747970653A2025640A00000042617474F2
S315080165606572792063617061636974793A2025647B
S315080165700A0000004261747465727920766F6C7442
S315080165806167653A2025640A000000004261747457
S315080165906572792076656E646F723A20252E34739A
S315080165A00A0000004261747465727920534E3A20DC
S315080165B0256C750A000000004261747465727920C1
S315080165C06D616E7566616374757265206461746563
S315080165D03A20253032642E253032642E2530346433
S315080165E00A00000042617474657279206379636CEC
S315080165F065733A2025640A004F776E206175746FBA
S315080166003A2025640A0000004556494E3A20252EAF
S315080166103137730A0000000045565F53575F5645E8
S31508016620523A20252E38730A0000000042524D20A6
S3150801663054696D656F75740A0000000042617474CF
S3150801664065727920696E666F3A0A00006D61784352
S3150801665056202564560A00006D6178434320256457
S31508016660410A0000746F74452025646B57680A0057
S315080166706D617854202564430A000000534F432076
S315080166802564700A00000000566F6C742E2025647C
S31508016690560A00004243502054696D656F75740AA5
S315080166A00000000042524F2054696D656F75740AE7
S315080166B0000000004556206E6F742072656164798A
S315080166C020666F722061203630730A0050535520B8
S315080166D06E6F742072656164792C2073746F7070A3
S315080166E0696E672E2E2E0A0042434C2F4243532FC2
S315080166F042534D2074696D656F75742C2073746FE0
S315080167007070696E672E2E2E0A0000004C6F636B3F
S31508016710206572726F722C2073746F7070696E6760
S315080167202E2E2E0A00000000486F74706C756720C3
S3150801673064657465637465642C2073746F7070691D
S315080167406E672E2E2E0A0000436F6E6E6563746F98
S3150801675072206F76657268656174202564202564E8
S315080167602C2073746F7070696E672E2E2E0A0000C6
S315080167704253442054696D656F75740A0000000020
S3150801678044697361626C65640A000000436861725A
S3150801679067696E6720737461727465640A00000024
S315080167A057616974696E6720666F722042484D0A9F
S315080167B00000000057616974696E6720666F722070
S315080167C05053552072656164790A000049736F6CEC
S315080167D06174696F6E20746573740A005761697410
S315080167E0696E6720666F72206261747465727920BA
S315080167F0696E666F0A00000057616974696E6720E1
S31508016800666F72206261747465727920737461743B
S3150801681075730A0057616974696E6720666F72201D
S31508016820424D530A00000000496E697469616C693A
S315080168307A696E6720636861726765720A0000008B
S3150801684057616974696E6720666F722042434C0A04
S31508016850000000004368617267696E6720696E20EF
S3150801686070726F67726573730A000000436861721C
S3150801687067696E672053746F707065640A0000005B
S315080168804368617267696E672053746F70706564D7
S315080168902077697468204353440A0000436861728B
S315080168A067696E67204572726F720A004368617282
S315080168B067696E672046696E69736865640A0000D0
S315080168C0474254204572726F7220636F64653A209D
S315080168D0307825580A000000436F6E6E6563746F41
S315080168E0723A20556E6B6E6F776E0A00436F6E6E45
S315080168F06563746F723A20556E706C756767656467
S315080169000A000000436F6E6E6563746F723A204425
S31508016910697361626C65640A00000000436F6E6EFC
S315080169206563746F723A20507265706172696E6739
S315080169300A000000436F6E6E6563746F723A2041F8
S3150801694075746852657175697265640A000000009C
S31508016950436F6E6E6563746F723A20576169746925
S315080169606E67466F72456E657267790A00000000A8
S31508016970436F6E6E6563746F723A2043686172671E
S31508016980696E6750617573656445560A00000000B3
S31508016990436F6E6E6563746F723A204368617267FE
S315080169A0696E67506175736564455653450A0000FB
S315080169B0436F6E6E6563746F723A204368617267DE
S315080169C0696E670A00000000436F6E6E6563746F37
S315080169D0723A204175746854696D656F75740A0059
S315080169E0436F6E6E6563746F723A2046696E69739A
S315080169F06865640A00000000436F6E6E6563746F14
S31508016A00723A2046696E6973686564455653450A44
S31508016A1000000000436F6E6E6563746F723A20461C
S31508016A20696E697368656445560A0000436F6E6E40
S31508016A306563746F723A205265706C756767696E23
S31508016A40670A000042454D205265636569766564AB
S31508016A502C20666F7263652073746F7070696E6738
S31508016A602E2E2E0A0000000042454D3A20253032CE
S31508016A7058202530325820253032582025303258B2
S31508016A8000000000202530325820253032582025B4
S31508016A9030325820253032580A000000425354201B
S31508016AA052656365697665642C2073746F707069C5
S31508016AB06E672E2E2E0A00004253543A2025303294
S31508016AC05820253032582025303258202530325862
S31508016AD0000000004C6F636B206572726F720A00CA
S31508016AE04C6F636B206572726F7220726573657481
S31508016AF00A000000474254204368617267657220A4
S31508016B007625642E25640A0053657269616C206EC8
S31508016B10756D6265723A2025640A0000426F6172DA
S31508016B2064207265766973696F6E3A2025640A0076
S31508016B3046572076657273696F6E3A2025642E254D
S31508016B40642E25640A000000505355206F6E207488
S31508016B50696D656F75740A00436F6E746163746F4E
S31508016B6072206572726F722C2073746F7070696E01
S31508016B70672E2E2E0A000000505355206F66662098
S31508016B8074696D656F75740A000000005365742099
S31508016B90436F6E6669673A2025732025640A0000EB
S31508016BA0506F776572206C696D69743A2025640A9D
S31508016BB000000000436861726765207065726D693F
S31508016BC0743A2025640A0005E093040000000000D9
S31508016BD0000000000102030406070809000000007E
S31508016BE00102030400000405060708090000000065
S31508016BF0000D00000102030405060708090A0B0C2B
S31508016C000D0E0F1000000405060708090000000014
S31508016C10000D00000102030405060708090A0B0C0A
S31508016C200D0E0F10494E4600696E66004E414E0024
S31508016C306E616E00300030313233343536373839CB
S31508016C4041424344454600303132333435363738CC
S31508016C5039616263646566005245454E54206D612B
S31508016C606C6C6F6320737563636565646564002F77
S31508016C706275696C642F676E752D746F6F6C732DF1
S31508016C80666F722D73746D33325F31332E332E7204
S31508016C90656C312E32303234303932362D31373156
S31508016CA0352F7372632F6E65776C69622F6E657700
S31508016CB06C69622F6C6962632F74696D652F676DE4
S31508016CC074696D652E63002C2066756E6374696F31
S31508016CD06E3A2000617373657274696F6E2022259E
S31508016CE07322206661696C65643A2066696C652061
S31508016CF0222573222C206C696E652025642573254F
S31508016D00730A00496E66696E697479004E614E00B0
S31508016D102F6275696C642F676E752D746F6F6C734E
S31508016D202D666F722D73746D33325F31332E332EA8
S31508016D3072656C312E32303234303932362D313774
S31508016D4031352F7372632F6E65776C69622F6E65A5
S31508016D50776C69622F6C6962632F7374646C6962FC
S31508016D602F64746F612E630042616C6C6F632073CC
S31508016D70756363656564656400232D302B2000689F
S31508016D806C4C00656667454647002F6275696C64F9
S31508016D902F676E752D746F6F6C732D666F722D73F9
S31508016DA0746D33325F31332E332E72656C312E3268
S31508016DB0303234303932362D313731352F737263EB
S31508016DC02F6E65776C69622F6E65776C69622F6CB9
S31508016DD06962632F7374646C69622F6D707265637F
S31508016DE02E63004300504F534958002E00000000FF
S31508016DF005000000190000007D00000000000000E9
S31508016E000080E03779C34143176E05B5B5B8934697
S31508016E10F5F93FE9034F384D321D30F94877825A63
S31508016E203CBF737FDD4F1575000000000000F03F81
S31508016E300000000000002440000000000000594046
S31508016E400000000000408F40000000000088C34099
S31508016E5000000000006AF8400000000080842E410E
S31508016E6000000000D01263410000000084D797415A
S31508016E700000000065CDCD41000000205FA0024260
S31508016E80000000E876483742000000A2941A6D42D5
S31508016E90000040E59C30A2420000901EC4BCD642C8
S31508016EA000003426F56B0C430080E03779C3414373
S31508016EB000A0D8855734764300C84E676DC1AB43E9
S31508016EC0003D9160E458E143408CB5781DAF154407
S31508016ED050EFE2D6E41A4B4492D54D06CFF08044E2
S31508016EE0F64AE1C7022DB544B49DD9794378EA44F7
S31508016EF0002020202020202020202828282828207B
S31508016F002020202020202020202020202020202072
S31508016F1020881010101010101010101010101010DA
S31508016F2010040404040404040404041010101010CA
S31508016F301010414141414141010101010101010194
S31508016F4001010101010101010101010110101010E6
S31508016F501010424242424242020202020202020266
S31508016F6002020202020202020202020210101010BA
S31508016F7020000000000000000000000000000000E2
S31508016F8000000000000000000000000000000000F2
S31508016F9000000000000000000000000000000000E2
S31508016FA000000000000000000000000000000000D2
S31508016FB000000000000000000000000000000000C2
S31508016FC000000000000000000000000000000000B2
S31508016FD000000000000000000000000000000000A2
S31508016FE00000000000000000000000000000000092
S30908016FF0000000008E
S30D08016FF43412FF7F01000000C1
S30908016FFC0D820008EB
S30908017000E98100080B
S31508017004E4010000010164000000FF000000000023
S315080170140000000000000000400000320A3200406F
S3150801702400000000008000320A32000080000000DF
S315080170340000FA320A32000000FA000000FF0032AA
S315080170440A32000020000000FFFFFF320A3200FF67
S31508017054FFFF0000FF0000320A3200200000000092
S3150801706452555301000000FE529E66000024F400A6
S3150801707410000000010000000000000003000000E9
S31508017084640E00208800002000000000640E002021
S31508017094CC0E0020340F0020000000000000000080
S315080170A400000000000000000000000000000000CD
S315080170B400000000000000000000000000000000BD
S315080170C400000000000000000000000000000000AD
S315080170D4000000004300000000000000000000005A
S315080170E4000000000000000000000000000000008D
S315080170F4000000004300000000000000000000003A
S31508017104000000000000000000000000000000006C
S315080171140000000043000000000000000000000019
S31508017124000000000000000000000000000000004C
S3150801713400000000430000000000000000000000F9
S31508017144000000000000000000000000000000002C
S3150801715400000000430000000000000000000000D9
S31508017164000000000000000000000000000000000C
S3150801717400000000430000000000000000000000B9
S3150801718400000000000000000000000000000000EC
S315080171940000000043000000000000000000000099
S315080171A400000000000000000000000000000000CC
S315080171B400000000B56301088163010800000000AE
S315080171C4F06E0108EB6D0108026D0108026D0108F4
S315080171D4026D0108026D0108026D0108026D0108BC
S315080171E4026D0108026D0108026D0108FFFFFFFF28
S315080171F4FFFFFFFFFFFFFFFFFFFF000001004153F1
S315080172044349490000000000000000000000000096
S3150801721400000000000000000000000000004153C7
S315080172244349490000000000000000000000000076
S31508017234000000000000000000000000000000003B
S7050800E6CD3F
